:100000000C94EC0E0C941D0F0C941D0F0C941D0FF2
:100010000C941D0F0C941D0F0C941D0F0C941D0FB0
:100020000C941D0F0C941D0F0C941D0F0C941D0FA0
:100030000C941D0F0C94E2710C941D0F0C941D0F69
:100040000C941D0F0C941D0F0C941D0F0C941D0F80
:100050000C941D0F0C941D0F0C941D0F0C94476EE7
:100060000C941D0F0C9404D30C94DAD20C941D0F35
:100070000C941D0F0C941D0F0C941D0F0C941D0F50
:100080000C941D0F0C941D0F0C941D0F0C941D0F40
:100090000C94B0D20C9486D20C941D0F0C946D73FA
:1000A0000C941D0F0C941D0F0C941D0F0C941D0F20
:1000B0000C941D0F0C941D0F0C941D0F0C941D0F10
:1000C0000C941D0F0C941D0F0C941D0F0C945CD2FE
:1000D0000C9432D20C941D0F0C9408D20C94DED1E7
:1000E0000C941D0F084AD73B3BCE016E84BCBFFD6C
:1000F000C12F3D6C74319ABD56833DDA3D00C77FF8
:1001000011BED9E4BB4C3E916BAAAABE0000008090
:100110003F07634236B79BD8A71A39685618AEBA5C
:10012000AB558C1D3CB7CC5763BD6DEDFD753EF6F0
:10013000177231BF000000803F08000000BE92240B
:1001400049123EABAAAA2ABECDCCCC4C3E00000040
:1001500080BEABAAAAAA3E00000000BF000000803B
:100160003F0000000000084178D3BB4387D1133D16
:10017000190E3CC3BD4282AD2B3E68EC8276BED9DF
:100180008FE1A93E4C80EFFFBE01C4FF7F3F00001E
:10019000000000000C94C26B0C9412590C94C7AA76
:1001A0000C9414610C942F610C94FFAA0C94585970
:1001B0000C946F510C94756C0C949B4D0C94455F92
:1001C0000C945A510C94144D0C94246C0C94356C72
:1001D0000C94FF4C0C940E5E0C94DA6B0C94A76B91
:1001E0000C94404D0C94EBAA0C94CF5F0C94E1AAB4
:1001F0000C9466510C9416590C9469510C9411543A
:100200000C94256C0C94BDAC0C9445510C94B06BC3
:100210000C946C510C94795E0C94E25C0C94486CD8
:100220000C94D2550C94BC6D0C94D66B0C946461F8
:100230000C944B6D0C94AD570C94936E0C94196107
:100240000C94C6740C9460510C940F610C94BE6BAA
:100250000C94A9580C94D06B0C94C86B0C94BA6B8A
:100260000C94236C0C943F4E0C943B520C94956B65
:100270000C94924D0C94494D0C94E7D40C945D5120
:100280000C94C75F0C94FD580C94F56B0C9470ACF7
:100290000C94264D0C945C610C94095B0C94634E99
:1002A0000C94C65C0C94A36B0C9485560C94CE6095
:1002B0000C94A76C0C94D0510C949F6B0C941D4D16
:1002C0000C94D5AA0C94FF610C94484E0C94A44D48
:1002D0000C94B3AA0C94C1520C94266C0C94CC6B65
:1002E0000C94D56B0C945DAA0C94784D0C94B46B63
:1002F0000C94A46C0C94684C0C945A4E0C940A54B4
:100300000C94AA6B0C949B6B0C94426B0C945EAA9D
:100310000C945C590C94A4AA0C94514E0C94EDD5F9
:100320000C947C6D0C94F5AA0C94B2570C942F4D40
:100330000C9463510C94894D4E414E494E49545989
:10034000494E46CDCCCC3D0AD7233C17B7D13877A0
:10035000CC2B329595E6241FB14F0A0000204100B6
:1003600000C84200401C4620BCBE4CCA1B0E5AAE00
:10037000C59D7400407A10F35A00A0724E1809000F
:1003800010A5D4E80000E87648170000E40B5402FA
:100390000000CA9A3B000000E1F505000080969835
:1003A00000000040420F000000A086010000001085
:1003B0002700000000E803000000006400000000C7
:1003C000000A00000000000100000000002C76D8A8
:1003D00088DC674F0823DFC1DFAE59E1B1B796E58E
:1003E000E3E453C63AE651997696E8E6C28426EBF2
:1003F000898C9B62ED407C6FFCEFBC9C9F40F2BA05
:10040000A56FA5F490055A2AF75C936B6CF9676D9C
:10041000C11BFCE0E40D47FEF520E6B500D0ED90F1
:100420002E0300943577050080841E080000204EBE
:100430000A000000C80C333333330F986E12831157
:1004400041EF8D2114893BE65516CFFEE6DB18D12E
:10045000844B381BF77C1D901DA4BBE42420328400
:10046000725E228100C9F124ECA1E53D27236E6F65
:10047000206D61676E657469632073656E736F725A
:1004800021004D4D43353838334D413D2000482D36
:100490006669656C643A20280020202020202020F6
:1004A000202020202020202020002020202020206C
:1004B000202020202020202020200020202020205C
:1004C000202020202020202020202000202020204C
:1004D000202020202020202020202020002020203C
:1004E000202020202020202020202020002020202C
:1004F0002020202020202020202020200044233ADB
:1005000043616C6962726174696F6E00442A3A5388
:10051000657474696E67730044423A52657365741A
:10052000204C6F676765720044433A436C656172A3
:10053000204C43440043303A416D6D6F6E69610059
:1005400043393A4E6974726174650043383A466FB4
:100550007263652F4D6173730043373A436F6E6466
:1005600075637469766974790043363A44697373C4
:100570006F6C766564204F320043312D353A536CF1
:100580006F74312D35204F6E0044443A4D756C74B4
:100590006953656E736F72730044393A43757272B2
:1005A000656E7400566F6C746167652B437572726B
:1005B000656E740044383A456C6563747269630013
:1005C00044373A4D6F74696F6E0044363A44532095
:1005D00054656D700044353A555620496E74656E09
:1005E000736974790044343A4F3220636F6E632E1E
:1005F0000044333A434F3220636F6E632E0044321F
:100600003A504D28313A322E353A313029004432B1
:100610003A504D28313A322E353A3130292A0044A9
:10062000313A5475726269646974790044303A569B
:100630006F6C7461676500393A6F722033442061D2
:100640006363656C2E00393A496E636C2E20616ECF
:10065000672E00383A70482076616C756500373A2D
:1006600049522054656D7000373A49522054656DE7
:10067000702A00363A4D61676E6574696320666959
:10068000656C6400353A476173204C6576656C0093
:10069000343A495220466C616D6500333A4C6967C3
:1006A000687420496E742E00323A616E6420486589
:1006B0006967687400323A54656D702050726573D2
:1006C0007375726500313A54656D702048756D69B7
:1006D0006469747900303A536F756E64204C6576A6
:1006E000656C00303A536F756E64204C6576656CAE
:1006F0002A0054696D65206C617073653A00576912
:1007000046692049503A00436F6E74726F6C002343
:10071000507265737320442320746F20656E61628C
:100720006C652000536C6F74230050686F6E6520F9
:1007300053656E736F7200416363656C65726174BB
:10074000696F6E004F7269656E742E2F496E636C0F
:100750002E00416E672E2056656C6F6369747900B8
:10076000436F6D702E202620482D6669656C6400ED
:100770004750530050726F78696D697479004C6905
:1007800067687420496E74656E7369747900416995
:10079000722050726573737572650054656D7020B8
:1007A000262048756D6964697479004D6F74696FAE
:1007B0006E00555620496E742E00555620496E74B1
:1007C000656E73697479004F3220436F6E63004326
:1007D0004F3220436F6E630053656E736F722065F6
:1007E00072726F722100234E6F2073656E736F7289
:1007F0002100434F3220436F6E63004D6561737576
:1008000072696E6700234E6F2054422073656E73C9
:100810006F723F00234E6F2073656E736F722100FD
:10082000536F756E64204C6576656C004D65617321
:100830007572696E672E2E00234E6F2073656E737E
:100840006F722100536F756E64204C6576656C0085
:10085000234E6F2073656E736F7220666F72207403
:10086000656D7020262068756D6964697479210052
:100870004E6F2053656E736F72210020666F722079
:1008800074656D7020262068756D696469747921BE
:10089000002353656E736F72204572726F72200071
:1008A00053656E736F72204572726F722100235709
:1008B000726F6E672073656E736F7220666F722041
:1008C00074656D7020262068756D6964697479217E
:1008D0000057726F6E672053656E736F72210054FC
:1008E000656D702048756D6964697479004C69673D
:1008F000687420496E74656E7369747900466C6122
:100900006D6520495200482D6669656C6400536529
:100910006172636820446972656374696F6E002355
:100920004E6F2070482073656E736F72210070489F
:100930002076616C75650023496E76616C69642070
:100940006B65792100204D756C746973656E736FEA
:100950007273004D756C746973656E736F7273009A
:1009600044697361626C6500456E61626C6500523A
:1009700065626F6F74696E672E2E2E002344413AB4
:100980002D323300237265706C6965733D006765B5
:100990007453656C665465737442697428293A20EF
:1009A000006973496E74657272757074456E616228
:1009B0006C65642831293A2000676574496E746556
:1009C00072727570744D617070696E672831293A62
:1009D0002000676574496E74657272757074536F28
:1009E000757263652831293A2000676574496E7411
:1009F000657272757074536F7572636528293A2039
:100A0000006765745261746528293A20332E3134A9
:100A10003135393F00616363656C2E69734C6F77C4
:100A2000506F77657228293A2000616363656C2EE8
:100A3000697341736C65657028293A2000616363AE
:100A4000656C2E6973546170536F757263654F6E78
:100A50005A28293A2000616363656C2E69735461DA
:100A600070536F757263654F6E5928293A20006183
:100A70006363656C2E6973546170536F757263653F
:100A80004F6E5828293A2000616363656C2E6973A4
:100A90004163746976697479536F757263654F6EDB
:100AA0005A28293A2000616363656C2E697341639B
:100AB000746976697479536F757263654F6E5928DE
:100AC000293A200069734163746976697479536FB8
:100AD000757263654F6E5828293A20006973546116
:100AE00070446574656374696F6E4F6E5A28293B54
:100AF0002066616C73653F200069735461704465C2
:100B000074656374696F6E4F6E5A28293B20747246
:100B100075653F2000697354617044657465637442
:100B2000696F6E4F6E5928293B2066616C73653F73
:100B300020006973546170446574656374696F6EF5
:100B40004F6E5928293B20747275653F20006973E8
:100B5000546170446574656374696F6E4F6E582894
:100B6000293B2066616C73653F2000697354617096
:100B7000446574656374696F6E4F6E5828293B2015
:100B8000747275653F200067657453757070726587
:100B9000737342697428293B2066616C73653F203A
:100BA0000067657453757070726573734269742859
:100BB000293B20747275653F200069734163746935
:100BC00076697479416328293A20006973496E6116
:100BD000637469766974795A456E61626C656428DC
:100BE000293A20006973496E616374697669747982
:100BF00059456E61626C656428293A200069734921
:100C00006E616374697669747958456E61626C656A
:100C10006428293A2000697341637469766974799C
:100C20005A456E61626C656428293A2000697341F7
:100C30006374697669747959456E61626C6564287C
:100C4000293A20006973416374697669747958455B
:100C50006E61626C656428293A200067657446728B
:100C6000656546616C6C4475726174696F6E2829A4
:100C70003A20006765744672656546616C6C54681D
:100C8000726573686F6C6428293A20006765745434
:100C9000696D65496E616374697669747928293A6A
:100CA0002000676574496E6163746976697479546C
:100CB00068726573686F6C642829200067657441E9
:100CC000637469766974795468726573686F6C646B
:100CD00028292000676574446F75626C65546170E3
:100CE00057696E646F7728292000676574446F75B3
:100CF000626C655461704C6174656E637928293A41
:100D000020006765745461704475726174696F6E18
:100D100028293A2000676574417869734F666673C5
:100D200065742826782C2026792C20267A293A20CA
:100D3000006765745461705468726573686F6C64A1
:100D400028293A200058595A2047733A2000585908
:100D50005A20434F554E54533A2000736574206710
:100D600061696E735B5D3A00206661696C65640061
:100D7000207375636365737366756C0023676169BF
:100D80006E735F6F7269675B5D3A00234C33473463
:100D90003230304420636F6E6E656374696F6E002D
:100DA000756E6B6E6F776E0032303030206470730A
:100DB0000035303020647073003235302064707339
:100DC00000236779726F207363616C653D00234E69
:100DD0006F204C33473432303044206779726F20B3
:100DE00073656E736F722F636865636B20776972CA
:100DF000696E672100416E676C65732F00496E63F1
:100E00006C2E20616E672E004E6F2073656E736FBF
:100E100072210049522054656D706572617475725B
:100E200065004D6561737572696E672E2E004E6F99
:100E30002073656E736F723F0049522054656D7068
:100E400065726174757265004D6561737572696E66
:100E5000672E2E00234E6F2073656E736F722066AF
:100E60006F7220504D21004E6F2073656E736F724C
:100E70002100206E672F4C00504D313A322E353A0A
:100E80003130004D6561737572696E672E2E004EAC
:100E90006F2053656E736F7221004E6F2044532094
:100EA000546865726D6F6D657465722100445320DE
:100EB000546865726D2E004D6F74696F6E004669DF
:100EC0006E64696E672057694669204950007365F2
:100ED000703D006976616C3D006E697465723D001D
:100EE000230043616C2E204661696C656400436198
:100EF0006C2E20446F6E65004E6F206E6565642118
:100F00000043616C69627261746421004D61676EB7
:100F100065746F6D657465720043616C69627261BE
:100F20007465202E2E36307300466F726365205331
:100F3000656E736F720043616C6962726174650003
:100F400062756666657220736F6C6E2E3200313D7D
:100F50004F4B20303D526563616C2E00496E7661C7
:100F60006C6964206B657900313D4F4B20303D52F8
:100F70006563616C2E0062756666657220736F6CC6
:100F80006E2E3100436F6E6475637469766974798F
:100F90000043616C69627261746500496E76616CD0
:100FA0006964206B657900313D4F4B20303D4578B9
:100FB000697400496E207361742E20736F6C6E2EFD
:100FC00000446973736F6C766564204F320043612F
:100FD0006C69627261746500436F6E74726F6C202D
:100FE00044697361626C656400436F6E74726F6C08
:100FF00020456E61626C656400496E76616C69645F
:10100000205028506129005365614C6576656C203D
:1010100050285061293A0043616C696272617465BD
:101020002050004169722054656D70286F43293A41
:101030000043616C2E204D6F74696F6E00445354F1
:101040002054656D702073656E736F720043757206
:1010500072656E742073656E736F72004F32207309
:10106000656E736F720055562073656E736F7200F4
:1010700043616C696272617465004661696C6564A4
:101080000054422063616C2E20646F6E65005570C1
:10109000706572204C696D69743A3E004C6F7765DB
:1010A00072204C696D69743A3E00547572626964CD
:1010B000697479004661696C6564007048206361F9
:1010C0006C2E20646F6E6500704831302050726560
:1010D000737320420070483420507265737320414E
:1010E0000043616C696272617465004E45543D4213
:1010F0006C7565746F6F7468204C45004E45543DA7
:10110000426C7565746F6F7468004E45543D576945
:1011100046690053657474696E67204661696C6541
:10112000640053657474696E6720446F6E65004394
:1011300068616E6765204E6574776F726B3E005410
:101140007970653A0042542F57694669204E65749C
:10115000776F726B004368616E67652053656E73CD
:101160006F723E0043757272656E742053656E73C4
:101170006F72004F7468657200496E642E20342DC2
:1011800032306D4100414353373132203C333041DE
:1011900000414353373132203C3230410041435308
:1011A000373132203C3541003E4D617820566F6C1E
:1011B000743A3E004368616E676520766F6C7461B7
:1011C00067653E00547970652000566F6C746167E6
:1011D000652053656E736F72004368616E676520AA
:1011E0007479706520746F0053656E736F723D443F
:1011F00048540054656D702048756D696469747950
:1012000000295C67411F856341B81E5D413D0A5757
:1012100041A47051410AD74B4152B846418FC24157
:1012200041C3F53C41E17A3841F6283441F6283093
:1012300041EC512C41E17A2841CDCC2441AE4721EB
:10124000418FC21D415C8F1A41295C1741EC51143A
:1012500041AE47114166660E4114AE0B41B81E09FE
:10126000415C8F0641000004418FC2014152B8FE2B
:1012700040713DFA407B14F64085EBF1408FC2EDA2
:10128000409A99E9408FC2E540713DE2406666DED2
:101290004048E1DA40295CD740F628D440C3F5D075
:1012A00040B81ECD402345432043616C69627261A2
:1012B00074696F6E205375636365737366756C0034
:1012C0002349737375652045433D4520746F205352
:1012D00061766520616E642045786974002345431A
:1012E0002043616C2E205375636365737366756C60
:1012F0002C4B3D002345432043616C69627261744D
:10130000696F6E204661696C656400234661696C93
:1013100065642C54727920416761696E00466F7272
:101320006365004D61737300282D313D6E6F6E65EE
:101330003B303D6F6C6420484D43353838333B318A
:101340003D6E6577204D4D43353838332900234DA8
:1013500061676E657469632053656E736F723D00DB
:1013600028303D6175746F3B313D616363656C3B53
:10137000323D696E636C20616E676C653B20333D66
:10138000616E672076656C290023416363656C6537
:10139000726174696F6E20413D002354696D652050
:1013A0006475726174696F6E3D002354696D6520C8
:1013B000696E74657276616C3D002354656D7020B2
:1013C000262048756D69646974792073656E736F42
:1013D000723A204448540028303D426C7565746F61
:1013E0006F74683B313D576946693B323D426C75CD
:1013F00065746F6F7468204C452900234E65743DF9
:1014000000235556207A65726F20766F6C74616781
:1014100065203D002343616C6962726174656420DC
:101420004F3220636F6E63203D0023566F6C7461F2
:1014300067652073656E6F723A00556E6B6E6F77DD
:101440006E00496E647573747269616C20342D325C
:10145000306D4100414353373132204D61783D3585
:1014600041002343757272656E742073656E736FED
:10147000723A002354757262696469747920766FD8
:101480006C74616765733A00234C43442061646463
:10149000726573733D307800235365612D6C6576FA
:1014A000656C2050726573737572653D00234F53F0
:1014B0002076657273696F6E3A2000234D6F626902
:1014C0006C65204C6F67676572204E616D653A20D0
:1014D00000696E7075742044535463616C69627264
:1014E0006174653A0023444F2043616C6962726104
:1014F00074696F6E204661696C65640023444F20F7
:1015000043616C6962726174696F6E2053756363C5
:1015100065737366756C0023444F20536174757254
:101520006174696F6E2043616C6962726174696F86
:101530006E2046696E697368656421002350757476
:1015400020444F2070726F626520696E746F207343
:10155000617475726174696F6E206F787967656EFA
:1015600020776174657221002354797065202731DA
:101570002720666F72204F4B206F72202730272064
:10158000746F206578697400237363616C652066ED
:101590006163746F723D002350757420302E3130BA
:1015A0006B672077656967687420666F7220636176
:1015B0006C69627261746F6E0043616C6962726122
:1015C000746520302E31306B6700313D4F4B203039
:1015D0003D4578697400234E6F20666F7263652005
:1015E00073656E736F72204858373131210023487C
:1015F00058373131205343414C453D00485837312D
:1016000031205343414C45002350726573732031A0
:101610003D4F4B206F7220303D4578697400313D5D
:101620004F4B20303D4578697400546172653A4EE5
:101630006F20776569676874002352656D6F766502
:1016400020616C6C2077656967687420746F207402
:1016500061726520666F72207A65726F0023436144
:101660006C6962726174696F6E20646F6E650023CD
:101670005374617274002343616C696272617469AE
:101680006F6E204D6F6465002343616C6962726107
:1016900074696F6E20636F6D706C65746564002390
:1016A000526F7461746520746865206C6F6767653C
:1016B0007220696E20382D736861706564207061D6
:1016C000746820322D332074696D65730023436183
:1016D0006C6962726174696E67206D61676E6574B2
:1016E0006F6D6574657220666F72203630732E2EB2
:1016F0002E004D4D43353838334D413D20002354A5
:1017000061726520666F7263652073656E736F72B8
:101710000054464F5243450023536574757020664C
:101720006F7263652073656E736F720049464F5226
:101730004345002343616C69627261746520666F82
:101740007263652073656E736F720043464F524338
:1017500045004D41535300464F52434500234973C2
:101760007375652045433D5320746F207374617217
:10177000742045432063616C6962726174696F6EA5
:1017800000235075742045432070726F62652D3EB2
:101790003134313375532F636D206F722031322E07
:1017A00038386D532F636D206275666665722073DD
:1017B0006F6C7574696F6E0020766F6C746167650D
:1017C0003D002354757262696469747920557070A4
:1017D0006572204C696D69743A200020766F6C74D4
:1017E0006167653D0023547572626964697479208C
:1017F0004C6F776572204C696D69743A20002354F0
:101800007572626964697479204C6F776572204CD7
:10181000696D69742056696E663A20004D617820C2
:1018200072616E67653D0023566F6C746167652059
:1018300073656E736F723A00342D32306D41004122
:101840004353373132204D61783D004143533731A6
:1018500032204D61783D3541002343757272656ECB
:10186000742073656E736F723A002344532054687A
:1018700065726D6F6D657465722063616C6962720B
:101880006174656420666F72202300445354002302
:101890004E6F206E65656420746F2063616C6962B1
:1018A000726174652063757272656E742073656E03
:1018B000736F7221002341435337313220637572B5
:1018C00072656E742073656E736F72206F666673D7
:1018D000657420563D00235556207A65726F207638
:1018E0006F6C74616765203D0055565A00234F3276
:1018F00020766F6C253D00234F322063616C696256
:10190000726174696F6E3A200023566F6C74616760
:10191000652870483D3130293A0023566F6C746158
:1019200067652870483D34293A00504834005554C2
:10193000454D503D004448543D004149413D004122
:1019400049413D00413D002354696D652064757235
:101950006174696F6E3D002354696D6520696E7412
:10196000657276616C3D00576946692049503A00BE
:10197000436F6E74726F6C2044697361626C65644E
:1019800000436F6E74726F6C20456E61626C6564AB
:1019900000234D5320456E61626C656400234D53F6
:1019A0002044697361626C6564002352657374201E
:1019B000706172616D657465727320746F20646507
:1019C0006661756C742076616C756573004C6F6729
:1019D000676572204E616D653A20006974657261B9
:1019E00074696F6E3D0073656E736F72233D0043C3
:1019F000757272656E74207374617475733A2063C6
:101A000079636C653D006E6379636C653D006E7350
:101A1000656E736F72733D006D61786E73656E7382
:101A20006F72733D00656E61626C65643D00234DAD
:101A3000756C746973656E736F7273206D65617315
:101A40007572656D656E742073657474696E677305
:101A50003A002353657474696E6773206F66206162
:101A60006C6C2073656E736F72733A002353697ADE
:101A700065206F6620686561646572202B20616C4B
:101A80006C2073656E736F72733A20002353697A0A
:101A900065206F66206865616465723A20004F6654
:101AA00066206169722D636F6E642100497427732B
:101AB00020746F6F20636F6F6C210054656D702010
:101AC00069732066696E6521004973206169722D12
:101AD000636F6E64206F6E3F0049742773207175C9
:101AE00069746520686F74210049742773207665D6
:101AF000727920686F742120004F666620616972D8
:101B00002D636F6E6421004974277320746F6F20FA
:101B1000636F6F6C210054656D7020697320666976
:101B20006E6521004973206169722D636F6E6420B8
:101B30006F6E3F0049742773207175697465206862
:101B40006F74210049742773207665727920686F5D
:101B500074210054656D702048756D6964697479ED
:101B6000002320616E6420726561647920746F20A7
:101B70007573652100206D6F62696C65206C6F67FD
:101B80006765722073746172746564200043616CD0
:101B90006962726174696F6E2050726573737572D9
:101BA000653D00536561206C6576656C2050286347
:101BB000616C63293D00234572726F723A707265E1
:101BC000737375726520424D503038352C20636830
:101BD00065636B20776972696E67210049522054F2
:101BE000656D702073656E736F7220666F756E64BD
:101BF00000206D6F62696C65206C6F67676572208D
:101C000073746172746564202E2E2E20005769460D
:101C1000692049503A00235769466920495020619C
:101C20006464726573733A20002323205345534C38
:101C30006F676765722023230023232057656C6339
:101C40006F6D65202323004C4344206164647265FA
:101C500073733D30780053656E736F7220736C6FD1
:101C60007420616E6420747970653A00005EBCE295
:101C7000613FDD83C29C7E20A3FD1F41009D23BEEA
:101C800046DB65F88C11AF32CA57E97400002100B9
:101C9000240027002A002D0030003300010100003D
:101CA000040107010A0100002200250028002B0082
:101CB0002E003100340002010000050108010B0173
:101CC000000020002300260029002C002F003200F5
:101CD00000010000030106010901050505050705CE
:101CE00008080808020202020A0A08080404040498
:101CF00001010101010101010303030303030303C4
:101D0000040707070C0C0C0C0C0C0C0C0202020252
:101D100006060606060606060B0B0B0B0B0B0B0B3B
:101D200001021020200808102040102040800201ED
:101D300002010804020101020408102040808040D2
:101D400020100804020180040201804020100804D1
:101D5000020108040201010204081020408001026F
:101D600004081020408000000A0B02090C0D0E0828
:101D70000703040100000000000000000000000054
:101D80000000000000000000000000000000000053
:101D90000000121110000000000000000000000010
:101DA00000000000000000000000000023456E64F9
:101DB000206F66204D756C746973656E736F722049
:101DC0004379636C652300496E76616C6964206BAE
:101DD00065792100EDD5E7D411241FBECFEFD1E204
:101DE000DEBFCDBF00E00CBF1CE0A0E0B2E0E2EC43
:101DF000F1ED01E00BBF02C007900D92A039B107D1
:101E0000D9F726E1A0E9BCE001C01D92AB33B207CF
:101E1000E1F71EE0CBEEDEE000E006C0219701090D
:101E2000802FFE010E94EFE5CA3ED10780E008073F
:101E3000A9F70E9428D90C94CFE80C9400000F93C6
:101E40001F93CF93DF93CDB7DEB7A2970FB6F89469
:101E5000DEBF0FBECDBF8E010B5E1F4F682FC801C6
:101E60000E94B67118870F831D821E82198289E035
:101E70008A8381E08B838C831C8A1B8ACE01019626
:101E80000E940B71CE0101960E94AE6F60E0CE0100
:101E900001960E949F70A2960FB6F894DEBF0FBE07
:101EA000CDBFDF91CF911F910F9108950F931F9395
:101EB00060E08091A6040E944E6D83E090E001975F
:101EC000F1F761E08091A6040E944E6D83E290E0FC
:101ED0000197F1F760E08091A6040E944E6D809119
:101EE000A4049091A5049927FC01E05EF24E649150
:101EF000FC01E652F34EE491F0E0EE0FFF1FE054D8
:101F0000F34E8591949100E717E120E030E0462FF1
:101F10000E942ED3611571058105910529F06F5F2F
:101F20007F4F8F4F9F4F9F700E94CBE020E030E4A7
:101F30004CE156E40E9443E32091E20C3091E30C23
:101F40004091E40C5091E50C0E942AE120E030E041
:101F500048E453E40E9443E31F910F910895CF9208
:101F6000DF92EF92FF920E94560F6B017C0120E0FE
:101F700030E040E050E40E944CE4181624F40E9443
:101F8000560F6B017C0120E030E040E050E4C701D7
:101F9000B6010E944CE4181624F40E94560F6B01FF
:101FA0007C0120E030E040E050E4C701B6010E942F
:101FB0004CE4181624F40E94560F6B017C0120E0BB
:101FC00030E040E050E4C701B6010E944CE418162E
:101FD00024F40E94560F6B017C0120E030E040E0C9
:101FE00050E4C701B6010E944CE418162CF4C12C31
:101FF000D12CE12C80E4F82EC701B601FF90EF90C0
:10200000DF90CF900895CF93DF9320919D042223FA
:10201000A9F02091FB04222389F0EC016FED86E208
:1020200096E10E947DCB8C819D81892B39F0BE0188
:1020300086E296E1DF91CF910C949AD1DF91CF9116
:10204000089580919D04882349F08091FB048823A2
:1020500029F060E086E296E10C94C67408950F932F
:102060001F93CF93DF938C011092E70C1092E60C34
:10207000C091E60CD091E70CC832D105A4F4809150
:1020800006020E94C06DCC0FDD1FC45FD04F998344
:1020900088838091E60C9091E70C01969093E70C71
:1020A0008093E60CE5CF0E9415AE20E030E040EAD8
:1020B00050E40E942AE120E030E040E85AE30E9428
:1020C0002AE10430110599F420E030E040E650E4C4
:1020D0000E942AE19B01AC0160E070E080E890E49E
:1020E0000E9464E2DF91CF911F910F9108950A3011
:1020F000110569F420E030E040E650E40E942AE156
:102100009B01AC0160E070E080E291E4E9CF60E027
:1021100070E0CB01E7CF23E333E948E853E40E94C2
:1021200043E320E030E040E85FE30E9465E20E9484
:102130006DE526E636EA45EA53E40E942AE160931B
:10214000E20C7093E30C8093E40C9093E50C0895FB
:1021500081E08093FB0480919D04882341F088E016
:102160008093311660E086E296E10C9494740895B1
:1021700080919D04811110C081E080939D04809323
:10218000FB0480912C16982F946090932C168C60F1
:102190000E94D7AD0C94A8108091FB048823D1F342
:1021A0001092311660E086E296E10E9494741092DB
:1021B000FB0480912C168B7F80932C1688600E94E4
:1021C000D7AD10929D0408952F923F924F925F9247
:1021D0006F927F928F929F92AF92BF92CF92DF9237
:1021E000EF92FF920F931F93CF93DF936C01C7E69B
:1021F000D5E083EB882E84E0982E01EF12E1EE24E7
:10220000E394F12C22E1222E312C33E1432E512C88
:1022100040E1642E712C51E1A52EB12C8091B304C4
:102220009091B4048E159F050CF4C9C021E0C2162C
:10223000D10409F0BDC0F80182AD93ADF4019383E0
:102240008283F40182819381009709F58A819B81C1
:102250009093050280930402F4018281938184307B
:102260009105C1F52A813B81309307022093060234
:102270008531910509F47BC08631910509F040C094
:102280002A813B8130938A04209389044EC0813097
:10229000910539F48A819B8190939F0480939E04D9
:1022A000DBCF8230910539F48A819B8190930302C0
:1022B00080930202D1CF039779F68A819B81909314
:1022C00001028093000261E47CE08BE295E10E94D0
:1022D000E2C5C2CF8530910539F42A813B81309324
:1022E000880420938704C4CF8630910529F2873073
:1022F0009105B9F42A813B8130938E0420938D049B
:102300008731910591F42A813B8128303105B1F55F
:102310007092A7046092A604B092A504A092A404AF
:1023200004C08A30910509F0A3CF9C012B503109DC
:102330002A30310590F42A813B81309301022093A9
:10234000000239E1389FB001399F700D1124625F9E
:102350007D4F8BE295E10E9445C68FEFE81AF80A9F
:102360002296E2E08E0E911C0E5F1F4F57CF2A81FE
:102370003B8130938C0420938B04D7CF27303105D9
:1023800049F43092A7042092A6045092A5044092EA
:10239000A404CBCF2630310541F621E030E0309364
:1023A000A7042093A6041092A5041092A404BDCF04
:1023B000F40182819381F80193AF82AF42CFDF9124
:1023C000CF911F910F91FF90EF90DF90CF90BF9032
:1023D000AF909F908F907F906F905F904F903F90C5
:1023E0002F9008954F925F926F927F929F92AF923B
:1023F000BF92CF92DF92EF92FF920F931F93CF93F2
:10240000DF93982E8EE0A82EB12CEE24EA9493E070
:10241000F92E0FEF13E0D12CC12CD0E0C0E0412CFD
:10242000512C3201892D0E94C06DC817D90708F4BC
:102430004AC0C816D90608F46C018017910708F441
:1024400044C08E159F0508F47C01BC0190E080E03B
:102450000E94C9E09B01AC01C301B2010E9465E288
:102460002B013C0165E070E080E090E00E94086E86
:1024700081E0A81AB108B1F6BE016C0D7D1D6E0D8C
:102480007F1D600F711F90E080E00E94C9E09B01FA
:10249000AC01C301B2010E9464E220E030E040E2FE
:1024A00051E40E9443E3DF91CF911F910F91FF9080
:1024B000EF90DF90CF90BF90AF909F907F906F9004
:1024C0005F904F900895EC01B8CF8C01BECFCF92B2
:1024D000DF92EF92FF92CF93C0912013C4304CF45F
:1024E000C1300CF04BC0CC2359F160E070E0CB015F
:1024F0003FC0C430D1F70E94F21120E030E040EA42
:1025000050E40E942AE120E030EC4FE754E40E94BE
:1025100043E320E030E040EA50E40E9443E320E05F
:1025200030E040E851E40E942AE120E030E040E859
:1025300050E40E9465E220E030E04AE754E416C02F
:102540000E94F21120E030E040EA50E40E942AE1CB
:1025500020E030EC4FE754E40E9443E32091211344
:102560003091221340912313509124130E9443E38E
:10257000CF91FF90EF90DF90CF9008950E94F211DD
:102580002AE137E64CE950E40E942AE12091211328
:102590003091221340912313509124130E9464E23E
:1025A0006B017C01EC2FEE0FFF0BE15AFA4F6081BB
:1025B0007181072E000C880B990B0E94CBE09B01C8
:1025C000AC01C701B601D2CF1F93CF93DF93182F71
:1025D000CCE0DFE0812F0E94C06D899399936CE37A
:1025E00070E080E090E00E94086E8FE0CC35D80764
:1025F00089F70E9415AE20E030E040EA50E40E94E6
:102600002AE120E030E040E85AE30E942AE1DF912D
:10261000CF911F910895CF93DF93FC0124813581E1
:10262000232B99F0EC01BC018BEA9FE00E94A8D11A
:102630006EE170E080E090E00E94086EBE0182E8EA
:1026400091E1DF91CF910C94A8D1DF91CF910895C2
:10265000CF93DF93FC0124813581232B69F0EC01BA
:10266000BC0182E891E10E949AD1BE018BEA9FE011
:10267000DF91CF910C949AD1DF91CF910895809101
:102680009D048823F9F08091FB048823D9F081E030
:102690000E94D7AD8BE39FE10197F1F760E080E006
:1026A0000E94E8AD6DEE74E086E296E10E94BAD138
:1026B00061E080E00E94E8AD6DED74E086E296E1B5
:1026C0000C94BAD10895EF92FF920F931F93CF937A
:1026D000DF9320919D04222309F461C02091FB0423
:1026E000222309F45CC08A01EB017C01209719F1D7
:1026F000C095D09561E08C2F0E94E8ADB70186E2CD
:1027000096E10E949AD16CEC74E086E296E10E9418
:10271000BAD1F701848161E08C0F0E94E8ADB80165
:10272000110F880B990BDF91CF911F910F91FF90A3
:10273000EF900C94086E0E943B6EAB01BC0180913F
:10274000A00C9091A10CA091A20CB091A30C8C595B
:102750009F4FAF4FBF4F84179507A607B707F8F4F1
:1027600061E080E00E94E8ADB70186E296E10E9458
:102770009AD16BEB74E086E296E10E94BAD161E0F7
:10278000F70184810E94E8AD0E943B6E6093A00C2B
:102790007093A10C8093A20C9093A30CC0CFDF91F7
:1027A000CF911F910F91FF90EF900895FF920F939B
:1027B0001F93CF93DF93EC01F62E08811981C80196
:1027C0000E94EBE1F81621F06F2DC8010E94F3E1A1
:1027D000CE01DF91CF911F910F91FF900895DC0101
:1027E000ED91FC910190F081E02D19948F929F92D0
:1027F000AF92BF92CF92DF92EF92FF920F931F930F
:10280000CF93DF938C01862F0B30110509F092C016
:1028100090913E15992309F0F89462E10E945EC1FF
:10282000EC0180913E15882309F07894209701F1FE
:1028300080E090ECA9E7B4EC8093311590933215C9
:10284000A0933315B09334158093351590933615B6
:10285000A0933715B0933815CE3F8FEFD80709F402
:102860009DC0CF3FDC0709F4EFC1CCEFDFEF24C1FF
:10287000C0913915E0903A156E2D70E090E080E03F
:102880000E94CBE02DEC3CEC4CEC5DE30E942AE195
:102890004B015C016C2F70E090E080E00E94CBE087
:1028A0009B01AC01C501B4010E9465E26093311542
:1028B000709332158093331590933415D0913B1556
:1028C000F0903C156D2F6F7770E090E080E00E94F3
:1028D000CBE04B015C016F2D70E090E080E00E9446
:1028E000CBE02DEC3CEC4CEC5DE30E942AE19B013B
:1028F000AC01C501B4010E9465E2D7FD19C0609327
:102900003515709336158093371590933815CE0D85
:10291000CD0FCF0D81E090E020913D15C21302C094
:1029200090E080E0892B09F487C0CFEFDFEF8CC106
:102930009058E5CFCFEFDFEF0631110509F0BCC0AD
:1029400090913E15992309F0F89461E00E945EC1D0
:10295000EC0180913E15882309F07894209709F1C5
:1029600080E090ECA9E7B4EC809331159093321598
:10297000A0933315B0933415809335159093361585
:10298000A0933715B0933815CF3FDC0709F45CC12D
:10299000209709F451C0229609F067CFCEEFDFEF00
:1029A0008BC0C0913A15D09139156091391570914D
:1029B0003A1576276727762790E080E00E94C9E0E5
:1029C0002DEC3CEC4CEC5DE30E942AE16093311568
:1029D000709332158093331590933415E0903C1525
:1029E000F0903B156F2D6F77762F6E2D90E080E085
:1029F0000E94C9E02DEC3CEC4CEC5DE30E942AE126
:102A0000F7FC18C060933515709336158093371511
:102A1000909338158C2F8D0F8E0D8F0DC1E0D0E067
:102A200090913D15891302C0D0E0C0E0D195C195C9
:102A3000D109AACF9058E6CFC0903115D090321569
:102A4000E0903315F090341520E030E048EC52E48B
:102A5000C701B6010E944CE4D0E0C0E0181614F49F
:102A6000CBEFDFEF20E030E0A901C701B6010E9403
:102A7000C4E087FF02C0CAEFDFEFC0903515D090E9
:102A80003615E0903715F090381520E030E048EC2E
:102A900052ECC701B6010E94C4E087FF02C0C9EF33
:102AA000DFEF20E030E040EF52E4C701B6010E94C2
:102AB0004CE418160CF4C3C00C30110509F0C4C066
:102AC0008CE50E94CDAD70E060E089ED94E10E945C
:102AD000EF1389ED94E10E94917465E08CE50E940A
:102AE000DAB11092090F8093080FC82FD0E0209719
:102AF00009F4A8C0C530D1050CF4B6C00BED1DE03B
:102B00000E94C7B1F80180870F5F1F4FC8018B5D1E
:102B10009D408C179D07A4F3C091E30D0091E40D37
:102B2000602F70E090E080E00E94CBE02DEC3CEC68
:102B30004CEC5DE30E942AE16B017C016C2F70E09C
:102B400090E080E00E94CBE09B01AC01C701B601A0
:102B50000E9465E26B017C01C092DB0DD092DC0D1E
:102B6000E092DD0DF092DE0DD091E50D1091E60DB5
:102B70006D2F6F7770E090E080E00E94CBE04B011A
:102B80005C01612F70E090E080E00E94CBE02DECD2
:102B90003CEC4CEC5DE30E942AE19B01AC01C501D9
:102BA000B4010E9465E2D7FD5DC06093DF0D7093B4
:102BB000E00D8093E10D9093E20DC00FCD0FC10F9A
:102BC0008091E70DC813B1CE20E030E048EC52E42C
:102BD000C701B6010E944CE4D0E0C0E0181614F41E
:102BE000CBEFDFEF20E030E040EA50E4C701B60170
:102BF0000E94C4E087FF02C0CAEFDFEFC090DF0D84
:102C0000D090E00DE090E10DF090E20D20E030E09A
:102C100040EF51ECC701B6010E94C4E087FF02C03B
:102C2000C9EFDFEF20E030E040EF52E4C701B6012A
:102C30000E944CE4181644F4C8EFDFEF05C0C8EF5B
:102C4000DFEF3ACFCEEFDFEFCE01DF91CF911F91D3
:102C50000F91FF90EF90DF90CF90BF90AF909F903B
:102C60008F9008959058A1CFCDEFDFEFEDCFCF93A8
:102C7000DF93EC019A01AB01E889F98982E0808356
:102C8000211581EE38074105510581F160E079E0B9
:102C90008DE390E00E9433E221503109410951094E
:102CA0005695479537952795EC85FD851082EE85DD
:102CB000FF852083188EEC89FD8986E08083EA8970
:102CC000FB89808180618083EA89FB8980818860BB
:102CD0008083EA89FB89808180688083EA89FB8917
:102CE00080818F7D8083DF91CF910895E889F98974
:102CF000108220E1D9CF2F923F924F925F926F9234
:102D00007F928F929F92AF92BF92CF92DF92EF927B
:102D1000FF920F931F93CF93DF93CDB7DEB76697E4
:102D20000FB6F894DEBF0FBECDBF1C0185EE90E15B
:102D30000E94E8B040E855E260E070E085EE90E186
:102D40000E94371664E670E080E090E00E94086E12
:102D50008CED95E0A0E0B0E08093E9109093EA104C
:102D6000A093EB10B093EC1064E670E080E090E08C
:102D70000E94086E8FEF8A8781E08B8786E88C87B8
:102D80001D861E861F86188A198A89E78A8BC101CB
:102D9000880F991F9E8B8D8BD12CC12CF12CE12C8F
:102DA000412C512C320185EE90E10E94A4AA089793
:102DB0004CF049E050E0BE01665F7F4F85EE90E148
:102DC0000E945EAA65E070E080E090E00E94086EDC
:102DD00010E000E0812C912C540185EE90E10E94DE
:102DE000D5AA892B39F4F4E08F169104A104B1041B
:102DF0000CF04EC0023011050CF04AC085EE90E197
:102E00000E94D5AA892B69F085EE90E10E94B3AAB1
:102E1000E1E0F0E0EC0FFD1FE00FF11F80830F5F9A
:102E20001F4F65E070E080E090E00E94086E023085
:102E3000110509F073C099818A8598136FC09A8132
:102E40008C8598136BC0FE013396FC8BEB8B85EE63
:102E500090E10E94D5AA892B39F4F4E08F169104F1
:102E6000A104B1040CF053C00930110509F05CC095
:102E70008B8190E0982F88272C81820F911D092E3D
:102E8000000CAA0BBB0B480E591E6A1E7B1E43C0CA
:102E90008FEFC81AD80AE214F30434F4ED89FE89DE
:102EA000EC15FD0509F07FCF85EE90E10E94E8B0BA
:102EB000E114F10409F47101C301B2010E94CBE0F5
:102EC0004B015C01B701FF0C880B990B0E94CBE012
:102ED0009B01AC01C501B4010E9443E366960FB6A5
:102EE000F894DEBF0FBECDBFDF91CF911F910F9140
:102EF000FF90EF90DF90CF90BF90AF909F908F901A
:102F00007F906F905F904F903F902F900895043086
:102F100011050CF0ADCFFFEFEF1AFF0A8FEF881A03
:102F2000980AA80AB80A59CF85EE90E10E94B3AA80
:102F3000EB89FC898193FC8BEB8B0F5F1F4F87CF55
:102F40004F925F926F927F92AF92BF92CF92DF9239
:102F5000FF920F931F93CF93DF9300D000D0CDB794
:102F6000DEB75C0185EE90E10E94E8B040E052ECF3
:102F700061E070E085EE90E10E9437168CED95E0FF
:102F8000A0E0B0E08093E9109093EA10A093EB10DA
:102F9000B093EC1064E670E080E090E00E94086E70
:102FA000D12CC12CF12C65E070E080E090E00E9413
:102FB000086E10E000E0412C512C3201F1103AC0B3
:102FC00085EE90E10E94D5AA892B31F485E148165F
:102FD00051046104710474F5033011055CF585EE4C
:102FE00090E10E94D5AA892B69F085EE90E10E94BC
:102FF000B3AAE1E0F0E0EC0FFD1FE00FF11F8083CA
:103000000F5F1F4F65E070E080E090E00E94086E67
:10301000023011054CF089818B3B31F4FF24F3948D
:103020008A818A3A09F0F12C8FEF481A580A680A07
:10303000780AC4CF8FEFC81AD80A64E670E080E03F
:1030400090E00E94086EAC14BD0409F0ACCF8F2D47
:1030500026960FB6F894DEBF0FBECDBFDF91CF919D
:103060001F910F91FF90DF90CF90BF90AF907F9016
:103070006F905F904F900895CF93DF93EC01FB0129
:10308000248135810E941CC9CE01DF91CF91089522
:10309000CF92DF92EF92FF920F931F93CF93DF9324
:1030A000CDB7DEB762970FB6F894DEBF0FBECDBFC7
:1030B0002091AC0D222309F4D8C02091D10D30917C
:1030C000D20D263531050CF0D0C0409195045091B9
:1030D0009604493D5F400CF0C8C08C012F5F3F4F04
:1030E0003093D20D2093D10D0E943B6EC090A40D61
:1030F000D090A50DE090A60DF090A70D6C197D095C
:103100008E099F090E94C9E020E030E04AE754E4BC
:103110000E9443E36093A80D7093A90D8093AA0DBC
:103120009093AB0D809195049091960488359240D0
:1031300034F488E592E0909396048093950480910E
:1031400095049091960438EAE32E3DE0F32E9C011D
:10315000285A3D406901C6018E0D9F1D9A838983BF
:10316000F70161917F01CE0101960E94D613FCEA1E
:10317000EF16FDE0FF0679F7809195049091960493
:1031800004969093960480939504B801CE0101961D
:103190000E9402C9CE0101960E94FEC7BC01CE0169
:1031A0000D960E9402C9CE0101960E949FC8F801A7
:1031B00084819581849708F123E230E050E040E07B
:1031C000B801CE0101960E941CC9BE016F5F7F4FFE
:1031D000CE0107960E9402C9CE0107960E94FEC743
:1031E000BC01CE010D960E9443C8CE0107960E94F5
:1031F0009FC8CE0101960E949FC849895A894115EE
:10320000510549F08DEA9DE0009729F0BC01CE01FF
:103210000D960E949BB0809195049091960421EDAB
:10322000C22E2DE0D22E0DEA1DE09C012D5A3D400C
:103230007901C701800F911F9A838983F8016191F9
:103240008F01CE0101960E94D613C016D10689F7D0
:10325000809195049091960484969093960480931F
:103260009504CE010D960E949FC862960FB6F89401
:10327000DEBF0FBECDBFDF91CF911F910F91FF90A9
:10328000EF90DF90CF900895AF92BF92CF92DF92F0
:10329000EF92FF920F931F93CF93DF93CDB7DEB7DB
:1032A00062970FB6F894DEBF0FBECDBF20919D048C
:1032B000222309F447C02091FB04222309F442C0D1
:1032C0007A016B015C010E943B6EAB01BC018091F5
:1032D0009C0C90919D0CA0919E0CB0919F0C8C59D0
:1032E0009F4FAF4FBF4F84179507A607B70750F5FD
:1032F00060E08FEFC816D806B1F580E00E94E8AD17
:1033000000E0B50186E296E10E949AD16AEA74E093
:1033100086E296E10E94BAD1F501848160E0800FD7
:103320000E94E8AD0E943B6E60939C0C70939D0CD4
:1033300080939E0C90939F0CB701FF0C880B990B08
:103340000E94086E62960FB6F894DEBF0FBECDBF26
:10335000DF91CF911F910F91FF90EF90DF90CF9071
:10336000BF90AF90089580E00E94E8AD0E943B6E50
:1033700028EE33E040E050E00E9401E2CA01B901CA
:1033800020E831E541E050E00E9401E2AB01BC01E0
:10339000CE0101960E94ECC5BE016F5F7F4FCE014A
:1033A00007960E9402C965E87BE0CE0107960E945D
:1033B00066C7BC01CE010D960E9402C9CE010796D8
:1033C0000E949FC8CE0101960E949FC8BE01635F04
:1033D0007F4F86E296E10E949AD109891A89C11429
:1033E000D10431F00C0D1D1D60E0802F0E94E8AD6E
:1033F000CE010D960E949FC884CFBF92CF92DF92DC
:10340000EF92FF920F931F93CF93DF93CDB7DEB769
:1034100062970FB6F894DEBF0FBECDBF6C018B0173
:103420007A0180919D04882369F18091FB048823AF
:1034300049F177FF37C00095109560E0802F0E941A
:10344000E8ADB60186E296E10E949AD169E974E09E
:1034500086E296E10E94BAD1F601848160E0800F95
:103460000E94E8AD0E943B6E60939C0C70939D0C93
:1034700080939E0C90939F0CB701FF0C880B990BC7
:103480000E94086E62960FB6F894DEBF0FBECDBFE5
:10349000DF91CF911F910F91FF90EF90DF90CF9030
:1034A000BF90089560E080E00E94E8AD0E943B6E0E
:1034B00028EE33E040E050E00E9401E2CA01B90189
:1034C00020E831E541E050E00E9401E2AB01BC019F
:1034D000CE0101960E94ECC5BE016F5F7F4FCE0109
:1034E00007960E9402C965E87BE0CE0107960E941C
:1034F00066C7BC01CE010D960E9402C9CE01079697
:103500000E949FC8CE0101960E949FC8BE01635FC2
:103510007F4F86E296E10E949AD1B98860E08B2DB8
:103520000E94E8AD0115110531F40B2DCE010D9669
:103530000E949FC886CF60E0802F0E94E8ADF6CF42
:10354000CF93DF93EC01483085E0580761057105A2
:1035500009F448C008F099C0493481E05807610572
:10356000710509F4B2C008F040C0443481E0580746
:103570006105710509F476C000F5413481E0580712
:103580006105710509F456C048F4403451406105A5
:10359000710509F4E4C061E47CE0E3C0423481E0F9
:1035A00058076105710509F409C1433451406105AB
:1035B000710589F76CE97BE0D4C0463481E0580797
:1035C0006105710509F40CC108F49FC0473481E01E
:1035D00058076105710509F455C04834514061052B
:1035E0007105C9F66CED75E0BCC0423085E0580746
:1035F0006105710509F4E2C000F5443781E0580720
:103600006105710509F4F2C040F44237514061058B
:10361000710509F66DEE77E0A4C0411585E0580705
:103620006105710509F49BC0413055406105710584
:1036300009F0B1CF62EA7BE094C0453085E05807DD
:103640006105710509F461C080F4433085E05807D5
:103650006105710509F4AECF44305540610571052F
:1036600009F099CF69E97BE07CC0463085E05807D6
:103670006105710509F4B4C0473055406105710515
:1036800009F089CF6AED75E06CC04D3B82E45807C4
:103690008FEF6807710509F4AFC008F048C04F3ECE
:1036A00080E158078FEF6807710561F3F8F4423342
:1036B00085E058076105710509F4ACCF48F449303D
:1036C00055406105710509F066CF6EED75E049C0A2
:1036D000443385E058076105710509F487C04D3F03
:1036E00052406F4F710509F495CF55CF4D3D82E2A1
:1036F00058078FEF6807710509F478C048F4473E12
:1037000058416F4F710509F046CF66E97BE029C04B
:103710004F3C80E358078FEF6807710509F4A2CF8B
:10372000473C58436F4F710509F45CCF34CF47399C
:1037300088E658078FEF6807710509F47BCF48F5D5
:103740004D3A82E558078FEF6807710509F451C0BB
:1037500078F4453B5A446F4F710509F01CCF67ED73
:1037600077E0CE010E940BC9CE01DF91CF91089581
:10377000453A8AE558078FEF6807710509F4A5CF28
:103780004D3952466F4F710509F005CF65E079E07C
:10379000E8CF473588EA58078FEF6807710519F1B8
:1037A00080F445388AE758078FEF68077105C1F044
:1037B000473658496F4F710509F0EDCE6FE97BE050
:1037C000D0CF4F3480EB58078FEF6807710509F4AD
:1037D000F1CE4D33524C6F4F710509F41BCFDBCE48
:1037E00068ED75E0BECF6AE07BE0BBCF6EE778E0C6
:1037F000B8CF6BE379E0B5CF69EF77E0B2CF3F9216
:103800004F925F926F927F928F929F92AF92BF92F0
:10381000CF92DF92EF92FF920F931F93CF93DF939C
:10382000CDB7DEB7EB970FB6F894DEBF0FBECDBFB6
:103830002B013C0188E490E10E94E8B064E670E06E
:1038400080E090E00E94086E40E855E260E070E0A1
:1038500088E490E10E94371664E670E080E090E032
:103860000E94086E63E87EE088E994E10E941EC829
:1038700068E974E1CE0101960E9402C942E350E07A
:103880006FEF7FEFCE0101960E94FD19CE010196E8
:103890000E949FC868E77EE088E994E10E941EC804
:1038A00068E974E1CE0101960E9402C942E350E04A
:1038B0006FEF7FEFCE0101960E946313CE01019658
:1038C0000E949FC88091F20D9091F30D8D7F312C55
:1038D000D12CC12CF12CE12C10E000E0019709F46F
:1038E0007AC09E01205E3F4F39AF28AFCE014E9681
:1038F0009BAF8AAF0E943B6E6419750986099709D0
:10390000683B7B408105910508F065C088E490E143
:103910000E94D5AA892B09F44DC08CED95E0A0E05A
:10392000B0E080934C1090934D10A0934E10B09344
:103930004F100E94EAAF97FD3DC082349105C9F750
:10394000DE0111964D015D010E94EAAF97FF39C07B
:1039500089818D3479F590E080E0D4012D914D017D
:10396000820F911DEAADFBADAE17BF07B1F78E5BBD
:103970009F4F2E8D30E0322F22274F8D240F311D87
:1039800082179307B9F40C8110E0102F00278D8166
:10399000080F111DEE80F12CFE2CEE248F81E80E15
:1039A000F11CC884D12CDC2CCC248985C80ED11CF8
:1039B0003324339462E370E080E090E00E94086E6C
:1039C00099CFD5018D935D01E8ADF9ADAE17BF0775
:1039D00009F0BACFBDCF0E943B6E64197509860904
:1039E0009709683B7B408105910510F43110BBC0FD
:1039F0000E943F1368E974E1CE0180960E9402C9DB
:103A000042E350E066E070E0CE0180960E94FD192E
:103A1000CE0180960E949FC8332009F4CCC082E07A
:103A200090E09093F30D8093F20DB601CE01C29613
:103A30000E9419C6B701CE018C960E9419C6B80122
:103A4000CE0180960E9419C6BE01605E7F4FCE01F6
:103A500086960E9402C960E677E0CE0186960E94B3
:103A600066C7BE01645D7F4F0E947CC760E677E059
:103A70000E9466C7BE016E5C7F4F0E947CC7BC017E
:103A80008EE994E10E9443C8CE0186960E949FC8A9
:103A9000CE0180960E949FC8CE018C960E949FC83E
:103AA000CE01C2960E949FC86EE974E1CE01809655
:103AB0000E9402C94AE050E06FEF7FEFCE0180968E
:103AC0000E946313CE0180960E949FC862E77EE049
:103AD00086E296E10E94BAD1B601CE01C2960E945A
:103AE00019C6B701CE018C960E9419C6B801CE0145
:103AF00086960E9419C660EE75E0CE0180960E94FF
:103B00000BC9BE016A5D7F4FCE0180960E947CC7C3
:103B10006EE277E00E9466C7BE01645D7F4F0E943F
:103B20007CC76EE277E00E9466C7BE016E5C7F4F85
:103B30000E947CC760EF75E00E9466C7BC018EE9F9
:103B400094E10E9443C8CE0180960E949FC8CE0196
:103B500086960E949FC8CE018C960E949FC8CE0177
:103B6000C2960E949FC862E370E080E090E00E94ED
:103B7000086E88E490E10E94E8B062E370E080E0C3
:103B800090E00E94086EEB960FB6F894DEBF0FBE71
:103B9000CDBFDF91CF911F910F91FF90EF90DF90FC
:103BA000CF90BF90AF909F908F907F906F905F90DD
:103BB0004F903F90089567E67EE08EE994E10E9481
:103BC0001EC86EE974E1CE0180960E9402C94AE0E7
:103BD00050E070E060E0CE0180960E946313CE0159
:103BE00080960E949FC864E57EE08EE994E10E9481
:103BF0001EC88091F20D9091F30D029709F0B3CF9A
:103C00001092F30D1092F20DAECF0F931F93CF933E
:103C1000DF9300D000D0CDB7DEB720917E0E2223F7
:103C2000A9F08C016BE379E0CE0101960E940BC9EB
:103C3000B801CE0101960E947CC7BC0182E891E1E7
:103C40000E94A8D1CE0101960E949FC826960FB669
:103C5000F894DEBF0FBECDBFDF91CF911F910F91C2
:103C60000895CF93DF93CDB7DEB72C970FB6F894B6
:103C7000DEBF0FBECDBF8130910509F06EC09093BD
:103C80006813809367136AE071E1CE0101960E9488
:103C9000F9C8CE0101960E94051ECE0101960E9430
:103CA0009FC866EF75E0CE0101960E940BC96EE0D9
:103CB00076E1CE0101960E947CC7BC01CE01079639
:103CC0000E9402C948EC50E06FEF7FEFCE010796EB
:103CD0000E94FD19CE0107960E949FC8CE01019651
:103CE0000E949FC88BEA9FE00E94E8B040E052EC3F
:103CF00061E070E08BEA9FE00E94371690E080E080
:103D00000E9471B065E076E0CE0101960E940BC979
:103D10006AE176E1CE0101960E947CC7BC01CE012A
:103D200007960E9402C940ED57E06FEF7FEFCE018A
:103D300007960E946313CE0107960E949FC8CE018A
:103D400001960E949FC881E02C960FB6F894DEBFC2
:103D50000FBECDBFDF91CF9108950097E1F510928E
:103D60006813109267136CEF70E1CE0101960E9408
:103D7000F9C8CE0101960E94051ECE0101960E944F
:103D80009FC86CEF75E0CE0101960E940BC96EE0F2
:103D900076E1CE0101960E947CC7BC01CE01079658
:103DA0000E9402C948EC50E06FEF7FEFCE0107960A
:103DB0000E94FD19CE0107960E949FC8CE01019670
:103DC0000E949FC88BEA9FE00E94E8B040E855E25D
:103DD00060E070E08FCF82309105A9F49093681372
:103DE000809367136BEE70E1CE0101960E94F9C8D3
:103DF000CE0101960E94051ECE0101960E949FC829
:103E000060E076E0C0CF80E09FCFBF92CF92DF929C
:103E1000EF92FF920F931F93CF93DF93CDB7DEB74F
:103E200062970FB6F894DEBF0FBECDBF8C016B0159
:103E30006EE277E0CE010D960E940BC960EE7EE047
:103E4000C8010E94F9C876012FEFE21AF20AB70101
:103E5000CE0101960E9419C6BE016F5F7F4FCE0151
:103E600007960E9402C960E677E0CE0107960E949D
:103E700066C7BC01C8010E9417C8CE0107960E9400
:103E80009FC8CE0101960E949FC88AE0B82EBE9CB2
:103E9000C001BF9C900D1124FC01E856FC4E7F012F
:103EA0008081082E000C990B0E945EE8892B09F492
:103EB000B2C0B701CE0101960E940BC9BE016F5F6F
:103EC0007F4FCE0107960E9402C960E87BE0CE01D9
:103ED00007960E9466C7BC01C8010E9417C8CE01A0
:103EE00007960E949FC8CE0101960E949FC8BC9C65
:103EF000C001BD9C900D11249C0128563C4E7901B7
:103F0000F9016685062E000C770BCE0101960E9402
:103F100019C6BE016F5F7F4FCE0107960E9402C98E
:103F200062E67CE0CE0107960E9466C7BE01635F31
:103F30007F4F0E947CC7BC01C8010E9417C8CE01F8
:103F400007960E949FC8CE0101960E949FC869ED06
:103F50007EE0C8010E948FC7F7016785062E000C1E
:103F6000770BCE0101960E9419C6BE016F5F7F4F8D
:103F7000CE0107960E9402C9BE01635F7F4FCE014A
:103F800007960E947CC7BC01C8010E9417C8CE01D9
:103F900007960E949FC8CE0101960E949FC863EDBC
:103FA0007EE0C8010E948FC7F70160897189CE0148
:103FB00001960E9419C6BE016F5F7F4FCE01079622
:103FC0000E9402C9BE01635F7F4FCE0107960E9427
:103FD0007CC7BC01C8010E9417C8CE0107960E9489
:103FE0009FC8CE0101960E949FC86EEC7EE0C8017A
:103FF0000E948FC7F70162897389CE0101960E94E2
:1040000019C6BE016F5F7F4FC8010E9417C8CE015D
:1040100001960E949FC8CE010D960E949FC8C801BC
:1040200062960FB6F894DEBF0FBECDBFDF91CF9181
:104030001F910F91FF90EF90DF90CF90BF90089568
:104040004F925F926F927F929F92AF92BF92CF9268
:10405000DF92EF92FF920F931F93CF93DF93CDB731
:10406000DEB7A9970FB6F894DEBF0FBECDBF982E6E
:10407000882351F080917E0E882331F061E47CE04A
:1040800082E891E10E946BCB0E9405C360E08DE263
:104090000E9443C260E18DE20E9443C268E08DE26B
:1040A0000E9443C2809177139091781397FD63C06B
:1040B00010E000E010929B0E10929C0E10929D0E4C
:1040C00010929E0E10929F0E1092A00E1092A10EB2
:1040D0001092A20E1092A30E1092A40E1092A50E92
:1040E0001092A60E1092B30E1092A70E1092A80E68
:1040F0001092A90E1092AA0E1092AB0E1092AC0E56
:104100001092AD0E1092AE0E1092AF0E1092B00E35
:104110001092B10E1092B20E1092B40E1092B50E13
:104120001092B60E1092B70E0E9405C389E60E9447
:10413000CDAD6FE089ED94E10E94756C89ED94E15D
:104140000E94917489E60E94CDAD41E050E069E69D
:1041500070E089ED94E10E94DD740E94C7B1F82EF1
:1041600089ED94E10E94917483EDF816A1F1043178
:10417000110509F04EC6992009F4ADC08091E10CFB
:10418000811153C0409041155090421560904315E5
:1041900070904415498E5A8E6B8E7C8EC09045155A
:1041A000D0904615E0904715F0904815CD8EDE8EE4
:1041B000EF8EF8A28091491590914A15A0914B1568
:1041C000B0914C158EA39FA3A8A7B9A789A39AA3C2
:1041D000ABA3BCA3ABC06FEA80E20E94EEC260E07A
:1041E00081E20E94EEC268E082E20E94EEC260E2DA
:1041F00083E20E94EEC289E29CE5AFE8BDE38093D2
:10420000B80E9093B90EA093BA0EB093BB0E60E0B7
:1042100084E20E94EEC20431110509F4ACCF81E0C2
:104220008093E10C992009F456C061EC7DE0CE0149
:1042300001960E94F9C8CE0101960E942813CE0172
:1042400001960E949FC889E60E94CDAD63E289ED88
:1042500094E10E94756C89ED94E10E94917489E665
:104260000E94CDAD41E050E069E670E089ED94E157
:104270000E94DD749091080F8091090F9817F1F357
:104280000E94C7B18C0189ED94E10E949174C8012C
:1042900024E0959587952A95E1F78370992761EB3E
:1042A0007DE08130910559F068EA7DE0823091052A
:1042B00031F069EB7DE0892B11F060EA7DE0CE0101
:1042C00001960E94F9C8CE0101960E940B13CE01FF
:1042D00001960E949FC840904115509042156090F1
:1042E000431570904415498E5A8E6B8E7C8EC0900B
:1042F0004515D0904615E0904715F0904815CD8EA5
:10430000DE8EEF8EF8A28091491590914A15A0910A
:104310004B15B0914C158EA39FA3A8A7B9A789A34D
:104320009AA3ABA3BCA3992009F44CC06BE87DE031
:1043300082E891E10E94BAD18091E10C60E77DE0D2
:10434000811102C068E67DE082E891E10E94BAD165
:1043500082E891E10E9450CB6CE77DE0CE010196AE
:104360000E94F9C8CE0101960E94051ECE01019659
:104370000E949FC88E01075E1F4F5E0195E2A90E45
:10438000B11CD8016D917D918D919D918D0146E07B
:1043900050E00E9466CC6EE277E082E891E10E94F4
:1043A000C4CC0A151B0569F761E47CE0CE010196D7
:1043B0000E940BC9CE0101960E94051ECE010196F6
:1043C0000E949FC823E938E144E85FE3C301B201DA
:1043D0000E942AE12B013C014D865E866F86788A19
:1043E00022E430E645E85FE3C701B6010E942AE116
:1043F0006B017C01C98ADA8AEB8AFC8A25E83BEEEC
:1044000041E95FE36EA17FA188A599A50E942AE1F9
:104410006D8B7E8B8F8B988F4092411550924215F9
:104420006092431570924415C0924515D09246157E
:10443000E0924715F09248156093491570934A151C
:1044400080934B1590934C15992009F4A2C080914C
:104450007E0E882309F49DC06BE57DE0CE010196B8
:104460000E94F9C8CE0101960E94051ECE01019658
:104470000E949FC88E01035F1F4F6E01B9E1CB0EF2
:10448000D11C7801F80161917191819191918F0115
:1044900042E050E00E9466CC6EE277E082E891E173
:1044A0000E94C4CCC016D10669F761E47CE0CE015D
:1044B00001960E940BC9CE0101960E94051ECE01F5
:1044C00001960E949FC84DE455E166E070E082E3EA
:1044D0000E94E9C1A0904D15B0904E15C0904F15A7
:1044E000D090501500915115109152156EE47DE059
:1044F00082E891E10E94BAD14AE050E0B50182E839
:1045000091E10E9477CC6EE277E082E891E10E942F
:10451000C4CC4AE050E0B60182E891E10E9477CC39
:104520006EE277E082E891E10E94C4CC4AE050E07C
:10453000B80182E891E10E9477CC61E47CE082E8F6
:1045400091E10E946BCBCE0101960E9485C265E489
:104550007DE082E891E10E94BAD18E010F5F1F4F8A
:10456000D8016D917D918D919D918D014AE050E032
:104570000E9466CC6EE277E082E891E10E94C4CCB2
:104580000E151F0569F761E47CE082E891E10E9465
:104590006BCB61E08DE10E9443C29920B1F0809124
:1045A0007E0E882391F061E37DE082E891E10E9434
:1045B000BAD1AE014B5D5F4F61E070E08DE10E94CA
:1045C000E9C18DA190E00E94B1CC62E08EE10E9431
:1045D00043C263E08FE10E9443C264E080E20E9434
:1045E00043C2992009F450C080917E0E882309F4BB
:1045F0004BC065E17DE082E891E10E94BAD1AE0155
:104600004B5D5F4F61E070E08EE10E94E9C1CDA09B
:10461000D12CAE014B5D5F4F61E070E08FE10E94F5
:10462000E9C1EDA0F12CAE014B5D5F4F61E070E0A0
:1046300080E20E94E9C10DA110E04AE050E0B6011D
:1046400082E891E10E9477CC6EE277E082E891E126
:104650000E94C4CC4AE050E0B70182E891E10E9498
:1046600077CC6EE277E082E891E10E94C4CC4AE028
:1046700050E0B80182E891E10E9477CC61E47CE0EF
:1046800082E891E10E946BCB65E081E20E9443C227
:104690009920B1F080917E0E882391F062E07DE058
:1046A00082E891E10E94BAD1AE014B5D5F4F61E0BB
:1046B00070E081E20E94E9C18DA190E00E94B1CC3E
:1046C00066E082E20E9443C29920B1F080917E0EA2
:1046D000882391F06AEE7CE082E891E10E94BAD1F1
:1046E000AE014B5D5F4F61E070E082E20E94E9C184
:1046F0008DA190E00E94B1CC67E083E20E9443C2AA
:104700009920B1F080917E0E882391F064ED7CE0D9
:1047100082E891E10E94BAD1AE014B5D5F4F61E04A
:1047200070E083E20E94E9C18DA190E00E94B1CCCB
:1047300068E084E20E9443C29920B1F080917E0E2D
:10474000882391F06CEB7CE082E891E10E94BAD181
:10475000AE014B5D5F4F61E070E084E20E94E9C111
:104760008DA190E00E94B1CC69E085E20E9443C235
:104770009920B1F080917E0E882391F062EA7CE06E
:1047800082E891E10E94BAD1AE014B5D5F4F61E0DA
:1047900070E085E20E94E9C18DA190E00E94B1CC59
:1047A0006AE086E20E9443C29920B1F080917E0EB9
:1047B000882391F06CE87CE082E891E10E94BAD114
:1047C000AE014B5D5F4F61E070E086E20E94E9C19F
:1047D0008DA190E00E94B1CC6BE088E20E9443C2C0
:1047E0009920B1F080917E0E882391F063E77CE000
:1047F00082E891E10E94BAD1AE014B5D5F4F61E06A
:1048000070E088E20E94E9C18DA190E00E94B1CCE5
:104810006CE089E20E9443C2992009F479C080913A
:104820007E0E882309F474C06BE57CE082E891E198
:104830000E94BAD1AE014B5D5F4F61E070E089E24A
:104840000E94E9C18DA190E00E94B1CC64E47CE0BB
:1048500082E891E10E94BAD166E070E087E20E94AE
:1048600028C290E00E94B1CC6DE27CE082E891E148
:104870000E94BAD165E070E087E20E9428C290E011
:104880000E94B1CC66E17CE082E891E10E94BAD15D
:1048900064E070E087E20E9428C290E00E94B1CC00
:1048A0006DEF7BE082E891E10E94BAD162E070E0B6
:1048B00087E20E9428C290E00E94B1CC64EE7BE0C7
:1048C00082E891E10E94BAD161E070E087E20E9443
:1048D00028C290E00E94B1CC6BEC7BE082E891E1D1
:1048E0000E94BAD170E060E087E20E9428C290E0A6
:1048F0000E94B1CC6AEB7BE082E891E10E94BAD1E0
:1049000063E070E087E20E9428C290E00E94B1CC90
:1049100041E067E070E087E20E945AC241E063E054
:1049200070E087E20E945AC241E063E070E08AE2F0
:104930000E945AC2992091F080917E0E882371F0D6
:1049400061EA7BE082E891E10E94BAD163E070E025
:104950008AE20E9428C290E00E94B1CC40E063E06D
:1049600070E08AE20E945AC2992091F080917E0EF6
:10497000882371F067E87BE082E891E10E94BAD178
:1049800063E070E08AE20E9428C290E00E94B1CC0D
:1049900041E062E070E08AE20E945AC2992091F000
:1049A00080917E0E882371F06BE67BE082E891E1D6
:1049B0000E94BAD162E070E08AE20E9428C290E0D0
:1049C0000E94B1CC40E062E070E08AE20E945AC2EC
:1049D000992091F080917E0E882371F06EE47BE047
:1049E00082E891E10E94BAD162E070E08AE20E941E
:1049F00028C290E00E94B1CC41E061E070E08AE220
:104A00000E945AC2992091F080917E0E882371F005
:104A100062E37BE082E891E10E94BAD161E070E05C
:104A20008AE20E9428C290E00E94B1CC40E061E09E
:104A300070E08AE20E945AC2992091F080917E0E25
:104A4000882371F065E17BE082E891E10E94BAD1B0
:104A500061E070E08AE20E9428C290E00E94B1CC3E
:104A600041E070E060E08AE20E945AC2992091F031
:104A700080917E0E882371F069EF7AE082E891E1FF
:104A80000E94BAD170E060E08AE20E9428C290E001
:104A90000E94B1CC40E070E060E08AE20E945AC21D
:104AA000992091F080917E0E882371F06CED7AE070
:104AB00082E891E10E94BAD170E060E08AE20E944F
:104AC00028C290E00E94B1CC41E066E070E087E24D
:104AD0000E945AC241E065E070E087E20E945AC23B
:104AE00041E064E070E087E20E945AC240E062E088
:104AF00070E087E20E945AC240E061E070E087E225
:104B00000E945AC240E070E060E087E20E945AC210
:104B1000992009F475C080917E0E882309F470C035
:104B200064EC7AE082E891E10E94BAD166E070E03C
:104B30008BE20E9428C290E00E94B1CC66EA7AE043
:104B400082E891E10E94BAD165E070E08BE20E94B8
:104B500028C290E00E94B1CC68E87AE082E891E156
:104B60000E94BAD164E070E08BE20E9428C290E01B
:104B70000E94B1CC6FE67AE082E891E10E94BAD15E
:104B800062E070E08BE20E9428C290E00E94B1CC0B
:104B900066E57AE082E891E10E94BAD161E070E0D6
:104BA0008BE20E9428C290E00E94B1CC6DE37AE0D3
:104BB00082E891E10E94BAD170E060E08BE20E944D
:104BC00028C290E00E94B1CC6AE27AE082E891E1EA
:104BD0000E94BAD163E070E08BE20E9428C290E0AC
:104BE0000E94B1CC65E17AE082E891E10E94BAD1FD
:104BF00064E070E08CE20E9428C290E00E94B1CC98
:104C000040E064E070E08CE20E945AC2AE014B5D6D
:104C10005F4F61E070E08CE20E94E9C16DA1607FAE
:104C200066608CE20E9443C2992009F45EC08091C4
:104C30007E0E882309F459C061E07AE082E891E1B0
:104C40000E94BAD1AE014B5D5F4F61E070E08CE233
:104C50000E94E9C16DA16F706650770B072E000CA2
:104C6000880B990B0E94CBE09B01AC0160E070E0E7
:104C700080E090E40E9417E520E030E048EC50E44A
:104C80000E942AE10E9468CC6AEE79E082E891E114
:104C90000E94BAD1AE014B5D5F4F61E070E080E3EE
:104CA0000E94E9C16DA14AE050E082E891E10E94D2
:104CB00054CB62ED79E082E891E10E94BAD161E0E3
:104CC00070E080E30E9428C290E00E94B1CC69EBC2
:104CD00079E082E891E10E94BAD161E070E08FE270
:104CE0000E9428C290E00E94B1CC41E061E070E0F7
:104CF0008FE20E945AC2992091F080917E0E882303
:104D000071F061EA79E082E891E10E94BAD161E054
:104D100070E08EE20E9428C290E00E94B1CC41E097
:104D200061E070E08EE20E945AC240E067E070E00D
:104D300081E30E945AC2992009F455C080917E0EE9
:104D4000882309F450C06EE879E082E891E10E947E
:104D5000BAD167E070E081E30E9428C290E00E942F
:104D6000B1CC6AE076E082E891E10E94C4CCAE0169
:104D70004B5D5F4F61E070E080E00E94E9C18DA172
:104D80000E94D27261E47CE082E891E10E946BCBE8
:104D90000DE110E06CE679E082E891E10E94C4CC7C
:104DA00040E150E0B80182E891E10E9477CC6EE0EA
:104DB00076E082E891E10E94C4CCAE014B5D5F4F8A
:104DC00061E070E0802F0E94E9C18DA10E94D27243
:104DD00061E47CE082E891E10E946BCB0F5F1F4FA2
:104DE0000A331105B9F6A9960FB6F894DEBF0FBEC7
:104DF000CDBFDF91CF911F910F91FF90EF90DF908A
:104E0000CF90BF90AF909F907F906F905F904F90AA
:104E10000895992091F080917E0E882371F06EECB8
:104E20007DE0CE0101960E94F9C8CE0101960E9454
:104E30000B13CE0101960E949FC864E670E080E0EB
:104E400090E00E94086E0F5F1F4F34C91F93CF93ED
:104E5000DF9300D000D0CDB7DEB7182F8091871335
:104E6000909188138130910509F059C0112331F0D8
:104E700062E874E082E891E10E94BAD10E9406C122
:104E8000112339F04AE050E0682F82E891E10E9456
:104E900054CB0E94EDBE112309F4D5C00E94FDBC85
:104EA00061E176E0CE0101960E940BC940910C159C
:104EB00050910D1560910E1570910F15CE01019650
:104EC0000E94B9C768E176E0CE0101960E940DC844
:104ED0004091101550911115609112157091131594
:104EE000CE0101960E94B9C76CE176E0CE01019631
:104EF0000E940DC84091141550911515609116151A
:104F000070911715CE0101960E94B9C7CE01019686
:104F10000E940B13CE0101960E949FC894C0009777
:104F200009F0A4C08AE097E5A4EFB2E48093D00E24
:104F30009093D10EA093D20EB093D30E8BE794E151
:104F4000A6E6B3E48093CC0E9093CD0EA093CE0E44
:104F5000B093CF0E8DEC9CEEA2ECB3E48093C80E20
:104F60009093C90EA093CA0EB093CB0E89E29CE534
:104F7000AFE8BFE38093090590930A05A0930B0562
:104F8000B0930C0587ED93EAA0E9BFE38093050594
:104F900090930605A0930705B09308058AE097ED66
:104FA000A3E8BFE38093010590930205A093030556
:104FB000B09304058EE10E94CDAD61E070E089ED13
:104FC00094E10E94EF1386EF98E2ACE9BFE380938F
:104FD0000D0590930E05A0930F05B093100560E4A6
:104FE00089ED94E10E94756C63E070E089ED94E1D5
:104FF0000E94EF1389ED94E10E9491748091E60E76
:105000009091E70E18161906C4F462E276E082E881
:1050100091E10E94C4CC60910D0570910E058091C4
:105020000F059091100542E050E00E9466CC66E3C7
:1050300076E082E891E10E946BCB11110EC01092D4
:10504000E70E1092E60E26960FB6F894DEBF0FBE5E
:10505000CDBFDF91CF911F91089581E090E09093B3
:10506000E70E8093E60E0E94C6CCEDCF019639F490
:105070006DE674E0CE0101960E94F9C847CF64EF57
:1050800071E080E090E00E94086EDDCF4F925F9269
:105090006F927F928F929F92AF92BF92CF92DF9248
:1050A000EF92FF921F93CF93DF93CDB7DEB72C978C
:1050B0000FB6F894DEBF0FBECDBF182F80919A0DAA
:1050C0008111D2C080E492E090930902809308029B
:1050D0000E94916E8093DC1581E492E00E94916EB3
:1050E0008093DD1582E492E00E94916E8093DE153C
:1050F00083E492E00E94916E8093DF1580E492E059
:105100000E94916E8F3FE1F0E0900802F09009025A
:1051100030EEA32E35E1B32E6501C7018C5D9541BC
:105120004C0124EEC21625E1D20609F441C0C401A7
:105130008C0D9D1D0E94916EF60181936F01F1CF40
:1051400081E492E00E94916E8F3FF1F682E492E05A
:105150000E94916E8F3FC1F683E492E00E94916EAF
:105160008F3F91F680E090E0A0E8BFE38093DC15EC
:105170009093DD15A093DE15B093DF152CEDC22EB4
:1051800025E1D22EF12CE12C8091080290910902A8
:10519000E4E0EE16F10409F4B7CFF60161916F0176
:1051A0008E0D9F1D0E94F3E1FFEFEF1AFF0AECCF77
:1051B000C70104960E94916E8F3F99F5C70105962D
:1051C0000E94916E8F3F69F5C70106960E94916E0D
:1051D0008F3F39F5C70107960E94916E8F3F09F501
:1051E00080E090E0A0E8BFE38093E0159093E115A4
:1051F000A093E215B093E315F12CE12CF501619138
:105200005F01809108029091090204968E0D9F1D06
:105210000E94F3E1FFEFEF1AFF0A24E0E216F10427
:1052200069F78091DC159091DD15A091DE15B091A4
:10523000DF158093D8159093D915A093DA15B09304
:10524000DB150E943B6E6093960D7093970D8093D3
:10525000980D9093990D81E080939A0D68EE73E01C
:1052600080E090E00E94086E80918E0D81110DC04B
:105270000E943B6E60938A0D70938B0D80938C0D12
:1052800090938D0D81E080938E0D0E943B6EC090B7
:105290008A0DD0908B0DE0908C0DF0908D0D6C19D7
:1052A0007D098E099F09693E73408105910508F4C7
:1052B0004BC10E943B6E60938A0D70938B0D80935F
:1052C0008C0D90938D0D8BE30E94C06DBC01990FE6
:1052D000880B990B0E94CBE020E030E040E85AE3D5
:1052E0000E942AE120E030E44CE955E40E942AE1E2
:1052F0006B017C01C092860DD092870DE092880DE3
:10530000F092890D87E390E00E941F0F4B015C0132
:1053100080920A0290920B02A0920C02B0920D02AF
:1053200020E030E04AE754E4C701B6010E942AE1D8
:1053300020E030E04DE454E40E9443E320E030E01C
:1053400048E453E40E9443E36B017C01C092EC15F6
:10535000D092ED15E092EE15F092EF152091D81550
:105360003091D9154091DA155091DB150E942AE150
:105370002B013C0120E030E040E250E40E944CE48C
:1053800018160CF02AC18091E0159091E115A091BA
:10539000E215B091E3158093D8159093D915A09399
:1053A000DA15B093DB152091D8153091D9154091BD
:1053B000DA155091DB15C701B6010E942AE16B0195
:1053C0007C0120E030E048EC51E4C501B4010E94CA
:1053D00064E220E53DE847E95CE30E942AE120E041
:1053E00030E040E85FE30E9465E29B01AC01C70149
:1053F000B6010E9443E3AB01BC014093D415509326
:10540000D5156093D6157093D71522E0CE01079677
:105410000E94A7C86EE376E0CE0101960E940BC9F8
:10542000BE01695F7F4FCE0101960E947CC762E496
:1054300076E00E9466C7BC0188E994E10E9443C8F7
:10544000CE0101960E949FC8CE0107960E949FC878
:1054500040910A0250910B0260910C0270910D0272
:1054600021E0CE0107960E94A7C86DEB76E0CE0141
:1054700001960E940BC9BE01695F7F4FCE01019664
:105480000E947CC7BC0184EA94E10E9443C8CE011B
:1054900001960E949FC8CE0107960E949FC868E9A6
:1054A00074E1CE0101960E9402C96EE277E0CE015E
:1054B00001960E9466C764EA74E10E947CC768E4B2
:1054C00076E00E9466C7BC018EE994E10E9443C861
:1054D000CE0101960E949FC864EA74E1CE01019654
:1054E0000E9402C94AE050E06FEF7FEFCE010196C3
:1054F0000E94FD19CE0101960E949FC865E070E0F0
:1055000080E090E00E94086E65E079E0CE010196AF
:105510000E940BC9CE0101960E940310CE01019694
:105520000E949FC868E974E1CE0101960E9402C9F9
:105530004AE050E06FEF7FEFCE0101960E946313C7
:10554000CE0101960E949FC80E943B6EC090960DAE
:10555000D090970DE090980DF090990D6C197D0901
:105560008E099F096235734081059105E0F00E9424
:105570003B6E6093960D7093970D8093980D90936A
:10558000990D87E390E00E941F0F60930A027093C9
:105590000B0280930C0290930D026EE170E080E0AC
:1055A00090E00E94086E11112BC010E0812F2C9604
:1055B0000FB6F894DEBF0FBECDBFDF91CF911F9124
:1055C000FF90EF90DF90CF90BF90AF909F908F9023
:1055D0007F906F905F904F90089520E030E040E022
:1055E00050E4C301B2010E94C4E087FFDCCE809189
:1055F000DC159091DD15A091DE15B091DF15CBCEB5
:1056000080900A0290900B02A0900C02B0900D02C4
:105610004090860D5090870D6090880D7090890D98
:105620004092E4155092E5156092E6157092E715E8
:105630008092E8159092E915A092EA15B092EB15C8
:10564000123059F0133009F431C1113009F0ADCFE7
:105650001093850D1092840DA9CF8091850D88231C
:1056600009F4A3CFC090EC15D090ED15E090EE15A5
:10567000F090EF1526E636E646E65FE3C701B60191
:105680000E944CE418160CF0B3C023E333E343EF5D
:105690005FE3C701B6010E94C4E087FFA9C020E014
:1056A00030E048EC51E4C501B4010E9464E220E519
:1056B0003DE847E95CE30E942AE120E030E040E871
:1056C0005FE30E9465E22FE23DED44EB5FE30E9461
:1056D0002AE16093800D7093810D8093820D9093E9
:1056E000830D20E038E240E258E46091800D709133
:1056F000810D8091820D9091830D0E942AE120E01E
:1057000030E04AE754E40E9443E3A30192010E947F
:1057100043E34B015C0120E030E040E05FE30E94A6
:105720004CE418160CF0B0C020E030E040EC5FE331
:10573000C501B4010E94C4E087FFA6C08092D815BD
:105740009092D915A092DA15B092DB1526E636E6CE
:1057500046E65FE3C701B6010E944CE418160CF060
:1057600075C023E333E343EF5FE3C701B6010E9453
:10577000C4E087FF6BC08092DC159092DD15A0928B
:10578000DE15B092DF1581E08093840D6DED72E13E
:10579000CE0101960E94F9C8CE0101960E942813FD
:1057A000CE0101960E949FC84091D8155091D915FD
:1057B0006091DA157091DB1523E0CE0101960E940D
:1057C000A7C8CE0101960E940B13CE0101960E943C
:1057D0009FC860EC72E1CE0101960E94F9C8CE012B
:1057E00001960E940B13CE0101960E949FC8DECE47
:1057F00020E030E040E151E4C701B6010E944CE4F2
:1058000018160CF06ECF26E636E646E851E4C701DE
:10581000B6010E94C4E087FF64CF20E030E048EC8E
:1058200051E4C501B4010E9464E220E53DE847E986
:105830005CE30E942AE120E030E040E85FE30E9460
:1058400065E22BE734E14EE451E441CF20E030E063
:1058500040E151E4C701B6010E944CE418160CF077
:1058600092CF26E636E646E851E4C701B6010E942B
:10587000C4E087FF88CF8092E0159092E115A09256
:10588000E215B092E3157FCF1092840D6BE073E1C7
:10589000CE0101960E94F9C8CE0101960E940B1319
:1058A000CE0101960E949FC815E180CE8091850DA2
:1058B000882309F47ACE82E891E10E9450CB80914E
:1058C000840D882309F47DC0C090EC15D090ED15AF
:1058D000E090EE15F090EF1526E636E646E65FE33B
:1058E000C701B6010E944CE41816ECF523E333E33C
:1058F00043EF5FE3C701B6010E94C4E087FF33C0F6
:105900009CEDC92E95E1D92EF12CE12CF601619187
:105910006F0180910802909109028E0D9F1D0E94D7
:10592000F3E1FFEFEF1AFF0A24E0E216F10471F74A
:105930001092840D1092850D1A3008F444C064EF63
:1059400072E11E3109F032CECE0101960E94F9C8F3
:10595000CE0101960E940B13CE0101960E949FC8B2
:105960001092A30D23CE20E030E040E151E4C701C6
:10597000B6010E944CE41816DCF626E636E646E848
:1059800051E4C701B6010E94C4E087FFD1CF80EE89
:10599000C82E85E1D82EF12CE12CF60161916F0122
:1059A000809108029091090204968E0D9F1D0E941D
:1059B000F3E1FFEFEF1AFF0A24E0E216F10469F7C2
:1059C000B7CF1EE1B5CF133009F0F0CD65EA72E133
:1059D000BBCF8F929F92AF92BF92CF92DF92EF9206
:1059E000FF920F931F93CF93DF93CDB7DEB72C9722
:1059F0000FB6F894DEBF0FBECDBFD82E0DB71EB7C1
:105A00008091740D811105C00E943B6E81E08093EE
:105A1000740D80916C0D811105C00E943B6E81E078
:105A200080936C0D8091640D811105C00E943B6EC6
:105A300081E08093640D60E08D2D0E94806D64E6AE
:105A400070E080E090E00E94086E1092630D10926A
:105A5000620DE090620DF090630D4EE1E416F104EA
:105A6000D4F48D2D0E94C06DF701EE0FFF1FEA5D8B
:105A7000F24F918380836EE170E080E090E00E94BD
:105A8000086E8091620D9091630D01969093630D65
:105A90008093620DDECF87E390E00E941F0F60933A
:105AA0007F04709380048093810490938204E6E2E3
:105AB000FDE028EE3CE0D9018DE0E236F80729F060
:105AC000819191918D939D93F7CF8EE190E090938A
:105AD000250D8093240DADB6BEB6ADB7BEB7DC972D
:105AE0000FB6F894BEBF0FBEADBFEDB7FEB731968F
:105AF0004F01DF0180E0F901619171919F016D9388
:105B00007D938F5F8E31B9F78DE190E0F40130E045
:105B100020E0281739079CF4619171912F5F3F4F66
:105B2000E080F180E616F706A4F76F0142E0C41AA0
:105B3000D108D601ED92FC9271836083EACF019780
:105B400029F7F401668D778D848D958D680F791F07
:105B500077FF02C06F5F7F4F759567950FB6F8941A
:105B6000BEBE0FBEADBE072E000C880B990B0E9467
:105B7000CBE020E030E44CE955E40E942AE120E04B
:105B800030EC4FE754E40E9443E36B017C01C09288
:105B90009E0DD0929F0DE092A00DF092A10D20E0FD
:105BA00030E040E05FE36091D30D7091D40D8091BF
:105BB000D50D9091D60D0E9465E20E94EFE3FB01A6
:105BC000EE0FFF1FEE0FFF1FEF5FFD4E259135918A
:105BD00045915491C701B6010E942AE12091D70D49
:105BE0003091D80D4091D90D5091DA0D0E9443E3C8
:105BF000AB01BC0140937C0D50937D0D60937E0DF5
:105C000070937F0D22E0CE0107960E94A7C868E539
:105C100076E0CE0101960E940BC9BE01695F7F4FFD
:105C2000CE0101960E947CC76CE576E00E9466C7B3
:105C3000BC0188E994E10E9443C8CE0101960E940C
:105C40009FC8CE0107960E949FC840917F04509143
:105C50008004609181047091820421E0CE01079656
:105C60000E94A7C86DEB76E0CE0101960E940BC999
:105C7000BE01695F7F4FCE0101960E947CC7BC01C7
:105C800084EA94E10E9443C8CE0101960E949FC815
:105C9000CE0107960E949FC868E974E1CE01019683
:105CA0000E9402C964EA74E1CE0101960E947CC799
:105CB00062E676E00E9466C7BC018EE994E10E942C
:105CC00043C8CE0101960E949FC864EA74E1CE01E8
:105CD00001960E9402C94AE050E070E060E0CE0107
:105CE00001960E94FD19CE0101960E949FC865E0B1
:105CF00070E080E090E00E94086E65E079E0CE01FF
:105D000001960E940BC9CE0101960E940310CE019C
:105D100001960E949FC868E974E1CE0101960E9435
:105D200002C94AE050E06FEF7FEFCE0101960E947A
:105D30006313CE0101960E949FC80FB6F8941EBF50
:105D40000FBE0DBF2C960FB6F894DEBF0FBECDBFB1
:105D5000DF91CF911F910F91FF90EF90DF90CF9047
:105D6000BF90AF909F908F9008952F923F924F9247
:105D70005F926F927F928F929F92AF92BF92CF92DB
:105D8000DF92EF92FF920F931F93CF93DF93CDB7E4
:105D9000DEB768970FB6F894DEBF0FBECDBF2B01FC
:105DA0003C010E943B6E6D877E878F87988B88E4CD
:105DB00090E10E94E8B062E370E080E090E00E9431
:105DC000086E61E08091A6040E94806D60E0809181
:105DD000A4040E94806D64E670E080E090E00E9480
:105DE000086E6091A0047091A1048091A20490912A
:105DF000A3040E948B100E94AF0F7B018C010E94B4
:105E0000E36D4B015C0160E570E080E090E00E9492
:105E1000086E62E776E08EE994E10E94E2C520E038
:105E200030E04AE754E4C301B2010E942AE16D8BDD
:105E30007E8B8F8B988F412C512C320160E070E06B
:105E4000CB010E94CBE02D893E894F89588D0E945D
:105E5000C4E087FF87C10E943B6E2D853E854F853C
:105E60005889621B730B840B950B0E94C9E020E0DC
:105E700030E04AE754E40E9443E3AB01BC0123E075
:105E8000CE0101960E94A7C8BE016F5F7F4F88E9CF
:105E900094E10E945AC8CE0101960E949FC80E94B8
:105EA000AF0FD62EC72E382E292E0E94E36D698B98
:105EB0007A8B8B8B9C8BDC01CB0188199909AA0901
:105EC000BB094C015D0191ED891697E09906A1048B
:105ED000B104BCF020E030E0A9016D2D7C2D832DB4
:105EE000922D0E944CE4181684F426EA3BE944EC17
:105EF0005BE36D2D7C2D832D922D0E94C4E087FFE6
:105F000010C0812C912C54012EC026EA3BE944ECB0
:105F10005BEB6D2D7C2D832D922D0E944CE4181689
:105F200084F3C501B40128EE33E040E050E00E9464
:105F300001E2CA01B9010E94CBE04B015C0197016B
:105F4000A8016D2D7C2D832D922D0E9464E220E00E
:105F500030E04AE754E40E942AE1A50194010E943E
:105F600043E34B015C0168E974E1CE0101960E94B4
:105F700002C965E577E0CE0101960E9466C7BC01C3
:105F800088E994E10E9443C8CE0101960E949FC80F
:105F900023E04D2D5C2D632D722DCE0101960E94C4
:105FA000A7C8BE016F5F7F4FCE0107960E9402C94E
:105FB00060E976E0CE0107960E9466C7BC0182E9DF
:105FC00094E10E9443C8CE0107960E949FC8CE016B
:105FD00001960E949FC822E0B501A401CE01079658
:105FE0000E94A7C869EB77E0CE0101960E940BC919
:105FF00068E974E1CE0101960E947CC763E976E00E
:106000000E9466C762E974E10E947CC762E378E09F
:106010000E9466C7BE01695F7F4F0E947CC767E927
:1060200076E00E9466C7BC018EE994E10E9417C821
:10603000CE0101960E949FC8CE0107960E949FC87C
:1060400020E030E0A901C501B4010E944CE487FDC5
:1060500006C06EE277E082E994E10E940DC822E07A
:10606000B501A401CE0101960E94A7C8BE016F5FD1
:106070007F4FCE0107960E9402C967E976E0CE0104
:1060800007960E9466C7BC0182E994E10E9417C886
:10609000CE0107960E949FC8CE0101960E949FC81C
:1060A0006EE974E1CE0101960E9402C9CE0101960B
:1060B0000E940B13CE0101960E949FC8C301B2013A
:1060C00025E030E040E050E00E9401E2672B682BC1
:1060D000692B21F567EB7EE0CE0101960E94F9C89D
:1060E00045E050E070E060E0CE0101960E94FD19AD
:1060F000CE0101960E949FC862E974E1CE0101962B
:106100000E9402C945E050E06FEF7FEFCE0101969B
:106110000E946313CE0101960E949FC861E47CE057
:106120008EE994E10E94E2C562E370E080E090E0D5
:106130000E94086E0E943B6E2D853E854F855889D2
:10614000621B730B840B950B3FEF431A530A630AD0
:10615000730A89889A88AB88BC88ED2CFC2C032DA7
:10616000122D6FCE60E08091A6040E94806D68962B
:106170000FB6F894DEBF0FBECDBFDF91CF911F9158
:106180000F91FF90EF90DF90CF90BF90AF909F90D6
:106190008F907F906F905F904F903F902F900895D9
:1061A0008F929F92AF92BF92CF92DF92EF92FF9227
:1061B0000F931F93CF93DF93CDB7DEB7EA970FB658
:1061C000F894DEBF0FBECDBFF82E61E47CE0CE01B7
:1061D000C5960E940BC98E010B5E1F4F6F2DC80123
:1061E0000E94B67118870F831D821E82198289E072
:1061F0008A8381E08B838C831C8A1B8ACE01019663
:106200000E940B71CE0101960E94AE6FCE010196E5
:106210000E94C1C30E8110E00330110509F488C14A
:106220006DEA7EE0CE01C5960E941EC861E47CE066
:106230008EE994E10E94E2C5BE016B5C7F4FCE0106
:1062400083960E9402C94AE050E070E060E0CE010F
:1062500083960E94FD19CE0183960E949FC861E03B
:1062600080E00E94E8AD6DEB76E0CE01C5960E941D
:10627000E2C584EFC82E8DE0D82EF12CE12CE0167B
:10628000F1060CF0F0C06E2DCE0101960E949F70B9
:10629000F60121913191419151916F010E9465E286
:1062A0004B015C01FFEFEF1AFF0A20E030E04CEFFA
:1062B00052EC0E94C4E087FF33C0B701CE0189963B
:1062C0000E9419C664EC7AE0CE0183960E940BC945
:1062D000BE01675D7F4FCE0183960E947CC76BE94C
:1062E00076E00E9466C7BC018EE994E10E9417C85F
:1062F000CE0183960E949FC8CE0189960E949FC8B6
:106300000130110509F055C081E0E816F10409F0EB
:10631000B6CF6EE974E1CE01C5960E9443C8AFCFF7
:1063200022E0B501A401CE018F960E94A7C8B70153
:10633000CE0189960E9419C664EC7AE0CE0183965C
:106340000E940BC9BE01675D7F4FCE0183960E94FC
:106350007CC76EEE75E00E9466C7BE01615D7F4F2F
:106360000E947CC7BC0182E994E10E9443C8CE012F
:1063700083960E949FC8CE0189960E949FC8CE0135
:106380008F960E949FC862E974E1CE0183960E94B5
:1063900002C96EE277E0CE0183960E9466C7BC0117
:1063A0008EE994E10E9417C8CE0183960E949FC88F
:1063B000A7CF0230110511F522E0B501A401CE01ED
:1063C00083960E94A7C8BE016D5D7F4FCE0189965E
:1063D0000E9402C96EE277E0CE0189960E9466C7EC
:1063E000BC01CE01C5960E9417C8CE0189960E94B5
:1063F0009FC8CE0183960E949FC841CF03301105EC
:1064000009F43DCF62E974E1CE0183960E9402C98E
:1064100044E150E06FEF7FEFCE0183960E9463135B
:10642000CE0183960E949FC865E079E0CE018396F5
:106430000E940BC9CE0183960E940310CE01839661
:106440000E949FC880919D04882309F418CF8091F1
:10645000FB04882309F413CF60ED77E080E090E03F
:106460000E94086E0CCFCE01C5960E946AC68EE9C6
:1064700094E10E946AC60115110579F56AE97EE08A
:106480008EE994E10E941EC86FE87EE0CE018396FB
:106490000E94F9C84AE050E06FEF7FEFCE0183968B
:1064A0000E946313CE0183960E949FC8CE01C596B9
:1064B0000E949FC8EA960FB6F894DEBF0FBECDBF0C
:1064C000DF91CF911F910F91FF90EF90DF90CF90D0
:1064D000BF90AF909F908F900895043011050CF5F8
:1064E000BE016B5C7F4FCE0183960E9402C94AE0D9
:1064F00050E06FEF7FEFCE0183960E946313CE01D1
:1065000083960E949FC865E079E0CE0183960E9441
:106510000BC9CE0183960E940310CE0183960E9480
:106520009FC867EA76E08EE994E10E940DC8BECF6D
:106530006AEB76E0CE01C5960E94E2C5BE016B5CB7
:106540007F4FCE0183960E9402C94AE050E070E07E
:1065500060E0CE0183960E94FD19CE0183960E94D1
:106560009FC861E47CE08EE994E10E94E2C56EE997
:1065700074E1CE01C5960E9443C810E000E0602F90
:10658000CE0101960E949F706B017C0122E0BC014C
:10659000A601CE0183960115110509F077C00E946E
:1065A000A7C8BE016D5D7F4F86E296E10E949AD139
:1065B000CE0183960E949FC822E0B701A601CE01BA
:1065C00083960E94A7C8BE016D5D7F4FCE0189965C
:1065D0000E9402C96EE277E0CE0189960E9466C7EA
:1065E000BC018EE994E10E9417C8CE0189960E94F1
:1065F0009FC8CE0183960E949FC80F5F1F4F033034
:10660000110509F0BCCFCE01C5960E946AC6BE0135
:106610006B5C7F4FCE0183960E9402C94AE050E036
:106620006FEF7FEFCE0183960E946313CE018396B6
:106630000E949FC865E079E0CE0183960E940BC955
:10664000CE0183960E940310CE0183960E949FC8BC
:106650008EE994E10E946AC660EC76E0CE018396F2
:106660000E940BC96EE974E1CE0183960E947CC73B
:1066700067EA76E00E9466C7BC018EE994E10E9459
:1066800043C8CE0183960E949FC810CF0E94A7C81E
:10669000BE016D5D7F4FCE0189960E9402C96EE2F8
:1066A00077E0CE0189960E9466C7BC01CE01C596EF
:1066B0000E9417C8CE0189960E949FC879CFAF92D9
:1066C000BF92CF92DF92EF92FF920F931F93CF93DF
:1066D000DF93CDB7DEB72C970FB6F894DEBF0FBEB1
:1066E000CDBF80917D0E811102C00E943F13809129
:1066F000A9049091AA04029751F08091F20D909113
:10670000F30D009709F4BAC1039709F4B7C162E227
:106710007EE088E994E10E941EC868E974E1CE0138
:1067200001960E9402C944E150E070E060E0CE01B1
:1067300001960E94FD19CE0101960E949FC863E157
:106740007EE088E994E10E941EC868E974E1CE0108
:1067500001960E9402C944E150E06FEF7FEFCE0145
:1067600001960E946313CE0101960E949FC887E0A4
:106770000E941CC38C0186E00E941CC3BC0190E0F7
:1067800080E00E94C9E02AE037ED43EA5CE30E9422
:106790002AE123E333E948E853E40E9464E26B0111
:1067A0007C0184E0A82EB12C20E030E048EC52E4DB
:1067B000C701B6010E944CE418160CF05FC081E0DE
:1067C000A81AB108E9F064E670E080E090E00E9469
:1067D000086E86E00E941CC3BC0190E080E00E942D
:1067E000C9E02AE037ED43EA5CE30E942AE123E3B3
:1067F00033E948E853E40E9464E26B017C01D4CFA2
:1068000068E07EE088E994E10E941EC868E974E1CE
:10681000CE0101960E9402C94AE050E070E060E0BB
:10682000CE0101960E94FD19CE0101960E949FC8DB
:106830006AEC76E0CE0101960E940BC968E974E12A
:10684000CE0101960E947CC7BC018EE994E10E94B2
:1068500043C8CE0101960E949FC88091F20D90918D
:10686000F30D049721F41092F30D1092F20D81E0D4
:1068700090E09093AA048093A904DFC0B80190E04F
:1068800080E00E94C9E02AE037ED43EA5CE30E9421
:106890002AE123E333E948E853E40E9464E2AB01D0
:1068A000BC0121E0CE0101960E94A7C86CED76E004
:1068B000CE0107960E940BC9BE016F5F7F4FCE01CC
:1068C00007960E947CC7BC018EE994E10E9443C8F0
:1068D000CE0107960E949FC8CE0101960E949FC8D4
:1068E00083E090E09093F30D8093F20D6EE974E1F4
:1068F000CE0101960E9402C942E350E06FEF7FEFA4
:10690000CE0101960E946313CE0101960E949FC89A
:1069100065E079E0CE0101960E940BC9CE01019697
:106920000E940310CE0101960E949FC865EE76E09A
:106930008EE994E10E940DC821E0B701A601CE01C5
:1069400001960E94A7C86DEB76E0CE0107960E94E3
:106950000BC9BE016F5F7F4FCE0107960E947CC7B7
:10696000BC0184EA94E10E9443C8CE0107960E94CC
:106970009FC8CE0101960E949FC86EE277E0CE01CB
:1069800001960E940BC964EA74E1CE0101960E944F
:106990007CC7BC0188E994E10E9443C8CE010196FE
:1069A0000E949FC868E974E1CE0101960E9402C965
:1069B0004AE050E070E060E0CE0101960E94441988
:1069C000CE0101960E949FC865E079E0CE01019654
:1069D0000E940BC9CE0101960E940310CE010196C0
:1069E0000E949FC865EE76E084EA94E10E940DC89B
:1069F00064EA74E1CE0101960E9402C96EE277E07A
:106A0000CE0101960E9466C76EE974E10E947CC7C0
:106A1000BC018EE994E10E9443C8CE0101960E9418
:106A20009FC88091F20D9091F30D039731F484E0AB
:106A300090E09093F30D8093F20D64E670E080E0B7
:106A400090E00E94086E80917D0E882331F060E214
:106A500073E080E090E00E94086E2C960FB6F894E8
:106A6000DEBF0FBECDBFDF91CF911F910F91FF9081
:106A7000EF90DF90CF90BF90AF90089588E490E1C1
:106A80000E94E8B064E670E080E090E00E94086E4A
:106A900068E47EE088E994E10E941EC868E974E138
:106AA000CE0101960E9402C944E150E070E060E02E
:106AB000CE0101960E94FD19CE0101960E949FC849
:106AC00069E37EE088E994E10E941EC868E974E108
:106AD000CE0101960E9402C944E150E06FEF7FEFC2
:106AE000CE0101960E946313CE0101960E949FC8B9
:106AF0008CE40E9406B16B017C0104E010E0A70168
:106B00009601C701B6010E94B1E5882309F449C086
:106B10000150110961F068EC70E080E090E00E94A3
:106B2000086E8CE40E9406B16B017C01E8CF6EE236
:106B30007EE088E994E10E941EC868E974E1CE0114
:106B400001960E9402C94AE050E070E060E0CE0188
:106B500001960E94FD19CE0101960E949FC86AEC21
:106B600076E0CE0101960E940BC968E974E1CE017E
:106B700001960E947CC7BC018EE994E10E9443C843
:106B8000CE0101960E949FC88091F20D9091F30D65
:106B9000039721F41092F30D1092F20D82E090E031
:106BA00068CE21E0B701A601CE0107960E94A7C8D2
:106BB0006CED76E0CE0101960E940BC9BE01695FC3
:106BC0007F4FCE0101960E947CC7BC018EE994E103
:106BD0000E9443C8CE0101960E949FC8CE0107962D
:106BE0000E949FC883E090E09093F30D8093F20D94
:106BF0006EE974E1CE0101960E9402C942E350E0C1
:106C00006FEF7FEFCE0101960E946313CE010196D4
:106C10000E949FC865E079E0CE0101960E940BC9F1
:106C2000CE0101960E940310CE0101960E949FC8DA
:106C300065EE76E08EE994E10E940DC886E60E943A
:106C400006B16B017C0104E010E0A7019601C701C9
:106C5000B6010E94B1E5882381F00150110909F4C1
:106C600084C068EC70E080E090E00E94086E86E6E8
:106C70000E9406B16B017C01E8CF21E0B701A601BB
:106C8000CE0107960E94A7C86DEB76E0CE01019673
:106C90000E940BC9BE01695F7F4FCE0101960E9421
:106CA0007CC7BC0184EA94E10E9443C8CE010196EE
:106CB0000E949FC8CE0107960E949FC86EE277E0AF
:106CC000CE0101960E940BC964EA74E1CE010196DF
:106CD0000E947CC7BC0188E994E10E9443C8CE01B0
:106CE00001960E949FC868E974E1CE0101960E9456
:106CF00002C94AE050E06FEF7FEFCE0101960E949B
:106D00004419CE0101960E949FC865E079E0CE014A
:106D100001960E940BC9CE0101960E940310CE017C
:106D200001960E949FC865EE76E084EA94E10E9495
:106D30000DC864EA74E1CE0101960E9402C96EE2B8
:106D400077E0CE0101960E9466C76EE974E10E9469
:106D50007CC7BC018EE994E10E9443C8CE01019634
:106D60000E949FC883E090E064CE61E47CE084EA06
:106D700094E10E94E2C5DDCF4F925F926F927F92C5
:106D80008F929F92AF92BF92CF92DF92EF92FF923B
:106D9000CF93DF93CDB7DEB72C970FB6F894DEBF55
:106DA0000FBECDBF0E943F130E9411B32B013C01C7
:106DB0000E94D8B44B015C016091EB047091EC042B
:106DC0008091ED049091EE040E94CBE06B017C0178
:106DD0000E9411B30E94CBE0A70196010E9443E3F9
:106DE00021E03EED42E45EE30E9417E59B01AC0129
:106DF00060E070E080E89FE30E9464E220E03AE215
:106E00004DE257E40E942AE16B017C01C301B2010B
:106E10000E94CBE020E030E048EC52E40E9443E3E3
:106E2000AB01BC0122E0CE0101960E94A7C8BE01C1
:106E30006F5F7F4F82E994E10E945AC8CE010196AC
:106E40000E949FC866EC79E082E994E10E940DC837
:106E500062E974E188E994E10E9443C862EC79E058
:106E6000CE0101960E940BC962E974E1CE01019640
:106E70000E947CC7BC0182E994E10E9443C8CE0114
:106E800001960E949FC86DEB76E08EE994E10E9426
:106E9000E2C521E0B501A401CE0101960E94A7C878
:106EA000BE016F5F7F4F8EE994E10E9417C8CE014B
:106EB00001960E949FC868EE76E08EE994E10E94F8
:106EC0000DC821E0B701A601CE0101960E94A7C816
:106ED000BE016F5F7F4FCE0107960E9402C96BE42F
:106EE00078E0CE0107960E9466C7BC018EE994E166
:106EF0000E9417C8CE0107960E949FC8CE01019636
:106F00000E949FC862E974E1CE0101960E9402C905
:106F10006EE277E0CE0101960E9466C76EE974E1E9
:106F20000E947CC7BC018EE994E10E9443C8CE0157
:106F300001960E949FC821E0B501A401CE010196EF
:106F40000E94A7C8BE016F5F7F4F84EA94E10E9450
:106F50005AC8CE0101960E949FC864EA74E1CE012E
:106F600001960E9402C94AE050E070E060E0CE0164
:106F700001960E94FD19CE0101960E949FC865E00E
:106F800070E080E090E00E94086E65E079E0CE015C
:106F900001960E940BC9CE0101960E940310CE01FA
:106FA00001960E949FC868E974E1CE0101960E9493
:106FB00002C94AE050E06FEF7FEFCE0101960E94D8
:106FC0006313CE0101960E949FC820E0B701A6017D
:106FD000CE0101960E94A7C8BE016F5F7F4FCE0110
:106FE00007960E9402C96BE478E0CE0107960E94E2
:106FF00066C7BC0184EA94E10E9443C8CE010796AB
:107000000E949FC8CE0101960E949FC864EA74E165
:10701000CE0101960E9402C94AE050E064EF7FEF82
:10702000CE0101960E946313CE0101960E949FC873
:1070300065E070E080E090E00E94086E80917D0E37
:10704000882331F068E572E080E090E00E94086EED
:107050002C960FB6F894DEBF0FBECDBFDF91CF9157
:10706000FF90EF90DF90CF90BF90AF909F908F9068
:107070007F906F905F904F900895CF92DF92EF9244
:10708000FF920F931F93CF93DF93CDB7DEB7E097B7
:107090000FB6F894DEBF0FBECDBF8E01015E1F4F4D
:1070A0008130910509F0B7C06EEE76E0CE01019611
:1070B0000E940BC961EF76E0CE0107960E940BC9D2
:1070C00064EF76E0CE010D960E940BC963EF71E18B
:1070D000C8010E94F9C844E650E06FEF7FEFC80195
:1070E0000E94FD19C8010E949FC868EE71E18CEBF7
:1070F00094E10E941EC86091F0047091F104CE01E9
:1071000085960E9419C66CEB74E1C8010E9402C901
:10711000BE016B5D7F4FC8010E947CC7BC01CE01E0
:107120008B960E9402C940ED57E06FEF7FEFCE01D2
:107130008B960E946313CE018B960E949FC8C80154
:107140000E949FC8CE0185960E949FC869ED71E19B
:10715000C8010E94F9C844E650E06FEF7FEFC80114
:107160000E94FD19C8010E949FC867EF76E0C80120
:107170000E940BC923E030E0A801BE016F5F7F4F82
:10718000CE0185960E9435CABE016B5D7F4F8CEBA8
:1071900094E10E945AC8CE0185960E949FC8C801FA
:1071A0000E949FC88091C0149091C114892B09F44A
:1071B000E3C270E060E08CEB94E10E943AC7082ED5
:1071C000000C990BC0970A9708F0D6C28CEB94E19B
:1071D0000E945FC66B016BEF76E0C8010E940BC98D
:1071E00086E08C9DB0018D9D700D112481E090E0B2
:1071F0008C0F9D1F680F791FC8010E947CC7BC01BE
:107200008CEB94E10E9443C8C8010E949FC80E9471
:107210005195182FE2C08A3F2FEF920709F023C142
:1072200060E077E0CE0101960E940BC96AE077E04A
:10723000CE0107960E940BC962E177E0CE010D9660
:107240000E940BC96AE177E0CE0143960E940BC908
:107250006AEC71E1C8010E94F9C844E650E06FEFA2
:107260007FEFC8010E94FD19C8010E949FC864EC0D
:1072700071E18CEB94E10E941EC880911D13EE24F5
:10728000E394F12CEC0EFD1E96E08902E00CF11C5B
:1072900011246CEB74E1C8010E9402C9B701C80156
:1072A0000E947CC7BC01CE0185960E9402C940EDB8
:1072B00057E06FEF7FEFCE0185960E946313CE01FA
:1072C00085960E949FC8C8010E949FC864EB71E127
:1072D000C8010E94F9C844E650E06FEF7FEFC80193
:1072E0000E94FD19C8010E949FC860E277E0C801B2
:1072F0000E940BC924E030E0A801BE016F5F7F4F00
:10730000CE0185960E9435CABE016B5D7F4F8CEB26
:1073100094E10E945AC8CE0185960E949FC8C80178
:107320000E949FC88091C0149091C114892B09F4C8
:1073300098C070E060E08CEB94E10E943AC7082EA0
:10734000000C990BC0970A9708F08BC08CEB94E166
:107350000E945FC662307105810591050CF46EC014
:1073600068EA71E1C8010E94F9C844E650E06FEF95
:107370007FEFC8010E946313C8010E949FC844EFB9
:1073800051E063E070E0CE0185960E9462C966E23A
:1073900077E0C8010E940BC96CEB74E1C8010E9440
:1073A0007CC76DE277E00E9466C7BE016B5D7F4FD0
:1073B0000E947CC7BC018CEB94E10E9443C8C801C9
:1073C0000E949FC8CE0185960E949FC80E94519539
:1073D000182FCE0143960E949FC8CE010D960E94A1
:1073E0009FC8CE0107960E949FC8CE0101960E94B9
:1073F0009FC862E271E1111102C063E171E1CE0147
:1074000001960E94F9C848EC50E06FEF7FEFCE0183
:1074100001960E946313CE0101960E949FC8E096D8
:107420000FB6F894DEBF0FBECDBFDF91CF911F9195
:107430000F91FF90EF90DF90CF90089566E277E094
:10744000C8010E940BC96CEB74E1C8010E947CC7A3
:10745000BC018CEB94E10E9443C8C8010E949FC804
:10746000B5CF10E0B6CF0F9609F0ECC0CE01019673
:107470007C0161E47CE0C7010E940BC996E0E90E43
:10748000F11C0E151F05A9F760E377E0CE01019608
:107490000E94E2C580912013811130C020912113F8
:1074A00030912213409123135091241360E070E037
:1074B00080EA90E40E9443E3AB01BC0122E0CE01EC
:1074C00085960E94A7C866E377E0C8010E940BC9B1
:1074D000BE016B5D7F4FC8010E947CC76DEE77E0F7
:1074E0000E9466C7BC01CE0101960E9417C8C80160
:1074F0000E949FC8CE0185960E949FC86DE971E1E8
:10750000CE0107960E941EC861E971E1CE010D9679
:107510000E941EC865E871E1CE0143960E941EC814
:1075200069E771E1CE0149960E941EC863E771E1E7
:10753000C8010E941EC864E671E1C8010E94F9C832
:1075400044E650E06FEF7FEFC8010E94FD19C801CB
:107550000E949FC861E47CE08CEB94E10E94E2C54C
:107560008091201361E070E06C0F7D1F26E08202A5
:10757000600D711D1124C8010E9402C940ED57E041
:107580006FEF7FEFC8010E946313C8010E949FC87C
:1075900065E571E1C8010E94F9C844E650E06FEF6B
:1075A0007FEFC8010E94FD19C8010E949FC86CEBC3
:1075B00074E1C8010E9402C925E030E0A801BE01C3
:1075C0006F5F7F4FCE0185960E9435CABE016B5D0D
:1075D0007F4F8CEB94E10E945AC8CE0185960E94A1
:1075E0009FC8C8010E949FC88091C0149091C11487
:1075F000892B31F170E060E08CEB94E10E943AC796
:10760000082E000C990BC0970A97D0F469E377E035
:10761000C8010E940BC96CEB74E1C8010E947CC7D1
:10762000BC018CEB94E10E9443C8C8010E949FC832
:107630000E945195182FCE0149960E949FC8C9CE2D
:1076400010E0F9CF60E477E0CE0101960E940BC90B
:1076500063E477E0CE0107960E940BC968E477E007
:10766000CE010D960E940BC965E471E1C8010E942C
:10767000F9C844E650E06FEF7FEFC8010E94FD19A2
:10768000C8010E949FC86FE371E18CEB94E10E94F6
:107690001EC8809167139091681326E0289F70019F
:1076A000299FF00C112481E090E08C0F9D1FE80EC3
:1076B000F91E6CEB74E1C8010E9402C9B701C80150
:1076C0000E947CC7BC01CE0185960E9402C940ED94
:1076D00057E06FEF7FEFCE0185960E946313CE01D6
:1076E00085960E949FC8C8010E949FC86FE271E101
:1076F000C8010E94F9C844E650E06FEF7FEFC8016F
:107700000E94FD19C8010E949FC86CEB74E1C8017A
:107710000E9402C923E030E0A801BE016F5F7F4FE5
:10772000CE0185960E9435CABE016B5D7F4F8CEB02
:1077300094E10E945AC8CE0185960E949FC8C80154
:107740000E949FC88091C0149091C114892BA1F010
:1077500070E060E08CEB94E10E943AC7082E000CC8
:10776000990BC0970A9740F48CEB94E10E945FC696
:10777000CB010E94311E4DCD10E02FCE3F924F9293
:107780005F926F927F928F929F92AF92BF92CF92B1
:10779000DF92EF92FF920F931F93CF93DF93CDB7BA
:1077A000DEB7CA56D1090FB6F894DEBF0FBECDBF03
:1077B00069AF7AAF8BAF9CAF29962CAF3DAF4EAF80
:1077C0005FAF299761E47CE0CE01C1960E940BC9AE
:1077D000C9ACDAACEBACFCAC28EEC21623E0D206A6
:1077E000E104F10454F030E9C32EDD24D394E12CFC
:1077F000F12CC9AEDAAEEBAEFCAE2996CCACDDAC6A
:10780000EEACFFAC299720E1C21627E2D206E104D4
:10781000F10464F020E1C22E27E2D22EE12CF12CFB
:107820002996CCAEDDAEEEAEFFAE299780917D0EEF
:10783000882351F0C12CD12C7601C3942996CCAE6B
:10784000DDAEEEAEFFAE29970E943B6EA1966CAF07
:107850007DAF8EAF9FAFA1970E943B6E65966CAFD8
:107860007DAF8EAF9FAF6597A1966CAD7DAD8EADB0
:107870009FADA19728EE33E040E050E00E9401E286
:10788000AB962CAF3DAF4EAF5FAFAB97312C21968F
:107890001CAE1DAE1EAE1FAE21978E01075E1F4FA0
:1078A0009E01235F3F4F38AF2FABC9ACDAACEBACD6
:1078B000FCACF094E094D094C094C11CD11CE11CA9
:1078C000F11C6196CCAEDDAEEEAEFFAE6197659673
:1078D0006CAD7DAD8EAD9FAD6597A196CCACDDACAA
:1078E000EEACFFACA1976C197D098E099F09299612
:1078F000CCACDDACEEACFFAC29976C157D058E05EC
:107900009F050CF099C70E94CBE020E030E04AE7E9
:1079100054E40E9443E3AB01BC0123E0C8010E9490
:10792000A7C8B80188E994E10E945AC8C8010E941A
:107930009FC8A70196012A303105410551058CF4F5
:10794000AB964CAD5DAD6EAD7FADAB97C8010E94FF
:10795000ECC5B80188E994E10E945AC8C8010E94A8
:107960009FC880917D0E69EB77E0882309F4EDC212
:1079700088E994E10E94E2C580911C0E90911D0E51
:10798000039709F453C0CE0101960E9485C261E4B9
:107990007CE08EE994E10E94E2C5AE014F5F5F4F4B
:1079A0005A01C12CD12C7601D5014D905D906D907E
:1079B0007D905D01A3019201C301B2010E942AE101
:1079C0009B01AC01C701B6010E9465E26B017C011D
:1079D00023E0B301A201C8010E94A7C8B801CE01EB
:1079E0004F960E9402C96EE277E0CE014F960E9448
:1079F00066C7BC018EE994E10E9417C8CE014F967C
:107A00000E949FC8C8010E949FC8EFA9F8ADAE169A
:107A1000BF0651F6C701B6010E946DE52D966CAF09
:107A20007DAF8EAF9FAF2D97332433948091E10CBF
:107A3000882309F410C280911C0E90911D0E0397AB
:107A4000039708F008C289E60E94CDAD68EA70E0AD
:107A500089ED94E10E94EF1389ED94E10E94917405
:107A600046E050E069E670E089ED94E10E94DD7443
:107A70008091080F9091090F891B990B8630910511
:107A8000ECF30E94C7B1B82E0E94C7B1A82E0E9485
:107A9000C7B1D82E0E94C7B1C82E0E94C7B1F82E18
:107AA0000E94C7B1E82EA396AFAEA397A2961FAED1
:107AB000A297A3966EAD7FADA3976B29072E000CFE
:107AC000880B990B0E94CBE02B013C014092830E66
:107AD0005092840E6092850E7092860EA596CFAE5F
:107AE000A597A4961FAEA497A5966EAD7FADA5975A
:107AF0006D29072E000C880B990B0E94CBE04B01DF
:107B00005C018092870E9092880EA092890EB092AE
:107B10008A0EA796EFAEA797A6961FAEA697A79632
:107B20006EAD7FADA7976F29072E000C880B990BC0
:107B30000E94CBE025966CAF7DAF8EAF9FAF2597AF
:107B400060938B0E70938C0E80938D0E90938E0E9F
:107B50008091B30EC090B80ED090B90EE090BA0EDE
:107B6000F090BB0E882309F405C220919B0E309142
:107B70009C0E40919D0E50919E0EC301B2010E9439
:107B800064E2A70196010E942AE160938F0E709330
:107B9000900E8093910E9093920E20919F0E3091B3
:107BA000A00E4091A10E5091A20EC501B4010E94F9
:107BB00064E2A70196010E942AE16093930E7093FC
:107BC000940E8093950E9093960E2091A30E309173
:107BD000A40E4091A50E5091A60E25966CAD7DADDC
:107BE0008EAD9FAD25970E9464E2A70196010E9489
:107BF0002AE16093970E7093980E8093990E90935C
:107C00009A0E20E030E0A9016091B40E7091B50E9B
:107C10008091B60E9091B70E0E944CE418160CF0AD
:107C200081C0C0908F0ED090900EE090910EF09099
:107C3000920E20E030E0A901C701B6010E944CE499
:107C4000181624F0F7FAF094F7F8F094A7019601CB
:107C50006091A70E7091A80E8091A90E9091AA0E26
:107C60000E944CE4181644F410928F0E1092900E5D
:107C70001092910E1092920EC090930ED090940E8E
:107C8000E090950EF090960E20E030E0A901C7013B
:107C9000B6010E944CE4181624F0F7FAF094F7F8B5
:107CA000F094A70196016091AB0E7091AC0E80919B
:107CB000AD0E9091AE0E0E944CE4181644F4109252
:107CC000930E1092940E1092950E1092960EC090F4
:107CD000970ED090980EE090990EF0909A0E20E0BA
:107CE00030E0A901C701B6010E944CE4181624F047
:107CF000F7FAF094F7F8F094A70196016091AF0EAF
:107D00007091B00E8091B10E9091B20E0E944CE431
:107D1000181644F41092970E1092980E1092990E25
:107D200010929A0E4091930E5091940E6091950E80
:107D30007091960E8091970E9091980EA091990E49
:107D4000B0919A0EC0908F0ED090900EE090910E50
:107D5000F090920ECD86DE86EF86F88A498B5A8B9C
:107D60006B8B7C8B8D8B9E8BAF8BB88F61E47CE0B3
:107D7000CE01C1960E94E2C55E01FDE0AF0EB11CCE
:107D8000C12CD12C7601D5014D905D906D907D90E8
:107D90005D01A3019201C301B2010E942AE19B018E
:107DA000AC01C701B6010E9465E26B017C0120E0D5
:107DB000B301A201C8010E94A7C8B801CE014F9625
:107DC0000E9402C96EE277E0CE014F960E9466C71C
:107DD000BC01CE01C1960E9417C8CE014F960E94E9
:107DE0009FC8C8010E949FC8A016B10661F6C701CE
:107DF000B6010E946DE525966CAF7DAF8EAF9FAF4B
:107E0000259721E0AB01BC01CE014F960E94A7C887
:107E100060EE7BE0C8010E940BC968E974E1C8010B
:107E20000E947CC76CE477E00E9466C7BE01615E79
:107E30007F4F0E947CC760E577E00E9466C7BC0167
:107E4000CE01C1960E9417C8C8010E949FC8CE01EA
:107E50004F960E949FC8C9ACDAACEBACFCAC2DE2EB
:107E6000C21621E0D206E104F10434F00E943F136F
:107E700060E080E00E94E8AD80911C0E90911D0EA4
:107E8000039709F449C223E02D964CAD5DAD6EAD6C
:107E90007FAD2D97CE014F960E94A7C860EE7BE084
:107EA000C8010E940BC968E974E1C8010E947CC73F
:107EB00067E577E00E9466C7BE01615E7F4F0E9462
:107EC0007CC76BE577E00E9466C7BC018EE994E150
:107ED0000E9417C8C8010E949FC8CE014F960E94F9
:107EE0009FC82AE939E949E55FE32D966CAD7DAD80
:107EF0008EAD9FAD2D970E944CE418160CF05FC01C
:107F000023E333E343E95FE32D966CAD7DAD8EADA6
:107F10009FAD2D970E94C4E0880F880B3822809176
:107F20001C0E90911D0E181619060CF04AC08230D6
:107F3000910509F449C0853091050CF045C08330A6
:107F4000910509F078C3312CE7C1C8010E940BC923
:107F500068E974E1C8010E947CC765E87BE00E9483
:107F600066C7BC0188E994E10E9443C8C8010E9429
:107F70009FC802CDA3019201C701B6010E942AE168
:107F800060938F0E7093900E8093910E9093920E4B
:107F9000A5019401C701B6010E942AE16093930EE6
:107FA0007093940E8093950E9093960E25962CAD1B
:107FB0003DAD4EAD5FAD2597C701B60118CE312C52
:107FC000AECF332009F43AC389849A84AB84BC844D
:107FD00049805A806B807C80CD80DE80EF80F88481
:107FE00020E030E0A901C501B4010E94C4E088236B
:107FF00009F40EC3A3019201C301B2010E942AE158
:1080000069966CAF7DAF8EAF9FAF6997A701960160
:10801000C701B6010E942AE19B01AC0169966CADD3
:108020007DAD8EAD9FAD69970E9465E20E946DE5C2
:10803000A50194010E94E4E220EE3EE245E652E40E
:108040000E942AE169966CAF7DAF8EAF9FAF6997B2
:1080500020E030E0A901C701B6010E94C4E08823F6
:1080600009F4DBC2A3019201C301B2010E942AE11B
:108070006D966CAF7DAF8EAF9FAF6D97A5019401EC
:10808000C501B4010E942AE19B01AC016D966CAD63
:108090007DAD8EAD9FAD6D970E9465E20E946DE54E
:1080A000A70196010E94E4E220EE3EE245E652E49A
:1080B0000E942AE16D966CAF7DAF8EAF9FAF6D973A
:1080C00020E030E0A901C301B2010E94C4E088238E
:1080D00009F4A8C2A5019401C501B4010E942AE1D6
:1080E0004B015C01A7019601C701B6010E942AE17C
:1080F0009B01AC01C501B4010E9465E20E946DE5DF
:10810000A30192010E94E4E26B017C0168E974E141
:10811000C8010E9402C969E873E1C8010E947CC7D6
:10812000BC018EE994E10E9443C8C8010E949FC827
:108130006EE974E1C8010E9402C9C8010E942813B7
:10814000C8010E949FC821E069964CAD5DAD6EAD3F
:108150007FAD6997CE018B960E94A7C821E06D96EE
:108160004CAD5DAD6EAD7FAD6D97CE0185960E9435
:10817000A7C820EE3EE245E652E4C701B6010E94E0
:108180002AE1AB01BC0121E0C8010E94A7C8B801E7
:10819000CE014F960E9402C96EE277E0CE014F9663
:1081A0000E9466C7BE016B5D7F4F0E947CC76EE276
:1081B00077E00E9466C7BE01655D7F4F0E947CC765
:1081C000BC018EE994E10E9443C8CE014F960E9403
:1081D0009FC8C8010E949FC8CE0185960E949FC873
:1081E000CE018B960E949FC86EE577E0C8010E9481
:1081F0000BC96EE974E1C8010E947CC7BC0182E929
:1082000094E10E9443C8C8010E949FC862E974E1DA
:10821000C8010E9402C9C8010E944818C8010E94F2
:108220009FC86EE974E182E994E10E9443C86EE957
:1082300074E1C8010E9402C9C8010E940B13C80161
:108240000E949FC8C9ACDAACEBACFCAC2DE2C21604
:1082500021E0D206E104F10484F421966CAD7DADF9
:108260008EAD9FAD219725E030E040E050E00E94C8
:1082700001E2672B682B692BA9F56DEF7DE088E99A
:1082800094E10E941EC862E677E0C8010E940BC913
:1082900045E050E067EF7FEFC8010E94FD19C8017B
:1082A0000E949FC861E47CE0C8010E940BC9C8011C
:1082B0000E940310C8010E949FC86EE974E1C801C2
:1082C0000E9402C945E050E070E060E0C8010E94F1
:1082D0006313C8010E949FC861E47CE08EE994E1C9
:1082E0000E94E2C569AD7AAD8BAD9CADC9ACDAAC8C
:1082F000EBACFCACF7FE0CC02E966FAD2E972F9614
:108300007FAD2F9760968FAD609761969FAD619717
:108310000E94086E332433948091E10C882309F481
:10832000FEC080911C0E90911D0E0397039708F0DC
:10833000F6C06FE777E0C8010E940BC9BE016F5C11
:108340007F4FC8010E947CC7BC01CE01C1960E942C
:1083500043C8C8010E949FC8BE016F5C7F4FC8011F
:108360000E9402C9C8010E940B13C8010E949FC845
:10837000BE016F5C7F4FC8010E9402C9C8010E9404
:108380004818C8010E949FC821E025964CAD5DADFC
:108390006EAD7FAD2597CE014F960E94A7C86DE4C4
:1083A00077E0C8010E940BC9BE01615E7F4FC80122
:1083B0000E947CC760E577E00E9466C7BC01CE01E1
:1083C000C1960E9443C8C8010E949FC8CE014F9623
:1083D0000E949FC8BE016F5C7F4FC8010E9402C906
:1083E000C8010E944818C8010E949FC868E974E14A
:1083F000C8010E9402C9BE016F5C7F4FC8010E9484
:108400007CC7BC01CE01C1960E9443C8C8010E942E
:108410009FC861E977E088E994E10E940DC84D8921
:108420005E896F89788D20E0CE018B960E94A7C867
:1084300049895A896B897C8920E0CE0185960E9402
:10844000A7C84D855E856F85788920E0C8010E94A8
:10845000A7C8B801CE014F960E9402C96EE277E02C
:10846000CE014F960E9466C7BE016B5D7F4F0E9492
:108470007CC76EE277E00E9466C7BE01655D7F4FF4
:108480000E947CC7BC0182E994E10E9443C8CE01EE
:108490004F960E949FC8C8010E949FC8CE01859632
:1084A0000E949FC8CE018B960E949FC8C9ACDAACCF
:1084B000EBACFCAC2DE2C21621E0D206E104F104E3
:1084C00084F421966CAD7DAD8EAD9FAD219725E0F6
:1084D00030E040E050E00E9401E2672B682B692BFE
:1084E000F1F468E974E1C8010E9402C945E050E076
:1084F0006FEF7FEFC8010E94FD19C8010E949FC85D
:1085000062E974E1C8010E9402C945E050E070E0F0
:1085100060E0C8010E946313C8010E949FC8809157
:108520007D0E68E974E1882309F47BC1C8010E94CB
:1085300002C94AE050E067E070E0C8010E944419B7
:10854000C8010E949FC83320D1F065EF7DE0C801CB
:108550000E94F9C845E050E070E060E0C8010E9468
:10856000FD19C8010E949FC861E47CE0C8010E9417
:108570000BC9C8010E940310C8010E949FC88091C6
:108580001C0E90911D0E039779F062E974E1C80109
:108590000E9402C94AE050E06FEF7FEFC8010E94DD
:1085A0006313C8010E949FC80E943B6E6B017C014F
:1085B00065962CAD3DAD4EAD5FAD6597C21AD30A41
:1085C000E40AF50A2196CCAEDDAEEEAEFFAE219701
:1085D00089AD9AADABADBCADC816D906EA06FB06AF
:1085E00044F4BC01CD016C197D098E099F090E94DC
:1085F000086E0E943B6E65966CAF7DAF8EAF9FAFED
:10860000659761E47CE08EE994E10E94E2C55FC970
:108610006BED7FE089EC9FE30FCD6BED7FE089ECA4
:108620009FE342CD8BEDC82E8FE0D82E89ECE82E4B
:108630008FE3F82E6BCD059709F485CC69E677E0DA
:10864000C8010E940BC96EE974E1C8010E947CC791
:10865000BC018EE994E10E9443C8C8010E949FC8F2
:108660006EE974E1C8010E9402C9C8010E940B139F
:10867000C8010E949FC86EE974E1C8010E9402C946
:10868000C8010E944818C8010E949FC823E02D9687
:108690004CAD5DAD6EAD7FAD2D97CE014F960E9476
:1086A000A7C868E577E0C8010E940BC9BE01615EFA
:1086B0007F4FC8010E947CC76BE577E00E9466C7C8
:1086C000BC018EE994E10E9443C8C8010E949FC882
:1086D000CE014F960E949FC86EE974E1C8010E94C6
:1086E00002C9C8010E944818C8010E949FC868E9D1
:1086F00074E1C8010E9402C96EE974E1C8010E94D8
:108700007CC7BC018EE994E10E9443C8C8010E9465
:108710009FC866E777E088E994E10E940DC8498523
:108720005A856B857C8522E0CE018B960E94A7C876
:108730004D815E816F81788522E0CE0185960E9411
:10874000A7C849815A816B817C8122E0C8010E94BF
:10875000A7C8B801CE014F960E9402C96EE277E029
:10876000CE014F960E9466C7BE016B5D7F4F0E948F
:108770007CC76EE277E00E9466C7BE01655D7F4FF1
:108780000E947CC7BC0182E994E10E9443C8CE01EB
:108790004F960E949FC8C8010E949FC8CE0185962F
:1087A0000E949FC8CE018B960E949FC8C9ACDAACCC
:1087B000EBACFCAC2DE2C21621E0D206E104F104E0
:1087C0008CF421966CAD7DAD8EAD9FAD219725E0EB
:1087D00030E040E050E00E9401E2672B682B692BFB
:1087E00009F0B1CB68E974E1C8010E9402C945E013
:1087F00050E06FEF7FEFC8010E94FD19C8010E9491
:108800009FC862E974E1C8010E9402C945E050E0D6
:1088100070E060E0C8010E946313C8010E949FC815
:1088200092CBC8010E9402C94AE050E06FEF7FEF8F
:10883000C8010E94FD1984CECE01C1960E949FC836
:10884000C659DF4F0FB6F894DEBF0FBECDBFDF9124
:10885000CF911F910F91FF90EF90DF90CF90BF903D
:10886000AF909F908F907F906F905F904F903F90D0
:1088700008954F925F926F927F928F929F92AF92E4
:10888000BF92CF92DF92EF92FF920F931F93CF93FD
:10889000DF93CDB7DEB7A8970FB6F894DEBF0FBE53
:1088A000CDBF20918713309188132F3F3F4F09F49C
:1088B00063C38C0161E47CE0CE0149960E940BC940
:1088C00061E47CE0CE014F960E940BC98091871332
:1088D000909188138130910509F065C30E94FDBC19
:1088E00065E070E080E090E00E94086E80900C15DA
:1088F00090900D15A0900E15B0900F15C09010150A
:10890000D0901115E0901215F09013158091141568
:1089100090911515A0911615B09117158DA39EA3D2
:10892000AFA3B8A722E0AC01BD01CE0143960E94DF
:10893000A7C822E0B701A601CE010D960E94A7C8E4
:1089400022E0B501A401CE0101960E94A7C8BE0194
:108950006F5F7F4FCE0107960E9402C96EE277E0FB
:10896000CE0107960E9466C7BE01635F7F4F0E94DB
:108970007CC76EE277E00E9466C7BE016D5E7F4FE6
:108980000E947CC76EE277E00E9466C7BC018EE958
:1089900094E10E9443C8CE0107960E949FC8CE0171
:1089A00001960E949FC8CE010D960E949FC8CE01DD
:1089B00043960E949FC86EE974E1CE0101960E9421
:1089C00002C9CE0101960E940B13CE0101960E94AE
:1089D0009FC8A7019601C501B40190580E94E4E226
:1089E0002BED3FE049EC5FE30E9465E22091E70454
:1089F0003091E8044091E9045091EA040E9465E254
:108A00002B013C0120E030E0A9010E94C4E087FD79
:108A10005EC34092980C5092990C60929A0C70929E
:108A20009B0C4090980C5090990C60909A0C709010
:108A30009B0C2BED3FE049EC50E4C301B2010E94D6
:108A40004CE4181684F42BED3FE049EC50E4C301EC
:108A5000B2010E9464E26093980C7093990C809329
:108A60009A0C90939B0C20E030E044E353E4609137
:108A7000980C7091990C80919A0C90919B0C0E948B
:108A80002AE12BED3FE049E450E40E9443E3609388
:108A9000940C7093950C8093960C9093970C0E9475
:108AA000EFE3CE0107960E9419C669E977E0CE018F
:108AB00001960E940BC9BE01695F7F4FCE010196EE
:108AC0000E947CC763EA77E00E9466C7BC0184EA23
:108AD00094E10E9443C8CE0101960E949FC8CE0136
:108AE00007960E949FC84090940C5090950C6090FF
:108AF000960C7090970C20E030E044EB52E4C301F8
:108B0000B2010E94C4E018160CF4F2C220E030E07A
:108B100040E05FE3C301B2010E9465E20E94EFE31F
:108B2000CE0107960E9419C66AEA77E0CE01019647
:108B30000E940BC9BE01695F7F4FCE0101960E9462
:108B40007CC7BC01CE0149960E9443C8CE01019664
:108B50000E949FC8CE0107960E949FC86FE079E0EF
:108B6000CE014F960E94E2C5BE01675E7F4FCE01E7
:108B700001960E9402C94AE050E070E060E0CE0138
:108B800001960E94FD19CE0101960E949FC80E9485
:108B90003B6EAB01BC0180919C0C90919D0CA0910F
:108BA0009E0CB0919F0C8C599F4FAF4FBF4F8417B5
:108BB0009507A607B70708F020C361E47CE0CE0163
:108BC00001960E940BC9CE0101960E940310CE01AE
:108BD00001960E949FC8BE01615E7F4F86E296E1CA
:108BE0000E949AD16EE277E0CE0101960E940BC9F5
:108BF000BE01615E7F4FCE0101960E947CC7BC0121
:108C0000CE0149960E9417C8CE0101960E949FC8C6
:108C10000E943B6E4090A80C5090A90C6090AA0C4A
:108C20007090AB0C64197509860997090E94C9E018
:108C300020E030E04AE754E40E9443E3AB01BC018A
:108C400023E0CE0107960E94A7C869EB77E0CE012A
:108C500001960E940BC9BE01695F7F4FCE0101964C
:108C60000E947CC765E87BE00E9466C7BC0182E980
:108C700094E10E9443C8CE0101960E949FC8CE0194
:108C800007960E949FC862E974E1CE0101960E9496
:108C900002C964EA74E1CE0101960E947CC7BE015C
:108CA000675E7F4F0E947CC7BC01CE0149960E943F
:108CB00043C8CE0101960E949FC86EE874E08EE919
:108CC00094E10E941EC821E0B501A401CE010196E5
:108CD0000E94A7C8BE016F5F7F4F8EE994E10E949A
:108CE00017C8CE0101960E949FC821E04DA15EA148
:108CF0006FA178A5CE010D960E94A7C821E0B7010B
:108D0000A601CE0107960E94A7C86EE277E0CE01C9
:108D100001960E940BC9BE01695F7F4FCE0101968B
:108D20000E947CC76EE277E00E9466C7BE01635F67
:108D30007F4F0E947CC760EB77E00E9466C7BC0152
:108D40008EE994E10E9417C8CE0101960E949FC847
:108D5000CE0107960E949FC8CE010D960E949FC823
:108D6000A5019401C501B4010E942AE14B015C01F7
:108D7000A7019601C701B6010E942AE19B01AC013F
:108D8000C501B4010E9465E26B017C012DA13EA1E9
:108D90004FA158A5CA01B9010E942AE19B01AC016B
:108DA000C701B6010E9465E20E946DE56093900CD8
:108DB0007093910C8093920C9093930C64EB77E0FA
:108DC0008EE994E10E940DC84091900C5091910C55
:108DD0006091920C7091930C21E0CE0101960E945B
:108DE000A7C8BE016F5F7F4FCE0107960E9402C9E0
:108DF00062E77CE0CE0107960E9466C7BC0184EA68
:108E000094E10E9443C8CE0107960E949FC8CE01FC
:108E100001960E949FC864EA74E18EE994E10E9481
:108E200017C8C090900CD090910CE090920CF090EC
:108E3000930C20E030E04AE754E4C701B6010E94F9
:108E40004CE487FD29C020E030E04AE754E4C70144
:108E5000B6010E9443E3AB01BC0123E0CE010196C1
:108E60000E94A7C8BE016F5F7F4FCE0107960E9488
:108E700002C963E77CE0CE0107960E9466C7BC0189
:108E800084EA94E10E9443C8CE0107960E949FC8DD
:108E9000CE0101960E949FC820E030E64AE656E4E3
:108EA0006091900C7091910C8091920C9091930C28
:108EB0000E94C4E0BE01675E7F4F87FFBDC1CE0147
:108EC00001960E9402C968EB77E0CE0101960E94EC
:108ED00066C76EE974E10E947CC7BC018EE994E12B
:108EE0000E9443C8CE0101960E949FC8033011051D
:108EF000A1F46EE974E1CE0101960E9402C9CE018F
:108F000001960E940B13CE0101960E949FC861E456
:108F10007CE08EE994E10E94E2C56BEB77E0CE0144
:108F200001960E940BC964EA74E1CE0101960E9489
:108F30007CC7BC01CE0107960E9402C94AE050E0FE
:108F40006FEF7FEFCE0107960E946313CE01079665
:108F50000E949FC8CE0101960E949FC86AE070E0FF
:108F600080E090E00E94086ECE014F960E949FC85C
:108F7000CE0149960E949FC8A8960FB6F894DEBF0E
:108F80000FBECDBFDF91CF911F910F91FF90EF905A
:108F9000DF90CF90BF90AF909F908F907F906F9019
:108FA0005F904F900895892B09F013CD0E94E674CD
:108FB00040900D0550900E0560900F0570901005C3
:108FC0006091E40E7091E50E072E000C880B990B52
:108FD0000E94CBE0A30192010E942AE120910905A1
:108FE00030910A0540910B0550910C050E942AE131
:108FF0002091D00E3091D10E4091D20E5091D30ECF
:109000000E9465E24B015C018092DC0E9092DD0EC5
:10901000A092DE0EB092DF0E6091E20E7091E30E30
:10902000072E000C880B990B0E94CBE0A301920144
:109030000E942AE12091050530910605409107051F
:10904000509108050E942AE12091CC0E3091CD0E5E
:109050004091CE0E5091CF0E0E9465E26B017C01D3
:10906000C092D80ED092D90EE092DA0EF092DB0EBA
:109070006091E00E7091E10E072E000C880B990BA9
:109080000E94CBE0A30192010E942AE120910105F8
:109090003091020540910305509104050E942AE198
:1090A0002091C80E3091C90E4091CA0E5091CB0E3E
:1090B0000E9465E26DA37EA38FA398A76093D40E50
:1090C0007093D50E8093D60E9093D70E82CC2BED55
:1090D0003FE049EC50E4C301B2010E9465E26093B5
:1090E000980C7093990C80939A0C90939B0C99CC4C
:1090F00020E030E044E353E4C301B2010E94C4E045
:109100001816CCF0A301920160E070E884E393E4C8
:109110000E9464E26093940C7093950C8093960C7B
:109120009093970C0E94EFE3CE0107960E9419C618
:109130006DEA77E0FBCC20E030E047E853E4C30180
:10914000B2010E94C4E01816CCF120E030E044E304
:1091500053E4C301B2010E9464E220E030E040E049
:109160005FE30E9465E26093940C7093950C80938A
:10917000960C9093970C0E94EFE3CE0107960E9405
:1091800019C66DEA77E0CE0101960E940BC9BE01B7
:10919000695F7F4FCE0101960E947CC7BC01CE0162
:1091A00049960E9443C8CE0101960E949FC8CE01F5
:1091B00007960E949FC867E178E0D2CCA301920194
:1091C00060E070E084EB93E40E9464E220E030E031
:1091D00040E05FE30E9465E26093940C7093950C0D
:1091E0008093960C9093970C0E94EFE3CE01079624
:1091F0000E9419C66AEA77E0C6CF0E943B6E0E94C1
:10920000C9E02B013C0160919C0C70919D0C8091F8
:109210009E0C90919F0C0E94CBE020E030E048EC47
:1092200051E40E9465E29B01AC01C301B2010E94BE
:10923000C4E087FDC2CCD6CC8EE994E10E9443C83D
:109240008DCEDF92EF92FF920F931F93CF93DF9318
:10925000CDB7DEB72C970FB6F894DEBF0FBECDBFEB
:109260008C0110929C0D61E47CE0CE0107960E9477
:109270000BC9F12CE12CDD24D3948BEA9FE00E94F2
:10928000D5AA1816190694F480919C0D81110EC070
:109290008BEA9FE00E94B3AA8A30D1F58B859C852A
:1092A000892B09F443C0D0929C0D40C062E370E06A
:1092B00080E090E00E94086EEF2851F08BEA9FE07A
:1092C0000E94BDAC64E670E080E090E00E94086E11
:1092D00080919C0D811131C08B859C85892B69F50E
:1092E00061E47CE0C8010E940BC9CE0107960E9490
:1092F0009FC8C8012C960FB6F894DEBF0FBECDBF35
:10930000DF91CF911F910F91FF90EF90DF90089523
:109310008D3021F290919C0D9111C0CF682FCE011C
:1093200007960E94EAC78FEFE81AF80A6FE070E02C
:1093300080E090E00E94086EA0CF80917E0E88238E
:1093400079F0BE01695F7F4FCE0101960E9402C98C
:10935000CE0101960E940B13CE0101960E949FC878
:10936000BE01695F7F4FC8010E94F0C8BECF8F92D7
:109370009F92AF92BF92CF92DF92EF92FF920F93A4
:109380001F93CF93DF93CDB7DEB768970FB6F894EE
:10939000DEBF0FBECDBF6C01809167139091681343
:1093A0000197C9F061E47CE0C6010E940BC9C601C7
:1093B00068960FB6F894DEBF0FBECDBFDF91CF9198
:1093C0001F910F91FF90EF90DF90CF90BF90AF90E3
:1093D0009F908F90089564EC77E0CE010D960E94E7
:1093E0000BC9BE01635F7F4F8BEA9FE00E949AD159
:1093F0006CE271E080E090E00E94086ECE0143963E
:109400000E94214964E670E080E090E00E94086ECE
:1094100010E000E085E0A82EB12C9AE0892E912C76
:109420006FEC77E0CE0101960E940BC9BE016F5F21
:109430007F4FCE0143960E941FC77C01CE0101964B
:109440000E949FC8A7014F5F5F4FBE016D5E7F4FB7
:10945000CE0101960E943C18BE016F5F7F4FCE0186
:109460000D960E945AC8CE0101960E949FC8898914
:109470009A89892B09F170E060E0CE010D960E9477
:109480003AC7082E000C990BC0970A97A8F461ED13
:1094900077E0CE0101960E940BC9BE016F5F7F4F3E
:1094A000CE010D960E944BC7E82ECE0101960E9478
:1094B0009FC8FF24F394E110F12C6EEB7EE0CE0107
:1094C00001960E94F9C844E150E06FEF7FEFCE01B2
:1094D00001960E944419CE0101960E949FC80F5F19
:1094E0001F4F62E370E080E090E00E94086EC801C8
:1094F000B5010E94DBE50197D1F461E070E0CE0197
:1095000001960E944B838D819E81892B09F46AC04C
:10951000BE016F5F7F4F8CEB94E10E9443C80E94B5
:1095200065A3FF24F394CE0101960E949FC8CE014B
:1095300001960E942149BE016F5F7F4FCE01439685
:109540000E945AC8CE0101960E949FC862E370E053
:1095500080E090E00E94086E0436110519F0FF20AB
:1095600009F45ECF80917E0E8823F1F06BE379E001
:10957000CE0101960E940BC9BE01635F7F4FCE01F1
:1095800001960E947CC7BC01CE0107960E9402C9C9
:10959000CE0107960E940B13CE0107960E949FC82A
:1095A000CE0101960E949FC889899A89892B61F012
:1095B00070E060E0CE010D960E943AC7082E000CC4
:1095C000990BC0970A9738F169ED77E0C6010E94C0
:1095D0000BC9CE0143960E949FC8CE010D960E94F2
:1095E0009FC8E5CE043111050CF49DCFC801B4012C
:1095F0000E94DBE5892B09F096CFBE01635F7F4FA8
:109600008BEA9FE00E949AD168EC70E080E090E0E5
:109610000E94086E88CF61ED77E0CE0101960E942E
:109620000BC9BE016F5F7F4FCE010D960E944BC7E5
:10963000182FCE0101960E949FC81111C5CFBE01FF
:10964000635F7F4FC6010E94F0C8C3CF3F924F9225
:109650005F926F927F928F929F92AF92BF92CF92C2
:10966000DF92EF92FF920F931F93CF93DF93CDB7CB
:10967000DEB7E4970FB6F894DEBF0FBECDBF809182
:109680009D0D8823D1F010929D0DE4960FB6F894AD
:10969000DEBF0FBECDBFDF91CF911F910F91FF9025
:1096A000EF90DF90CF90BF90AF909F908F907F9082
:1096B0006F905F904F903F90089581E080939D0D53
:1096C00061E47CE0CE0185960E940BC961E47CE0F8
:1096D000CE018B960E940BC910E000E082E0382E8C
:1096E00098EEC92E93E0D92EE12CF12CF801319798
:1096F000E231F105C0F48827EF57F44B8F4F0C94FB
:10970000EFE5684CFF4C144D1D4D264D2F4D404D3F
:10971000494D784D894D924D9B4DA44D3F4E484E3D
:10972000514E5A4E634E61E47CE0CE0185960E9414
:10973000E2C58091671390916813892B31F46CEF27
:1097400075E0CE0185960E94E2C5809167139091E5
:109750006813019731F466EF75E0CE0185960E949B
:10976000E2C58091671390916813029731F460E02D
:1097700076E0CE0185960E94E2C589A59AA5892B3F
:1097800031F06EE076E1CE0185960E9417C865E063
:1097900076E0CE0101960E940BC96AE176E1CE0126
:1097A00001960E947CC7BC01CE018B960E9443C8E3
:1097B000CE0101960E949FC8809167139091681313
:1097C000019709F046C0BE016B5D7F4FCE01019647
:1097D0000E9402C948EC50E06FEF7FEFCE01019686
:1097E0000E94FD19CE0101960E949FC8BE01655DD1
:1097F0007F4FCE0101960E9402C940ED57E06FEF06
:109800007FEFCE0101960E946313CE0101960E9464
:109810009FC8CE0101960E94B7498D819E81009715
:10982000A1F0E981FA812081222379F0079768F07D
:109830006EEF76E0CE0185960E941EC8BE016F5F76
:109840007F4FCE018B960E9443C8CE0101960E94A5
:109850009FC8BE016B5D7F4FCE0101960E9402C979
:1098600048EC50E06FEF7FEFCE0101960E94441963
:10987000CE0101960E949FC8BE01655D7F4FCE015B
:1098800001960E9402C948EC50E06FEF7FEFCE01D5
:1098900001960E946313CE0101960E949FC80E9408
:1098A0002DB5982EB12CA12C911016C28FEFA81AAD
:1098B000B80A95E6A916B10409F411C20E942DB5A3
:1098C000982E64E170E080E090E00E94086EECCF9A
:1098D00062EF76E0CE0185960E941EC80E943B6E24
:1098E0004B015C010E943B6EA70196010E9433E28E
:1098F000CA01B90120E831E541E050E00E9433E2BD
:1099000020E13EE040E050E00E9401E229AB3AABAA
:109910004BAB5CAB2CE330E040E050E00E9401E256
:1099200029013A01AB01BC01CE0101960E94ECC5B0
:10993000B301A201CE0107960E94ECC549A95AA91C
:109940006BA97CA9CE010D960E94ECC5C501B4019E
:1099500020E03CE546E255E00E9433E2BA01A9016D
:10996000CE0149960E94ECC5BE01675E7F4FCE01D5
:1099700043960E9402C965EE77E0CE0143960E94AD
:1099800066C7BE01635F7F4F0E947CC768EE77E0C9
:109990000E9466C7BE01695F7F4F0E947CC760E975
:1099A00076E00E9466C7BE016F5F7F4F0E947CC752
:1099B00065E577E00E9466C7BC01CE014F960E9424
:1099C00002C9CE0143960E949FC8CE0149960E94CB
:1099D0009FC8CE010D960E949FC8CE0107960E9497
:1099E0009FC8CE0101960E949FC8BE01615E7F4F55
:1099F000CE018B960E945AC8CE014F9628CF8091F7
:109A0000F20D9091F30D63EE76E0019711F065EDA4
:109A100076E0CE0185960E941EC865EC76E0CE0108
:109A20008B960E941EC815CF65EB76E0CE01859619
:109A30000E941EC868EA76E0F2CF6BE976E0CE01BC
:109A400085960E941EC860E976E0E9CF64E876E07A
:109A5000CE0185960E941EC863E776E0E0CF809134
:109A6000F20D9091F30D68E676E0039711F06EE544
:109A700076E0CE0185960E941EC863E576E0CFCFE2
:109A800066E476E0CE0185960E941EC867E376E024
:109A9000C6CF6CE276E0CE0185960E941EC860912A
:109AA0001E1370911F13CE0107960E9419C667E31B
:109AB00077E0CE0101960E940BC9BE01695F7F4F1E
:109AC000CE0101960E947CC768E077E00E9466C7DD
:109AD000BC01CE0185960E9417C8CE0101960E9456
:109AE0009FC8CE0107960E949FC86FE176E097CF8E
:109AF0008091F20D9091F30D6EE076E0029711F0F7
:109B00006EEF75E0CE0185960E941EC861EF75E08C
:109B100086CF65EE75E0CE0185960E941EC865ED84
:109B200075E07DCF6AEC75E0CE0185960E941EC877
:109B300060EC75E074CF64EB75E0CE0185960E9411
:109B40001EC864EA75E06BCFB090201369E975E038
:109B5000CE0185960E941EC883E08B1524F192E009
:109B6000B9160CF073C0BB2031F181E0B81609F4CE
:109B700064C060912013062E000C770BCE0107966F
:109B80000E9419C667E57BE0CE0101960E940BC9D1
:109B9000BE01695F7F4FCE0101960E947CC7BC0168
:109BA0008EE994E13FC094E0B912E3CF6FEE77E025
:109BB0008EE994E146C08090211390902213A090EA
:109BC0002313B090241320E030E048E452E4C501B0
:109BD000B4010E94C4E087FF02C033243394A5017E
:109BE000940160E070E080EA90E40E9443E3AB01FE
:109BF000BC01232DCE0107960E94A7C869EB77E030
:109C0000CE0101960E940BC9BE01695F7F4FCE0154
:109C100001960E947CC764EF77E00E9466C7BC0192
:109C2000CE0185960E9417C8CE0101960E949FC85A
:109C3000CE0107960E949FC806C06BEE77E0CE016A
:109C400085960E940DC869E875E0E9CE8B2D9AE0F3
:109C50008902B0011124CE0107960E9419C667E35C
:109C600077E0CE0101960E940BC9BE01695F7F4F6C
:109C7000CE0101960E947CC76DEE77E0CECF69E7FA
:109C800075E0CE0185960E941EC869E675E0C7CED4
:109C900069E575E0CE0185960E941EC86BE475E00B
:109CA000BECE60E475E0CE0185960E941EC865E3D5
:109CB00075E0B5CE68E275E0CE0185960E941EC8BB
:109CC00068E175E0ACCE6CE075E0CE0185960E944F
:109CD0001EC86DEF74E0A3CE10929D0D21C061E00F
:109CE00070E0CE0101960E944B83BE016F5F7F4FF3
:109CF0008CEB94E10E945AC8CE0101960E949FC845
:109D00008091C0149091C114892B51F480919D0DC4
:109D1000882331F00F5F1F4F0331110509F0E6CCA6
:109D2000CE018B960E949FC8CE0185960E949FC847
:109D3000ACCC2F923F924F925F926F927F928F9214
:109D40009F92AF92BF92CF92DF92EF92FF920F93CA
:109D50001F93CF93DF93CDB7DEB766970FB6F89416
:109D6000DEBF0FBECDBF8C01E090F00DF090F10D85
:109D700080917E0E882349F064E879E082E891E1E1
:109D80000E94BAD1C8010E94B1CCC80105960597BE
:109D900010F40C941E628091F00D9091F10D8017DB
:109DA0009107E1F00E943F130E94A8100C3E2FEF94
:109DB000120724F01093F10D0093F00DB801CE01BD
:109DC00001960E9419C6BE016F5F7F4F8AEA94E137
:109DD0000E945AC8CE0101960E949FC861E47CE0AF
:109DE0008EE994E10E94E2C56EE277E0CE01019631
:109DF0000E940BC94AE050E06FEF7FEFCE01019661
:109E00000E944419CE0101960E949FC8033EFFEFB5
:109E10001F0714F00C942A620E3C3FEF130749F021
:109E2000023E4FEF140729F078010A3B5FEF150758
:109E300051F541E050E066EB74E1CE0101960E94DD
:109E40003C18BE016F5F7F4F82E994E10E945AC8BF
:109E5000CE0101960E949FC882E994E10E945FC6EC
:109E60007801E61AF70A8091961490919714892B3D
:109E700039F0E0919214F09193148081811103C024
:109E80008AE0E81AF108C70188960A9708F0B5C079
:109E900062EE7FEF6E197F09CE0101960E9419C60E
:109EA0006EE778E0CE0107960E940BC9BE016F5F96
:109EB0007F4FCE0107960E947CC7BC0186EB94E1E0
:109EC0000E9443C8CE0107960E949FC8CE0101960A
:109ED0000E949FC867EF77E0CE0101960E940BC9F0
:109EE00066EB74E1CE0101960E947CC7BC0188E953
:109EF00094E10E9443C8CE0101960E949FC868E980
:109F000074E1CE0101960E9402C9CE0101960E9421
:109F10000B13CE0101960E949FC86BEF77E0CE0134
:109F200007960E940BC966EB74E1CE0107960E946A
:109F30007CC7BC01CE0101960E9402C948EC50E0EA
:109F40006FEF7FEFCE0101960E94FD19CE010196C1
:109F50000E949FC8CE0107960E949FC841E050E032
:109F600066EB74E1CE0101960E943C18BE016F5F62
:109F70007F4F82E994E10E945AC8CE0101960E9467
:109F80009FC882E994E10E945FC6DC01CB01019782
:109F9000A109B1096AE277E089309105A105B1050F
:109FA00008F075C1FC018827E752F04B8F4F0C94E5
:109FB000EFE545515A515D51605163516651695108
:109FC0006C516F510E94B81066960FB6F894DEBFC0
:109FD0000FBECDBFDF91CF911F910F91FF90EF90FA
:109FE000DF90CF90BF90AF909F908F907F906F90B9
:109FF0005F904F903F902F900895C701CC960A979D
:10A0000008F0CBC06EEC7FEF6E197F09CE01019690
:10A010000E9419C665E079E0CE0107960E940BC93F
:10A02000BE016F5F7F4FCE0107960E947CC7BC01C7
:10A0300086EB94E10E9443C8CE0107960E949FC818
:10A04000CE0101960E949FC841E050E066EB74E1AA
:10A05000CE0101960E943C18BE016F5F7F4F82E9DE
:10A0600094E10E945AC8CE0101960E949FC882E9DD
:10A0700094E10E945FC6B62EC62ED72EB6E0CB1650
:10A08000D10409F488C10CF02DC1F1E0CF16D10440
:10A090000CF4B7C064E277E08EE994E10E941EC838
:10A0A000F601E956FB4F80818A3008F024C1B601E1
:10A0B000CE0101960E9419C664EB7AE0CE010796A4
:10A0C0000E940BC9BE016F5F7F4FCE0107960E94B1
:10A0D0007CC7BC0184EA94E10E9443C8CE01079684
:10A0E0000E949FC8CE0101960E949FC861E078E05F
:10A0F000CE0101960E940BC94AE050E06FEF7FEF5E
:10A10000CE0101960E94FD19CE0101960E949FC8C2
:10A1100065E070E080E090E00E94086E64EA74E11F
:10A12000CE0101960E9402C94AE050E06FEF7FEF36
:10A13000CE0101960E946313CE0101960E949FC832
:10A140006FE077E08EE994E10E941EC864EA74E152
:10A150008EE994E10E9417C867E077E0CE0101968E
:10A160000E94F9C84AE050E06FEF7FEFCE01019600
:10A170000E94FD19CE0101960E949FC865E070E023
:10A1800080E090E00E94086E6EE974E1CE010196D5
:10A190000E9402C94AE050E086C0C701805B9F4F21
:10A1A0000A9718F56AEB7FEF6E197F09CE010196C9
:10A1B0000E9419C66DEE77E0CE0107960E940BC98A
:10A1C000BE016F5F7F4FCE0107960E947CC7BC0126
:10A1D00086EB94E10E9443C8CE0107960E949FC877
:10A1E000CE0101960E949FC80CC09EECE9169FEF1D
:10A1F000F90609F429CFA2EEEA16AFEFFA0609F440
:10A2000069CEF092F10DE092F00D8091A214909140
:10A21000A314009799F14197A8F40230110594F026
:10A220006EE974E1CE0101960E9402C94AE050E055
:10A230006FEF7FEFCE0101960E946313CE0101966E
:10A240000E949FC86EE974E1CE0101960E9402C986
:10A25000CE0101960E940B13CE0101960E949FC869
:10A260006EE974E1CE0101960E9402C9CE01019609
:10A270000E944818CE0101960E949FC864E670E0D3
:10A2800080E090E00E94086E9FCE6BE977E088E95D
:10A2900094E10E941EC868E974E1CE0101960E9413
:10A2A00002C94CED55E06FEF7FEFCE0101960E94A1
:10A2B000631396CF6EE877E0EACF6EE777E0E7CFFB
:10A2C00064E777E0E4CF60E777E0E1CF60E677E04E
:10A2D000DECF62E577E0DBCF64E477E0D8CF67E3F9
:10A2E00077E0D5CF27E0C216D10409F08ACF80E00D
:10A2F0000E94462886CF36E3B30E8A3031F58BE0D4
:10A30000808361E08B2D0E944E6DB601CE010796D1
:10A310000E9419C6BE01695F7F4FCE0101960E945F
:10A3200002C96EE078E0CE0101960E9466C7BC01CA
:10A330008EE994E10E9417C8CE0101960E949FC841
:10A34000CE0107960E949FC807CF8AE08083B6019E
:10A35000CE0107960E9419C6BE01695F7F4FCE01EC
:10A3600001960E9402C964E178E0CE0101960E9444
:10A3700066C7BC018EE994E10E9417C8CE01019620
:10A380000E949FC8CE0107960E949FC860E08B2D57
:10A390000E944E6DE1CE88E390E00E94E92C31CF1F
:10A3A0000E943F1389E390E00E94671220E030E0B2
:10A3B0004AE754E40E942AE1AB01BC0121E0CE014E
:10A3C00001960E94A7C864E37BE0CE0107960E9435
:10A3D0000BC9BE016F5F7F4FCE0107960E947CC7FD
:10A3E00069E178E00E9466C7BC018EE994E10E94B1
:10A3F00043C8CE0107960E949FC8CE0101960E94D5
:10A400009FC86DE178E088E994E10E94E2C568E9BF
:10A4100074E1CE0101960E9402C94AE050E068E072
:10A4200070E0CE0101960E94FD19CE0101960E94B6
:10A430009FC86EE974E1CE0101960E9402C94AE00C
:10A4400050E06FEF7FEFCE0101960E946313CE01C3
:10A4500001960E949FC868E974E18EE994E10E9428
:10A4600017C880917D0E882309F4CFCE64E670E092
:10A4700080E090E02BC4C0900402D09005020E94BE
:10A480003F1389E390E00E94671220E030E04AE742
:10A4900054E40E942AE10E94EFE3CE0101960E945B
:10A4A00019C664E37BE0CE0107960E940BC9BE018A
:10A4B0006F5F7F4FCE0107960E947CC769E178E00D
:10A4C0000E9466C7BC018EE994E10E9443C8CE0198
:10A4D00007960E949FC8CE0101960E949FC8809156
:10A4E000A2149091A31423E0F22E099710F092E0A9
:10A4F000F92E80911D1340E050E0BA018330DCF466
:10A50000C6010E94F2114B015C0160911E13709113
:10A510001F13072E000C880B990B0E94CBE0A5019E
:10A5200094010E942AE120E030EC4FE754E40E94BD
:10A5300043E3AB01BC012F2DCE0101960E94A7C8B9
:10A540006EE478E0CE0107960E940BC9BE016F5FF2
:10A550007F4FCE0107960E947CC765E278E00E949B
:10A5600066C7BC018EE994E10E9417C8CE01079628
:10A570000E949FC8CE0101960E949FC868E278E0C1
:10A5800042CF80917D0E882309F439C188E490E19F
:10A590000E94E8B062E370E080E090E00E94086E04
:10A5A00061E08091A6040E94806D60E08091A40427
:10A5B0000E94806D64E670E080E090E00E94086E8A
:10A5C0006091A0047091A1048091A2049091A304D1
:10A5D0000E948B100E94AF0FAB01BC0123E0CE01A3
:10A5E00007960E94A7C8BE01695F7F4FCE01019602
:10A5F0000E9402C96BE478E0CE0101960E9466C712
:10A60000BC0188E994E10E9443C8CE0101960E94F2
:10A610009FC8CE0107960E949FC864E976E0CE01EC
:10A6200001960E940BC968E974E1CE0101960E946F
:10A630007CC7BC018EE994E10E9443C8CE0101961B
:10A640000E949FC80E94AF0F6B017C010E94E36DC6
:10A650004B015C018BE19EE40197F1F70E94AF0F83
:10A660002B013C010E94E36D9B01AC0128193909C3
:10A670004A095B0949015A0131ED831637E0930617
:10A68000A104B104CCF0A7019601C301B2010E945C
:10A6900064E26B017C0120E030E0A9010E944CE4FF
:10A6A000181674F426EA3BE944EC5BE3C701B601F3
:10A6B0000E94C4E087FF0EC040E050E0BA0126C00F
:10A6C00026EA3BE944EC5BEBC701B6010E944CE48F
:10A6D000181694F3C501B40128EE33E040E050E0D1
:10A6E0000E9401E2CA01B9010E94CBE04B015C016A
:10A6F00020E030E04AE754E4C701B6010E942AE1B5
:10A70000A50194010E9443E3AB01BC0122E0CE010C
:10A7100007960E94A7C8BE01695F7F4FCE010196D0
:10A720000E9402C967E976E0CE0101960E9466C7E1
:10A73000BC0182E994E10E9443C8CE0101960E94C7
:10A740009FC8CE0107960E949FC861E378E0CE01C2
:10A7500001960E940BC962E974E1CE0101960E9444
:10A760007CC7BC018EE994E10E9417C8CE01019616
:10A770000E949FC86EE277E0CE0101960E940BC94D
:10A7800062E974E1CE0101960E947CC7BC0188E9B0
:10A7900094E10E9417C8CE0101960E949FC86BEAFF
:10A7A00077E0CE0101960E94F9C84AE050E070E0DF
:10A7B00060E0CE0101960E94FD19CE0101960E9433
:10A7C0009FC868E974E1CE0101960E9402C945E084
:10A7D00050E06FEF7FEFCE0101960E946313CE0130
:10A7E00001960E949FC865E378E08EE994E10E949B
:10A7F0000DC860E08091A6040E94806D06CD609136
:10A800008F047091900480919104909192040E9421
:10A81000B52EFBCC8091890490918A040E94D0309F
:10A82000F4CC40918B044E8B60E0842F0E94806DAD
:10A8300080917D0E811191C18091931381118DC101
:10A840008FE0C82ED12CE12CF12C6AEB77E08EE959
:10A8500094E10E941EC86EE974E1CE0101960E9447
:10A8600002C94AE050E06FEF7FEFCE0101960E94EF
:10A87000FD19CE0101960E949FC8312C212C198A06
:10A880001D8A1D861E861F86188AA2E36A2E712CD9
:10A89000812C912C54018E890E94C06D092E000CD0
:10A8A000AA0BBB0B880E991EAA1EBB1E65E070E0AA
:10A8B00080E090E00E94086E51E0651A710859F737
:10A8C0004090F2045090F3046090F4047090F5040A
:10A8D000C501B4010E94CBE020E030E040EA50E442
:10A8E0000E942AE120E030E040E85AE30E942AE199
:10A8F00020E030E048E452E40E9443E3A3019201E7
:10A900000E9464E220E030E040E751E40E942AE146
:10A910004B015C01A30192016AE979E989E390E4C2
:10A920000E9464E29B01AC01C501B4010E9443E3B3
:10A9300020E030E0A9010E9465E220E030E040E242
:10A9400051E40E942AE14B015C01232D322D4989FB
:10A950005D890E944CE4181624F4382C292CA98A0D
:10A96000BD8A20E030E0A901B401C5010E94C4E025
:10A9700087FF04C0812C912CA12CB12C22E0A401D2
:10A98000B501CE0107960E94A7C8BE01695F7F4F3F
:10A99000CE0101960E9402C968E478E0CE010196DA
:10A9A0000E9466C7BC0188E994E10E9443C8CE01B9
:10A9B00001960E949FC8CE0107960E949FC868E931
:10A9C00074E1CE0101960E9402C94AE050E070E0B5
:10A9D00060E0CE0101960E946313CE0101960E94B1
:10A9E0009FC80E943B6EAB01BC018091A00C90916E
:10A9F000A10CA091A20CB091A30C8C599F4FAF4F0A
:10AA0000BF4F84179507A607B70708F0ACC00E9490
:10AA100021106CE370E080E090E00E94086E8D856C
:10AA20009E85AF85B8890196A11DB11D8D879E8732
:10AA3000AF87B88BC816D906EA06FB060CF025CFFF
:10AA400064E670E080E090E00E94086E0E943F1390
:10AA500064E670E080E090E00E94086E62EB77E0D0
:10AA600088E994E10E941EC868E974E1CE0101966C
:10AA70000E9402C944E150E070E060E0CE0101961E
:10AA80000E94FD19CE0101960E949FC822E0432D2D
:10AA9000522D69897D89CE0107960E94A7C8BE0103
:10AAA000695F7F4FCE0101960E9402C968E478E099
:10AAB000CE0101960E9466C7BC0188E994E10E941C
:10AAC00043C8CE0101960E949FC8CE0107960E94FE
:10AAD0009FC868E974E1CE0101960E9402C942E371
:10AAE00050E06FEF7FEFCE0101960E946313CE011D
:10AAF00001960E949FC864E170E080E090E00E94AF
:10AB0000086E0E9421106EE170E080E090E00E94EB
:10AB1000086E6EE170E080E090E00E94086E6DE4E7
:10AB200078E0CE0101960E940BC968E974E1CE017C
:10AB300001960E947CC761E578E00E9466C76EE9D5
:10AB400074E10E947CC7BC018EE994E10E9443C875
:10AB5000CE0101960E949FC858CBB3E0CB2ED12CDA
:10AB6000E12CF12C72CE0E943B6E0E94C9E04B0199
:10AB70005C016091A00C7091A10C8091A20C90914D
:10AB8000A30C0E94CBE020E030E048EC51E40E94AE
:10AB900065E29B01AC01C501B4010E94C4E087FDE0
:10ABA00036CF37CF80918D0490918E0499270E94E3
:10ABB000F2112DE038E643E55BE30E942AE16B01E8
:10ABC0007C012091290530912A0540912B05509157
:10ABD0002C050E94C4E018160CF47BC0609111058E
:10ABE00070911205809113059091140520E030E0DA
:10ABF00048EC52E40E942AE120E030E048EA51E4C7
:10AC00000E942AE12091F6043091F7044091F80463
:10AC10005091F9040E9443E36B017C0167EC77E0FB
:10AC200088E994E10E941EC868E974E1CE010196AA
:10AC30000E9402C942E350E070E060E0CE0101965C
:10AC40000E94FD19CE0101960E949FC822E0B70123
:10AC5000A601CE0101960E94A7C86BE578E0CE015F
:10AC600007960E940BC9BE016F5F7F4FCE0107960A
:10AC70000E947CC765E578E00E9466C7BC018EE94A
:10AC800094E10E9443C8CE0107960E949FC8CE015E
:10AC900001960E949FC86EE974E1CE0101960E9460
:10ACA00002C942E350E06FEF7FEFCE0101960E94B0
:10ACB0006313CE0101960E949FC880917D0E882368
:10ACC00009F4A3CA60E273E080E090E00E94086E9D
:10ACD0009CCA20913D0530913E0540913F05509121
:10ACE0004005C701B6010E944CE487FF05C0C701BB
:10ACF000B6010E943FAF7ACF60912505709126057D
:10AD0000809127059091280571CF0E943F136BEF2A
:10AD100077E08EE994E10E941EC86EE974E1CE01ED
:10AD200001960E9402C94AE050E070E060E0CE0166
:10AD300001960E94FD19CE0101960E949FC862EF04
:10AD400077E088E994E10E941EC868E974E1CE01C9
:10AD500001960E9402C944E150E06FEF7FEFCE01FF
:10AD600001960E946313CE0101960E949FC88091B4
:10AD7000A40C9091A50C8230910509F041C00E946D
:10AD8000B5C4811104C01092A50C1092A40C80913E
:10AD9000A40C9091A50C029709F448C066EE77E0E8
:10ADA0008EE994E10E941EC86EE974E1CE0101961D
:10ADB0000E9402C94AE050E070E060E0CE010196D6
:10ADC0000E94FD19CE0101960E949FC86EE974E1B0
:10ADD000CE0101960E9402C96EE277E0CE01019693
:10ADE0000E9466C768E974E10E947CC7BC018EE9D5
:10ADF00094E10E9443C8CE0101960E949FC85DCF96
:10AE0000892B61F60E94B5C4882339F082E090E076
:10AE10009093A50C8093A40CBACF0E94B5C4811165
:10AE2000F5CF0E94B5C48111F1CFB1CF8AE090E097
:10AE30000E947B166B017C0120E030E0A9010E949A
:10AE4000C4E0181634F08AE090E00E947B166B0193
:10AE50007C01FBE0AF2EB12C20E030E042ED53E46A
:10AE6000C701B6010E94C4E018168CF091E0A91A3F
:10AE7000B10869F068EC70E080E090E00E94086E34
:10AE800083E090E00E947B166B017C01E5CF20E01F
:10AE900030E0A901C701B6010E94C4E018166CF1A8
:10AEA00068ED77E08EE994E10E941EC86EE974E1D6
:10AEB000CE0101960E9402C942E350E06FEF7FEF9E
:10AEC000CE0101960E946313CE0101960E949FC895
:10AED0006FEC77E088E994E10E941EC868E974E1AC
:10AEE000CE0101960E9402C942E350E070E060E0AA
:10AEF000CE0101960E94FD19DCCE20E030E048EC46
:10AF000052E4C701B6010E94C4E021E087FF20E0BF
:10AF1000B701A601CE0101960E94A7C86AE578E0B4
:10AF2000CE0107960E940BC9BE016F5F7F4FCE0115
:10AF300007960E947CC76FE578E00E9466C7BC0157
:10AF40008EE994E10E9443C8CE0107960E949FC8F3
:10AF5000CE0101960E949FC8A9CF0E943B6E0E941D
:10AF6000FF1B53C9E0908704F090880463E678E003
:10AF700088E994E10E94E2C50E943F1368E974E108
:10AF8000CE0101960E9402C94AE050E06FEF7FEFC8
:10AF9000CE0101960E94FD19CE0101960E949FC824
:10AFA000C7010E94E412698B7A8B8B8B9C8B8090FB
:10AFB000D7049090D804A090D904B090DA04A501E9
:10AFC00094016091D3047091D4048091D504909140
:10AFD000D6040E9464E22B013C0120E030E0A9018C
:10AFE0000E94C4E0882309F48AC0C090DF04D09096
:10AFF000E004E090E104F090E20420E030E0A901F8
:10B00000C701B6010E94C4E018160CF078C0209168
:10B01000DB043091DC044091DD045091DE042D8787
:10B020003E874F87588BC701B6010E94C4E0882332
:10B0300009F465C0A70196016D857E858F85988985
:10B040000E9443E30E949BE46D877E878F87988BE5
:10B05000A501940169897A898B899C890E9464E29F
:10B06000A30192010E9443E32D853E854F855889B7
:10B070000E942AE10E94BDE39B01AC01C701B60119
:10B080000E942AE16B017C0168E974E1CE0101961E
:10B090000E9402C94AE050E070E060E0CE010196F3
:10B0A0000E94FD19CE0101960E949FC820E030E663
:10B0B0004AEE56E4C701B6010E944CE418161CF58E
:10B0C00065E078E08EE994E10E941EC86EE974E1C3
:10B0D000CE0101960E9402C94AE050E06FEF7FEF77
:10B0E000CE0101960E946313CE0101960E949FC873
:10B0F00064E670E080E090E00E94086EDECDC12C36
:10B10000D12C7601C1CF21E0B701A601CE0107966F
:10B110000E94A7C86DE678E0CE0101960E940BC997
:10B12000BE01695F7F4FCE0101960E947CC761E737
:10B1300078E00E9466C7BC018EE994E10E9443C892
:10B14000CE0101960E949FC8CE0107960E949FC81B
:10B15000BDCFE0900402F09005020E943F1365E02D
:10B1600070E080E090E00E94086E80911D1340E046
:10B1700050E0BA018330DCF4C7010E94F2116B0188
:10B180007C0160911E1370911F13072E000C880B19
:10B19000990B0E94CBE0A70196010E942AE120E0D2
:10B1A00030EC4FE754E40E9443E3AB01BC0123E0E1
:10B1B000CE0101960E94A7C86EE478E0CE01079602
:10B1C0000E940BC9BE016F5F7F4FCE0107960E94A0
:10B1D0007CC765E278E00E9466C7BC018EE994E115
:10B1E0000E9443C8CE0107960E949FC8CE010196D7
:10B1F0000E949FC865E778E006C98091C00C91E085
:10B2000089278093C00C80917D0E882331F06EE9F0
:10B2100074E18BEA9FE00E94A8D168EC70E080E0C6
:10B2200090E054CD10927D0E0C94055181E08093F6
:10B230007D0E8093A11380919813882349F169E0D2
:10B240007BE08AEA94E10E94E2C586EE9FEF90934C
:10B25000F10D8093F00D20919B1330919C13809100
:10B260009D1390919E138217930724F010929E13C2
:10B2700010929D1310928F131092901310929113AD
:10B28000109292136CE271E080E090E00E94086EF0
:10B290006AEA74E180EB94E10E9443C88091F00D6A
:10B2A0009091F10D9093740E8093730E0C94055150
:10B2B0000E94264B0C94055185EE90E10E94E8B067
:10B2C00040E052EC61E070E085EE90E10E943716BC
:10B2D0008CED95E0A0E0B0E08093E9109093EA1047
:10B2E000A093EB10B093EC1064E670E080E090E087
:10B2F0000E94086E8091A40C9091A50C019709F012
:10B30000D3C083E090E00E94A01781110BC010927F
:10B31000A50C1092A40C8091A40C9091A50C0197FF
:10B3200009F0DBC06CE278E08EE994E10E941EC86F
:10B330006EE974E1CE0101960E9402C9CE01019628
:10B340000E94051ECE0101960E949FC862E370E034
:10B3500080E090E00E94086E6EE974E1CE010196F3
:10B360000E9402C942E350E06FEF7FEFCE010196E9
:10B370000E94FD19CE0101960E949FC860E278E00C
:10B3800088E994E10E941EC868E974E1CE01019643
:10B390000E9402C944E150E06FEF7FEFCE010196B9
:10B3A0000E946313CE0101960E949FC88BEB8F838E
:10B3B0008AEA888781E0898768011801412C512C2D
:10B3C0003201C6016AE070E00E94DBE5892B49F496
:10B3D00043E050E0BE01695F7F4F85EE90E10E943F
:10B3E0005EAA65E070E080E090E00E94086E5FEF8A
:10B3F000C51AD50A7801812C912C540185EE90E173
:10B400000E94D5AA892B39F484E088169104A104FE
:10B41000B1040CF081C096E0E916F1040CF07CC098
:10B4200085EE90E10E94D5AA892B71F085EE90E11E
:10B430000E94B3AAE1E0F0E0EC0FFD1FEE0DFF1D4E
:10B440008083AFEFEA1AFA0A65E070E080E090E0EE
:10B450000E94086EB6E0EB16F10401F599818F8128
:10B4600098131CC09A818885981318C09B81898580
:10B47000981314C08D8190E0B0E0A0E0BA2FA92FFE
:10B48000982F88272C81820F911DA11DB11D480E78
:10B49000591E6A1E7B1EEFEF2E1A3E0AFFEF8F1A0F
:10B4A0009F0AAF0ABF0AAACF81E090E00E94A017CE
:10B4B000882339F081E090E09093A50C8093A40C50
:10B4C0002ACF83E090E00E94A0178111F3CF83E0A0
:10B4D00090E00E94A0178111EDCF64E478E088E944
:10B4E00094E10E941EC868E974E1CE0101960E94B1
:10B4F00002C944E150E06FEF7FEFCE0101960E9458
:10B500006313CE0101960E949FC868E378E08EE93C
:10B5100094E10E941EC84AC034E02316310434F47A
:10B5200040E9C41641E0D40609F04BCFC301B20193
:10B530000E94CBE020E030E040E251E40E9443E38F
:10B5400020E030E040E85EE30E942AE16B017C01EC
:10B5500020E030E040EA51E40E944CE418160CF080
:10B5600055C021E0B701A601CE0101960E94A7C8EF
:10B570006FE67AE0CE0107960E940BC9BE016F5FAD
:10B580007F4FCE0107960E947CC76DE778E00E944E
:10B5900066C7BC018EE994E10E9443C8CE010796BC
:10B5A0000E949FC8CE0101960E949FC86EE974E177
:10B5B000CE0101960E9402C94AE050E070E060E0CE
:10B5C000CE0101960E94FD19CE0101960E949FC8EE
:10B5D0006EE974E1CE0101960E9402C96EE277E045
:10B5E000CE0101960E9466C768E974E10E947CC79B
:10B5F000BC018EE994E10E9443C8CE0101960E94ED
:10B600009FC885EE90E10E94E8B057CB64E178E0F6
:10B610007ECF6FED78E0CE0101960E94F9C84AE036
:10B6200050E06FEF7FEFCE0101960E946313CE01D1
:10B6300001960E949FC860919E0470919F04809122
:10B64000F0049091F1040E94F61374E1872E912C7E
:10B65000A12CB12CD12CC12C4FEFC41AD40AC50196
:10B66000B4010E94086E60919E0470919F048091C5
:10B67000F0049091F1040E94F6137C0153E0C5168A
:10B68000D10434F02EE1C216D10444F4EF2851F075
:10B6900034E1830E911CA11CB11CDECFE114F10436
:10B6A00009F00CC18091F0049091F1048B30910568
:10B6B00009F0DFC08091351590913615A0913715AE
:10B6C000B09138158093EC0D9093ED0DA093EE0D95
:10B6D000B093EF0D8091311590913215A0913315F3
:10B6E000B09134158093E80D9093E90DA093EA0D85
:10B6F000B093EB0D4091EC0D5091ED0D6091EE0D7E
:10B700007091EF0D21E0CE0101960E94A7C86DEB6C
:10B7100076E0CE0107960E940BC9BE016F5F7F4F96
:10B72000CE0107960E947CC7BC018EE994E10E947D
:10B7300043C8CE0107960E949FC8CE0101960E9481
:10B740009FC84091E80D5091E90D6091EA0D70910C
:10B75000EB0D21E0CE0101960E94A7C860E878E0D9
:10B76000CE0107960E940BC9BE016F5F7F4FCE01CD
:10B7700007960E947CC7BC018EE994E10E9417C81D
:10B78000CE0107960E949FC8CE0101960E949FC8D5
:10B7900068E578E08EE994E10E940DC861E47CE000
:10B7A000CE0101960E940BC944E150E070E060E0D8
:10B7B000CE0101960E94FD19CE0101960E949FC8FC
:10B7C000C090EC0DD090ED0DE090EE0DF090EF0DEF
:10B7D00020E030E0A901C701B6010E944CE420E05E
:10B7E00030E040E05FE387FD64C0C701B6010E941E
:10B7F00065E20E94EFE3AB01BC01CE0101960E941D
:10B80000ECC5BE016F5F7F4F88E994E10E945AC882
:10B81000CE0101960E949FC860E087E00E94E8ADDB
:10B8200068E974E186E296E10E949AD16FED86E2C2
:10B8300096E10E947DCB66E878E086E296E10E9480
:10B84000C4CC6091E80D7091E90D8091EA0D909162
:10B85000EB0D0E94EFE34AE050E086E296E10E94A1
:10B8600077CC68E578E086E296E10E94C4CC0C943F
:10B8700036528631910509F41DCF0C9709F03ACF65
:10B880008091DF0D9091E00DA091E10DB091E20D5E
:10B890008093EC0D9093ED0DA093EE0DB093EF0D12
:10B8A0008091DB0D9091DC0DA091DD0DB091DE0D4E
:10B8B00019CFC701B6010E9464E29BCF8FEFE81653
:10B8C000F806D4F061ED78E0CE0101960E94F9C847
:10B8D0004AE050E070E060E0CE0101960E94FD1960
:10B8E000CE0101960E949FC86EEA78E08EE994E14D
:10B8F0000E941EC80C9405519EEFE9169FEFF906B1
:10B9000081F160EA78E0CE0101960E94F9C84AE030
:10B9100050E070E060E0CE0101960E94FD19CE017A
:10B9200001960E949FC861E978E08EE994E10E9447
:10B930001EC8B701CE0101960E9419C6BE016F5FF5
:10B940007F4F8EE994E10E9417C8CE0101960E94B4
:10B950009FC86BE778E08EE994E10E948FC70C9452
:10B96000055160E778E0CE0101960E94F9C84AE0EF
:10B9700050E070E060E0CE0101960E94FD19CE011A
:10B9800001960E949FC860E578E0B0CF8091A8043E
:10B99000882311F40C94055161E47CE0CE010196FA
:10B9A0000E940BC94AE050E061E070E0CE010196D0
:10B9B0000E94FD19CE0101960E949FC80E94BC36CC
:10B9C0000C94055180917D0E811109C080919313D3
:10B9D0006EE1462E512C612C712C882329F053E006
:10B9E000452E512C612C712C6DEE78E08EE994E19E
:10B9F0000E941EC86EE974E1CE0101960E9402C940
:10BA00004AE050E06FEF7FEFCE0101960E94631392
:10BA1000CE0101960E949FC8812C912C54011D8655
:10BA20001E861F86188A83E20E94CDAD67E070E013
:10BA300089ED94E10E94EF1389ED94E10E949174E5
:10BA400066E970E080E090E00E94086E83E20E9468
:10BA5000CDAD60E270E089ED94E10E94EF1389EDD5
:10BA600094E10E94917466E970E080E090E00E94A9
:10BA7000086E42E050E063E270E089ED94E10E94DC
:10BA8000DD74C12CD12C76018091080F9091090FA3
:10BA9000891B990B181619065CF40E94C7B1FE2C7D
:10BAA000ED2CDC2CCC24C80ED11CE11CF11CECCFFD
:10BAB000C701B6010E94CBE02AE939E949E95FE311
:10BAC0000E9443E30E94EFE3AB01BC01841695069C
:10BAD000A606B70614F44A015C01CE0107960E943F
:10BAE000ECC5BE01695F7F4FCE0101960E9402C97D
:10BAF00069E878E0CE0101960E9466C7BC0188E93A
:10BB000094E10E9443C8CE0101960E949FC8CE01D5
:10BB100007960E949FC868E974E1CE0101960E94D1
:10BB200002C94EE150E070E060E0CE0101960E9453
:10BB30004419CE0101960E949FC82D853E854F85F0
:10BB400058892F5F3F4F4F4F5F4F2D873E874F875D
:10BB5000588B42165306640675060CF064CFB50187
:10BB6000A401CE0107960E94ECC5BE01695F7F4F1C
:10BB7000CE0101960E9402C969E878E0CE010196E3
:10BB80000E9466C7BC0188E994E10E9443C8CE01C7
:10BB900001960E949FC8CE0107960E949FC868E93F
:10BBA00074E1CE0101960E9402C94AE050E070E0C3
:10BBB00060E0CE0101960E94FD19CE0101960E941F
:10BBC0009FC8B501A401CE0101960E94ECC568ECA6
:10BBD00078E0CE0107960E940BC9BE016F5F7F4FD0
:10BBE000CE0107960E947CC76DE878E00E9466C788
:10BBF0006EE974E10E947CC7BC018EE994E10E9469
:10BC000043C8CE0107960E949FC8CE0101960E94AC
:10BC10009FC862E370E080E090E058C8E0900202C4
:10BC2000F090030281E08093FA0464E670E080E023
:10BC300090E00E94086E0E943F13C7010E94F2111B
:10BC40000E94EFE320E034E0A901461B570BBA0144
:10BC5000CE0101960E9419C662E978E0CE010796EE
:10BC60000E940BC9BE016F5F7F4FCE0107960E94F5
:10BC70007CC7BC018EE994E10E9443C8CE010796BF
:10BC80000E949FC8CE0101960E949FC860E087E095
:10BC90000E94E8AD6DEF78E0CE0101960E94F9C8F0
:10BCA00042E350E068E070E0CE0101960E94FD1989
:10BCB000CE0101960E949FC86EE974E1CE01019603
:10BCC0000E9402C942E350E06FEF7FEFCE01019680
:10BCD0000E946313CE0101960E949FC869E978E033
:10BCE000CE0101960E940BC96EE974E1CE01019666
:10BCF0007BC880910002909101020E94F2110E9483
:10BD0000EFE37093A70C6093A60C62E370E080E011
:10BD100090E00E94086E6091A60C7091A70CCE0175
:10BD200001960E9419C6BE016F5F7F4F8EE994E1B4
:10BD30000E945AC8CE0101960E949FC880912F157B
:10BD400090913015892B09F45EC06BE275E1CE014C
:10BD500007960E9402C9BE01695F7F4FCE0101961E
:10BD60000E9402C944E150E070E060E0CE0101961B
:10BD70000E94FD19CE0101960E949FC863EA78E0F7
:10BD8000CE0101960E940BC96EE974E1CE010196C5
:10BD90000E947CC7BC0188E994E10E9443C8CE019F
:10BDA00001960E949FC868E974E1CE0101960E9445
:10BDB00002C944E150E06FEF7FEFCE0101960E948F
:10BDC0006313CE0101960E949FC8BE01695F7F4F39
:10BDD000CE0101960E9402C96EE277E0CE01019683
:10BDE0000E9466C768E974E10E947CC7BC018EE9C5
:10BDF00094E10E9443C8CE0101960E949FC8CE01E3
:10BE000007960C945B566EEA78E088E994E10E940C
:10BE1000E2C568E974E1CE0101960E9402C944E1DD
:10BE200050E070E060E0CE0101960E94FD19CE0165
:10BE300001960E949FC862E978E0CE0101960E94B7
:10BE40000BC96EE974E1CE0101960E947CC7BC016A
:10BE500088E994E10E9443C8CE0101960E949FC8E0
:10BE600068E974E1CE0101960E9402C944E150E004
:10BE70006FEF7FEFCE0101960E946313CE01019612
:10BE80000E949FC863EA78E02BCF8091A8048823A2
:10BE900011F40C94055180917D0E811104C08091A4
:10BEA0009313882331F082E090E00E9439440C948F
:10BEB0000551C0908F04D0909004E0909104F090D0
:10BEC000920420E030E040E450E4C701B6010E9453
:10BED0004CE418160CF054C020E030E04AEF54E473
:10BEE000C701B6010E942AE10E94EFE36B017C01C9
:10BEF0000E943F1360E080E00E94E8AD6EE079E0D0
:10BF000086E296E10E94BAD161E080E00E94E8AD4D
:10BF100066E079E086E296E10E94BAD164E670E0DC
:10BF200080E090E00E94086E0E943B6E6093A80C37
:10BF30007093A90C8093AA0C9093AB0C0E943B6E5B
:10BF40008090A80C9090A90CA090AA0CB090AB0C7B
:10BF5000681979098A099B096C157D058E059F056D
:10BF600014F00C94055183E090E00E9439440E9443
:10BF70003B6E64E170E080E090E00E94086EDECFEE
:10BF800030E3C32E35E7D32EE12CF12CB1CF0E9444
:10BF90005F338BEA9FE00E94BDAC0C9405516EE2CA
:10BFA00079E088E994E10E941EC868E974E1CE0155
:10BFB00001960E9402C94AE050E070E060E0CE01C4
:10BFC00001960E94FD19CE0101960E949FC83090F3
:10BFD00006028091B80C811105C00E943B6E81E081
:10BFE0008093B80C8091B00C811105C00E943B6E0B
:10BFF00081E08093B00C1092E70C1092E60CE09078
:10C00000E60CF090E70C58E2E516F1040CF07EC067
:10C01000832D0E94C06DF701EE0FFF1FE45FF04F0C
:10C02000918380830E9415AE20E030E040EA50E426
:10C030000E942AE120E030E040E85AE30E942AE131
:10C040006B017C014090CF045090D0046090D104EB
:10C050007090D204A30192016091CB047091CC0442
:10C060008091CD049091CE040E9464E29B01AC01CA
:10C0700060E070E080EC90E40E9464E24B015C01BF
:10C0800020E030E0A9010E94C4E020E030E040E67A
:10C0900050E481111CC0C701B6010E942AE16093DF
:10C0A000AC0C7093AD0C8093AE0C9093AF0C64E12C
:10C0B00070E080E090E00E94086E8091E60C909124
:10C0C000E70C01969093E70C8093E60C98CFC7019C
:10C0D000B6010E942AE1A30192010E9465E220E0DC
:10C0E00030E040E850E40E9464E2A50194010E941F
:10C0F00043E320E030E040EC50E40E942AE120E0FD
:10C1000030E040E850E40E9465E2C9CFC090AC0C3A
:10C11000D090AD0CE090AE0CF090AF0C20E030E091
:10C12000A901C701B6010E944CE487FD22C022E0AC
:10C13000B701A601CE0107960E94A7C862EB78E07E
:10C14000CE0101960E940BC9BE01695F7F4FCE01EF
:10C1500001960E947CC7BC018EE994E10E9443C80D
:10C16000CE0101960E949FC8CE0107960E949FC8EB
:10C1700006C06FE179E08EE994E10E941EC86EE985
:10C1800074E1CE0101960E9402C94AE050E06FEFCF
:10C190007FEFCE0101960E9463135BC08091A804DB
:10C1A000882311F40C94055180917D0E81112EC0CD
:10C1B0008091931381112AC0C0908F04D090900475
:10C1C000E0909104F090920420E030E04AE754E4DB
:10C1D000C701B6010E942AE10E94EFE34B015C0116
:10C1E00020E030E040EA50E4C701B6010E942AE1B5
:10C1F00020E030E040EA50E40E9465E20E94EFE374
:10C20000A50194010E94BE3B0C94055121E030E051
:10C2100040E050E06AE070E080E090E0F3CFC701DA
:10C220000E943D380C940551C7010E945B620C943A
:10C23000055180917E0E882311F40C9405516CE712
:10C2400079E0CE0101960E94F9C8CE0101960E94C4
:10C250000B13CE0101960E949FC80C94055180914A
:10C260000A0F90910B0F892B81F481E090E090935D
:10C270000B0F80930A0F8EE492E00E941CB068ECD2
:10C2800070E080E090E00E94086E6FE679E0CE01F9
:10C2900001960E94F9C844E650E06FEF7FEFCE01AF
:10C2A00001960E946313CE0101960E949FC8F0E0A0
:10C2B000E0E019950C9405510E9478C50E943F1347
:10C2C0000E94A8100C9405518091981391E0892741
:10C2D00080939813882309F48BC068E679E08EE98F
:10C2E00094E10E941EC80E943B6E60938F1370936E
:10C2F0009013809391139093921380919B1390913C
:10C300009C13181619065CF420919D1330919E130E
:10C310002817390724F010929E1310929D139091C4
:10C320009F1380919A13981724F010929F131092E4
:10C33000A01380919813809393136EE974E1CE015A
:10C3400001960E9402C94AE050E068E070E0CE0128
:10C3500001960E94FD19CE0101960E949FC863E5D7
:10C3600079E0CE0101960E94F9C84AE050E06FEFF3
:10C370007FEFCE0101960E946313CE0101960E94C9
:10C380009FC865E479E08EE994E10E948FC76BE372
:10C3900079E0CE0101960E940BC96EE974E1CE01ED
:10C3A00001960E947CC7BC018EE994E10E9443C8BB
:10C3B000CE0101960E949FC880917D0E8093A113AB
:10C3C0008CE291E00E9447B080917D0E882311F4A9
:10C3D0000C94055169E07BE08AEA94E10E94E2C591
:10C3E00086EE9FEF9093F10D8093F00D0C94055124
:10C3F00060E679E08EE994E10E941EC89ACFF0923F
:10C40000F10DE092F00D8BEA9FE00E94BDAC67E376
:10C4100079E08EE994E10E941EC861E47CE0CE01DF
:10C4200001960E940BC94AE050E070E060E0CE0146
:10C4300001960E94FD19CE01019698CE0E3F2FEF76
:10C44000120711F40C94E24F61E47CE08EE994E170
:10C450000E94E2C5F8017C96E632F10580F6882755
:10C46000EB5CFD498F4F0C94EFE50F61FF61646158
:10C470005C612F611961FF611461FF61FF61FF6100
:10C48000FF61FF61D0513B52C1520A541154D25541
:10C490008556AD57B257A958FD5812591659FF6124
:10C4A00058595C59095BC65CE25C0E5E795E455F7B
:10C4B000C75FCF5FCE60CF92DF92EF92FF920F9374
:10C4C0001F93CF93DF93CDB7DEB762970FB6F89483
:10C4D000DEBF0FBECDBF8C0161E47CE08CEB94E14C
:10C4E0000E94E2C50830110509F011C161EE70E14A
:10C4F000CE0101960E94F9C844E650E06FEF7FEF4D
:10C50000CE0101960E94FD19CE0101960E949FC89E
:10C5100065ED70E1CE0101960E94F9C844E650E055
:10C5200070E060E0CE0101960E946313CE01019697
:10C530000E949FC88BEA9FE00E94BDAC4CE251E094
:10C5400061E070E0CE0107960E9462C980917E0E84
:10C550008823D1F066EB78E0CE0101960E940BC9EA
:10C56000BE01695F7F4FCE0101960E947CC769EBD7
:10C5700078E00E9466C7BC0182E891E10E94A8D1E0
:10C58000CE0101960E949FC86DEE77E0CE01019624
:10C590000E940BC9BE016F5F7F4FCE0107960E94BC
:10C5A0004BC7182FCE0101960E949FC8112309F492
:10C5B00091C06BEB78E08CEB94E10E94E2C588E0DF
:10C5C00090E09093F10D8093F00D6CEB74E1CE014F
:10C5D00001960E9402C9CE0101960E94D584182FAF
:10C5E000CE0101960E949FC868EC70E1CE010196D1
:10C5F0000E94F9C844E650E070E060E0CE01019688
:10C600000E946313CE0101960E949FC88BEA9FE0AF
:10C610000E94BDAC48E552E061E070E0CE010196B9
:10C620000E9462C9BE016F5F7F4FCE0107960E94D4
:10C630005AC8CE0101960E949FC880917E0E882321
:10C64000D1F066EB78E0CE0101960E940BC9BE01E5
:10C65000695F7F4FCE0101960E947CC769EB78E04D
:10C660000E9466C7BC0182E891E10E94A8D1CE0178
:10C6700001960E949FC86EE778E0CE0101960E9465
:10C680000BC9BE016F5F7F4FCE0107960E944BC75B
:10C69000082FCE0101960E949FC80023D9F060ECBC
:10C6A00078E08CEB94E10E94E2C56CEB74E1CE0182
:10C6B00001960E9402C9CE0101960E94D584082FDE
:10C6C000CE0101960E949FC8002321F06BEB70E120
:10C6D000111102C064EB70E1CE0101960E94F9C80D
:10C6E00044E650E070E060E0CE0101960E946313E2
:10C6F000CE0101960E949FC861E47CE08CEB94E13E
:10C700000E94E2C5CE0107960E949FC864C5093FFA
:10C710002FEF120709F025C16AEA70E1CE010196F8
:10C720000E94F9C844E650E06FEF7FEFCE0101961A
:10C730000E94FD19CE0101960E949FC86CE970E12C
:10C74000CE0101960E94F9C844E650E070E060E036
:10C75000CE0101960E946313CE0101960E949FC8EC
:10C760008BEA9FE00E94BDAC4CE251E064E070E0D7
:10C77000CE0101960E9462C980917E0E8823D1F07D
:10C7800066EB78E0CE0107960E940BC9BE016F5F91
:10C790007F4FCE0107960E947CC769EB78E00E942C
:10C7A00066C7BC0182E891E10E94A8D1CE0107963C
:10C7B0000E949FC870E060E0CE0101960E943AC7D7
:10C7C000082E000C990BC0970A9708F0AFC066ECD2
:10C7D00078E0CE0107960E940BC9BE016F5F7F4FC4
:10C7E000CE0107960E947CC7BC018CEB94E10E94AD
:10C7F00043C8CE0107960E949FC889EF9FEF909390
:10C80000F10D8093F00D6CEB74E1CE0107960E9460
:10C8100002C9CE0107960E94D584182FCE01079633
:10C820000E949FC86EE870E1CE0107960E94F9C889
:10C8300044E650E070E060E0CE0107960E9463138A
:10C84000CE0107960E949FC88BEA9FE00E94BDAC74
:10C8500048E552E065E070E0CE0107960E9462C9AB
:10C86000BE01695F7F4FCE0101960E945AC8CE017A
:10C8700007960E949FC880917E0E8823D1F066EBB8
:10C8800078E0CE0107960E940BC9BE016F5F7F4F13
:10C89000CE0107960E947CC769EB78E00E9466C7CC
:10C8A000BC0182E891E10E94A8D1CE0107960E94C6
:10C8B0009FC870E060E0CE0101960E943AC7082E42
:10C8C000000C990BC0970A9788F56BEC78E0CE01C5
:10C8D00007960E940BC9BE016F5F7F4FCE0107967E
:10C8E0000E947CC7BC018CEB94E10E9443C8CE013E
:10C8F00007960E949FC889EF9FEF9093F10D809358
:10C90000F00D6CEB74E1CE0107960E9402C9CE01D6
:10C9100007960E94D584082FCE0107960E949FC8D3
:10C92000002321F061E870E1111102C06AE770E1B3
:10C93000CE0107960E94F9C844E650E070E060E03E
:10C94000CE0107960E946313CE0107960E949FC8EE
:10C9500061E47CE08CEB94E10E94E2C5CE0101969B
:10C96000D3CE60E770E1CE0101960E94F9C844E69B
:10C9700050E06FEF7FEFCE0101960E94FD19CE01CE
:10C9800001960E949FC861E47CE08CEB94E10E94D8
:10C99000E2C5053F8FEF1807B9F460ED78E08CEB46
:10C9A00094E10E94E2C566E670E1CE0101960E9424
:10C9B000F9C844E650E06FEF7FEFCE0101960E9488
:10C9C0006313CE01019648C1063F9FEF190749F452
:10C9D00064ED78E08CEB94E10E94E2C56CE570E1D7
:10C9E000E4CF013FEFEF1E0749F46AED78E08CEBEE
:10C9F00094E10E94E2C56DE470E1D7CF023FFFEF02
:10CA00001F0749F460EE78E08CEB94E10E94E2C5E8
:10CA10006DE370E1CACF033F2FEF120709F085C025
:10CA200061E370E1CE0101960E94F9C844E650E04E
:10CA30006FEF7FEFCE0101960E94FD19CE010196A6
:10CA40000E949FC863E270E1CE0101960E94F9C87E
:10CA500044E650E06FEF7FEFCE0101960E94631332
:10CA6000CE0101960E949FC844EF51E062E070E061
:10CA7000CE0101960E9462C9BE016F5F7F4F8CEBB1
:10CA800094E10E945AC8CE0101960E949FC86CEEA4
:10CA900078E0CE0101960E940BC96CEB74E1CE01E7
:10CAA00001960E947CC7BC018CEB94E10E9443C8B4
:10CAB000CE0101960E949FC88091C0149091C1142C
:10CAC000892B09F488C36CEB74E1CE0101960E94B6
:10CAD00002C9CE0101960E94D584F82ECE0101969E
:10CAE0000E949FC868EC70E080E090E0FF2009F4AD
:10CAF00081C30E94086E6EEE7EE0CE0101960E9418
:10CB0000F9C844EF51E06FEF7FEFCE0101960E942C
:10CB10006313CE0101960E949FC81093F10D0093FC
:10CB2000F00DC8010E94994E56C30230110509F05C
:10CB300096C067E170E1CE0101960E94F9C844E613
:10CB400050E06FEF7FEFCE0101960E94FD19CE01FC
:10CB500001960E949FC867E070E1CE0101960E9495
:10CB6000F9C844E650E06FEF7FEFCE0101960E94D6
:10CB70006313CE0101960E949FC844EF51E066E026
:10CB800070E0CE0101960E9462C9BE016F5F7F4FC7
:10CB90008CEB94E10E945AC8CE0101960E949FC876
:10CBA0008091C0149091C1140597B0F070E060E0DE
:10CBB0008CEB94E10E943AC7082E000C990BC097A9
:10CBC0000A9750F48CEB94E10E945FC66135E3EC68
:10CBD0007E0781059105CCF469EF7FE0CE010196D7
:10CBE0000E94F9C848EE53E06FEF7FEFCE01019647
:10CBF0000E946313CE0101960E949FC861E47CE00D
:10CC00008CEB94E10E94E2C557CF0E94CBE020E07C
:10CC100030E048EC52E40E9443E3AB01BC0122E067
:10CC2000CE0107960E94A7C862EC79E0CE0101967A
:10CC30000E940BC9BE01695F7F4FCE0101960E9421
:10CC40007CC7BC018CEB94E10E9443C8CE010196E5
:10CC50000E949FC8CE0107960E949FC82DCFC80191
:10CC6000C796059708F05BC08EEC9FEF7C01E01A39
:10CC7000F10AC70189569B4F6C01FC0180818A3003
:10CC8000C8F569EE7FE0CE0101960E94F9C844E63E
:10CC900050E06FEF7FEFCE0101960E94FD19CE01AB
:10CCA00001960E949FC88BE0F6018083B701CE01F8
:10CCB00007960E9419C664EB7AE0CE0101960E94A5
:10CCC0000BC9BE01695F7F4FCE0101960E947CC7F0
:10CCD000BC01CE010D960E9402C944E650E06FEF00
:10CCE0007FEFCE010D960E946313CE010D960E9438
:10CCF0009FC8ACCF68ED7FE0CE0101960E94F9C8D5
:10CD000044E650E06FEF7FEFCE0101960E94FD19DF
:10CD1000CE0101960E949FC8F6011082C7CF083C41
:10CD2000FFEF1F0709F0A0C06EEC7FE0CE01019677
:10CD30000E94F9C844E650E06FEF7FEFCE01019604
:10CD40000E94FD19CE0101960E949FC861EC7FE010
:10CD5000CE0101960E94F9C844E650E06FEF7FEFE4
:10CD6000CE0101960E946313CE0101960E949FC8D6
:10CD700063EF78E0CE0101960E940BC9CE010196C7
:10CD80000E94D584CE0101960E949FC863EB7FE08C
:10CD9000CE0101960E94F9C844E650E06FEF7FEFA4
:10CDA000CE0101960E94FD19CE0101960E949FC8F6
:10CDB00067EA7FE0CE0101960E94F9C844E650E0A0
:10CDC0006FEF7FEFCE0101960E946313CE010196B3
:10CDD0000E949FC844EF51E061E070E0CE010196EF
:10CDE0000E9462C9BE016F5F7F4F8CEB94E10E948D
:10CDF0005AC8CE0101960E949FC88091C01490919C
:10CE0000C114892BA9F070E060E08CEB94E10E94E2
:10CE10003AC7082E000C990BC0970A9748F48CEB80
:10CE200094E10E945FC662307105810591051CF096
:10CE30006BE97FE0D3CE68EF78E0CE0101960E94E7
:10CE40000BC9CE0101960E94D584CE0101960E94A5
:10CE50009FC86DEF78E0CE0101960E940BC9CE010C
:10CE600001960E94D584ADCD073C2FEF120709F043
:10CE70000BC161E97FE0CE0101960E94F9C844E64A
:10CE800050E06FEF7FEFCE0101960E94FD19CE01B9
:10CE900001960E949FC864E87FE0CE0101960E943F
:10CEA000F9C844E650E06FEF7FEFCE0101960E9493
:10CEB0006313CE0101960E949FC862E079E0CE0123
:10CEC00001960E940BC9CE0101960E94D584CE0125
:10CED00001960E949FC866E77FE0CE0101960E94FE
:10CEE000F9C844E650E06FEF7FEFCE0101960E9453
:10CEF000FD19CE0101960E949FC868E67FE0CE0131
:10CF000001960E94F9C844E650E06FEF7FEFCE0132
:10CF100001960E946313CE0101960E949FC861E4AE
:10CF20007CE08CEB94E10E94E2C5F12CE12C44EF13
:10CF300051E061E070E0CE0101960E9462C9BE013D
:10CF40006F5F7F4F8CEB94E10E945AC8CE0101962F
:10CF50000E949FC88091C0149091C114892BA9F0A0
:10CF600070E060E08CEB94E10E943AC7082E000C60
:10CF7000990BC0970A9748F48CEB94E10E945FC626
:10CF80006230710581059105CCF16CE57FE0CE0141
:10CF900001960E94F9C848EE53E06FEF7FEFCE0193
:10CFA00001960E946313CE0101960E949FC86EE411
:10CFB0007FE0CE0101960E94F9C844E650E06FEF91
:10CFC0007FEFCE0101960E946313CE0101960E946D
:10CFD0009FC861E47CE08CEB94E10E94E2C58FEF96
:10CFE000E81AF80A64E670E080E090E00E94086EBB
:10CFF0009EE1E916F1040CF49ACF5ECD67E079E08A
:10D00000CE0101960E940BC9CE0101960E94D584E3
:10D01000CE0101960E949FC88CEB94E10E945FC6EE
:10D02000672B682B692BA1F460E47FE0CE010196A9
:10D030000E94F9C844E650E06FEF7FEFCE01019601
:10D040000E94FD19CE0101960E949FC8F12CE12C8F
:10D050008CEB94E10E945FC66130710581059105FA
:10D0600009F0BDCF6CE079E0CE0101960E940BC9BA
:10D07000CE0101960E94D584CE0101960E949FC8E0
:10D080008FE1E82EF12CABCF063CEFEF1E07D9F570
:10D0900066E37FE0CE0101960E94F9C844E650E0C5
:10D0A0006FEF7FEFCE0101960E94FD19CE01019630
:10D0B0000E949FC869E27FE0CE0101960E94F9C8F4
:10D0C00044E650E06FEF7FEFCE0101960E946313BC
:10D0D000CE0101960E949FC861E179E0CE010196E0
:10D0E0000E940BC9CE0101960E94D584CE01019603
:10D0F0000E949FC860ED77E080E090E00E94086E9B
:10D1000068E179E0A8CE0630110509F047C069E171
:10D110007FE0CE0101960E94F9C844E650E06FEF2F
:10D120007FEFCE0101960E94FD19CE0101960E946B
:10D130009FC86CE07FE0CE0101960E94F9C844E6EA
:10D1400050E06FEF7FEFCE0101960E946313CE0196
:10D1500001960E949FC86FE179E0CE0101960E947E
:10D160000BC9CE0101960E94D584CE0101960E9482
:10D170009FC864E670E080E090E00E94086E61E085
:10D180007FE0CE0101960E94F9C844E650E06FEFBF
:10D190007FEFCE0101960E94FD1913CC68EF7EE06F
:10D1A000CE0101960E94F9C844E650E06FEF7FEF90
:10D1B000CE0101960E946313CE0101960E949FC882
:10D1C00061E47CE08CEB94E10E94E2C50B3EFFEF52
:10D1D0001F0709F071CC62960FB6F894DEBF0FBE40
:10D1E000CDBFDF91CF911F910F91FF90EF90DF9016
:10D1F000CF9008950E94086E62EE7EE0CE01019607
:10D200000E94F9C844EF51E06FEF7FEFCE01019625
:10D210000E946313A3CB4F925F926F927F928F9283
:10D220009F92AF92BF92EF92FF920F931F93CF9373
:10D23000DF93CDB7DEB762970FB6F894DEBF0FBEAF
:10D24000CDBF7C015B0181ED9CE00E9474B6892B0F
:10D25000D9F461E47CE0C7010E940BC9C701629662
:10D260000FB6F894DEBF0FBECDBFDF91CF911F91F7
:10D270000F91FF90EF90BF90AF909F908F907F9015
:10D280006F905F904F9008954091D50C5091D60CBF
:10D290006091D70C7091D80CCE0107960E94A01A0D
:10D2A00080917E0E882359F166E279E0CE010196E5
:10D2B0000E940BC9BE01695F7F4FCE0101960E949B
:10D2C0007CC760E677E00E9466C7BC0182E891E116
:10D2D0000E949AD1CE0101960E949FC84091D50C20
:10D2E0005091D60C6091D70C7091D80C20E182E857
:10D2F00091E10E9404CB82E891E10E9450CB70E062
:10D3000060E0CE0107960E943AC7182F8A3211F0CA
:10D3100010929D0D0E943B6E6093750E7093760E79
:10D320008093770E9093780E61E47CE0CE010D96A9
:10D330000E940BC9812F110F990BC0970A9708F013
:10D3400068C0CE0107960E945FC6633071058105F3
:10D3500091050CF084C001E010E082E0982E0A15DF
:10D360001B0509F47CC06CE271E080E090E00E9453
:10D37000086E90921F1210922212412C512C3201F1
:10D3800081EC9CE00E9474B6892B91F48EE14816E2
:10D3900051046104710449F16EE170E080E090E0B5
:10D3A0000E94086E8FEF481A580A680A780AE8CF78
:10D3B0008EE14816510461047104B9F04091C50C26
:10D3C0005091C60C6091C70C7091C80CCE010196AB
:10D3D0000E94A01ABE016F5F7F4FCE010D960E9482
:10D3E0005AC8CE0101960E949FC889899A89892BC3
:10D3F00039F0BE01635F7F4FCE0107960E9417C8C8
:10D400000F5F1F4F61E47CE0CE010D960E94E2C5E4
:10D41000A6CF6CE271E080E090E00E94086E82E0AE
:10D4200080931F1210922212812C912C540181ECB6
:10D430009CE00E9474B6892B61F58EE188169104F8
:10D44000A104B10409F043C089899A89892B39F074
:10D45000BE01635F7F4FCE0107960E9417C864E646
:10D4600070E080E090E00E94086E82E080931F12DE
:10D4700010922212BE01695F7F4FC7010E94F0C85F
:10D48000CE010D960E949FC8CE0107960E949FC8AC
:10D49000E5CE8EE188169104A104B104A9F2409171
:10D4A000C50C5091C60C6091C70C7091C80CCE0190
:10D4B00001960E94A01ABE016F5F7F4FCE010D96AC
:10D4C0000E945AC8CE0101960E949FC8BDCF6EE14E
:10D4D00070E080E090E00E94086E8FEF881A980A52
:10D4E000A80AB80AA4CFAF92BF92CF92DF92EF9270
:10D4F000FF920F931F93CF93DF93CDB7DEB72C9797
:10D500000FB6F894DEBF0FBECDBF7C015B010E9459
:10D510002DB5182F811117C061E47CE0C7010E946E
:10D520000BC9C7012C960FB6F894DEBF0FBECDBF56
:10D53000DF91CF911F910F91FF90EF90DF90CF90EF
:10D54000BF90AF9008958A3211F010929D0D0E9405
:10D550003B6E6093750E7093760E8093770E90936A
:10D56000780E612FCE0107960E94D7C8812F012E19
:10D57000000C990BC0970A9768F5CE0107960E9498
:10D580005FC663307105810591050CF070C001E044
:10D5900010E00A151B0509F46AC062E370E080E040
:10D5A00090E00E94086E0E942DB5D12CC12C8111F3
:10D5B0003BC08FEFC81AD80A85E1C816D10409F418
:10D5C00056C06EE170E080E090E00E94086E0E941C
:10D5D0002DB5EDCF612FCE0101960E94D7C8BE01B7
:10D5E0006F5F7F4FCE0107960E945AC8CE01019609
:10D5F0000E949FC862E370E080E090E00E94086EA5
:10D600000E942DB510E000E0811121C00F5F1F4F77
:10D610000F31110561F16EE170E080E090E00E9451
:10D62000086E0E942DB5F0CF682FCE0101960E94A2
:10D63000D7C8BE016F5F7F4FCE0107960E9417C803
:10D64000CE0101960E949FC80F5F1F4FA2CF682F87
:10D65000CE0101960E94D7C8BE016F5F7F4FCE01F9
:10D6600007960E9417C8CE0101960E949FC8BE016E
:10D67000695F7F4FC7010E94F0C8CE0107960E94E4
:10D680009FC84FCF8FEF9AEA892B49F080E090E056
:10D69000892B29F00E94FFAA81110E94000085EFCA
:10D6A0009AEA892B49F080E090E0892B29F00E94CA
:10D6B000F5AA81110E9400008BEE9AEA892B49F0AD
:10D6C00080E090E0892B29F00E94EBAA81110E9452
:10D6D000000081EE9AEA892B49F080E090E0892BE6
:10D6E00029F00E94E1AA81110C9400000895815054
:10D6F000823108F05AC0E82FF0E08827ED57F4494E
:10D700008F4F0C94EFE5A36BA76B956B9B6B9F6B97
:10D71000D56BAA6BB06BB46BBA6BBE6BC26BC86BCC
:10D72000CC6BD56BD06BD66BDA6B809180008F772A
:10D73000809380000895809180008F7DF9CF809143
:10D740008000877FF5CF84B58F7784BD089584B539
:10D750008F7DFBCF8091B0008F778093B0000895CC
:10D760008091B0008F7DF9CF809190008F7780936A
:10D7700090000895809190008F7DF9CF8091900066
:10D78000877FF5CF8091A0008F778093A0000895C8
:10D790008091A0008F7DF9CF8091A000877FF5CF89
:10D7A000809120018F77809320010895809120013E
:10D7B0008F7DF9CF80912001877FF5CFDC0180E05C
:10D7C000615090F09D919827E92FEF70F0E0E459B7
:10D7D000F34E2491E92FE295EF70F0E0E458F34E18
:10D7E000E491822F8E27ECCF08958091080F9091BD
:10D7F000090F891B990B08952091470E260F332797
:10D80000331F21323105ECF42091820FFC0190E0AE
:10D8100080E0243069F082E00895A091470E2191C4
:10D82000AC01495D514FA40FB52FB11D2C9301964A
:10D83000861798F38091470E680F6093470E80E03B
:10D84000089581E00895089508950895E091090FDD
:10D850008091080FE81730F4F0E0E851F14F808133
:10D8600090E008958FEF9FEF08959091090F8091B8
:10D87000080F2FEF3FEF981748F4E92FF0E0E85139
:10D88000F14F208130E09F5F9093090FC901089507
:10D89000CF92DF92EF92FF920F931F93CF93DF937C
:10D8A0007C01CB018A012091880F222389F0EB01B2
:10D8B0006B01C40ED51ECC15DD0569F06991D70149
:10D8C000ED91FC910190F081E02DC7011995F3CF06
:10D8D000642F0E94FC6BC801DF91CF911F910F91C3
:10D8E000FF90EF90DF90CF900895CF93DF931F923A
:10D8F000CDB7DEB769832091880F2223F9F02091FC
:10D90000AA0F203258F021E030E0FC01338322835B
:10D9100090E080E00F90DF91CF9108958091890F82
:10D92000E82FF0E0E657F04F998190838F5F809366
:10D93000890F8093AA0F81E090E0ECCF61E0CE01E7
:10D9400001960E94FC6BF7CF90E080E008950C9464
:10D95000DDE6E1EFF2E114A215A216A217A210A6CD
:10D9600011A612A613A681E084A729E130E036A70C
:10D9700025A787A780E090E0A0EAB0E480AB91AB58
:10D98000A2ABB3AB80E090E0A8EAB1E484AB95AB86
:10D99000A6ABB7AB8093F6049093F704A093F8047A
:10D9A000B093F90480E090E0A0E8BFE380933B13DC
:10D9B00090933C13A0933D13B0933E138093F204D5
:10D9C0009093F304A093F404B093F50410926813B9
:10D9D000109267138BE090E090936A138093691321
:10D9E0009093F1048093F0041092781310927713BF
:10D9F000109288131092871390E080E00C9471B01D
:10DA0000FC01A48DA80FB92FB11DA35ABF4F2C91B3
:10DA1000848D90E001968F739927848FA689B789AA
:10DA20002C93A089B1898C91837080648C93938DA1
:10DA3000848D981306C00288F389E02D80818F7D44
:10DA400080830895CF93DF93282F30E0F901EA59BE
:10DA5000F24E8491F901E05EF24ED491F901E65262
:10DA6000F34EC491CC23A1F081110E94776BEC2F6F
:10DA7000F0E0EE0FFF1FE054F34EA591B491EC914E
:10DA8000ED2381E090E009F480E0DF91CF910895EB
:10DA900080E090E0FACF862F0C94226D1F93CF93F5
:10DAA000DF93282F30E0F901EA59F24E8491F90111
:10DAB000E05EF24ED491F901E652F34EC491CC23CC
:10DAC000A9F0162F81110E94776BEC2FF0E0EE0F7A
:10DAD000FF1FEA55F34EA591B4918FB7F894EC91DE
:10DAE000111108C0D095DE23DC938FBFDF91CF9159
:10DAF0001F910895DE2BF8CF862F642F0C944E6D66
:10DB0000CF93DF9390E0FC01E05EF24E24918652C9
:10DB1000934EFC0184918823C9F090E0880F991FEF
:10DB2000FC01E457F34EA591B491FC01EA55F34E84
:10DB3000C591D49161110DC09FB7F8948C91209537
:10DB400082238C938881282328839FBFDF91CF91E4
:10DB50000895623051F49FB7F8943C91822F8095DC
:10DB600083238C93E8812E2BEFCF8FB7F894EC9121
:10DB70002E2B2C938FBFEACF862F642F0C94806DB1
:10DB8000863308F0865320917B00982F9870277F6A
:10DB9000922B90937B002091FA0490E4299F9001AE
:10DBA00011248770822B80937C0080917A0080649E
:10DBB00080937A0080917A0086FDFCCF8091780076
:10DBC0009091790008953FB7F89480916F0E9091ED
:10DBD000700EA091710EB091720E26B5A89B05C073
:10DBE0002F3F19F00196A11DB11D3FBFBA2FA92FDC
:10DBF000982F8827BC01CD01620F711D811D911DD9
:10DC000042E0660F771F881F991F4A95D1F7089544
:10DC10008F929F92AF92BF92CF92DF92EF92FF923C
:10DC20006B017C010E94E36D4B015C01C114D104C6
:10DC3000E104F104B9F00E94E36D681979098A09D9
:10DC40009B09683E73408105910580F321E0C21A6B
:10DC5000D108E108F10888EE880E83E0981EA11C27
:10DC6000B11CE4CFFF90EF90DF90CF90BF90AF90CA
:10DC70009F908F9008952FB7F89460916B0E7091DC
:10DC80006C0E80916D0E90916E0E2FBF08951F92B5
:10DC90000F920FB60F9211242F933F938F939F9360
:10DCA000AF93BF9380916B0E90916C0EA0916D0E0F
:10DCB000B0916E0E30916A0E23E0230F2D3758F588
:10DCC0000196A11DB11D20936A0E80936B0E909357
:10DCD0006C0EA0936D0EB0936E0E80916F0E9091AE
:10DCE000700EA091710EB091720E0196A11DB11D22
:10DCF00080936F0E9093700EA093710EB093720E7E
:10DD0000BF91AF919F918F913F912F910F900FBE37
:10DD10000F901F90189526E8230F0296A11DB11DA4
:10DD2000D2CF0C94EBE10895DF92EF92FF920F9324
:10DD30001F93CF93DF937C018B01D42EDC011696C9
:10DD4000ED91FC9113861586148612861186108635
:10DD500017821682158214821382C0E0B801F7017F
:10DD6000868197810E9441C3D82F882329F0DC1631
:10DD700029F0CF5FDC1690F7D0E009C067E0C8015A
:10DD80000E94DE6BD80117969C918913F2CF8D2FDC
:10DD9000DF91CF911F910F91FF90EF90DF90089549
:10DDA000DC012C911196ED91FC91F8948181822BEC
:10DDB00081839281322F30959323928387E090E084
:10DDC0000197F1F781818323818383E290E00197BA
:10DDD000F1F790817894EFECF0E03197F1F792232E
:10DDE00081E009F480E00895FC0190810180F281D6
:10DDF000E02D292F209560FF14C0F89482818223A2
:10DE000082838181892B8183A3E2B0E01197F1F7AE
:10DE10008281982B9283789487ED90E00197F1F7B7
:10DE20000895F8948281822382838181892B818362
:10DE3000AFEFB0E01197F1F78281982B928378943D
:10DE40008FE090E0EBCFDF92EF92FF920F931F9362
:10DE5000CF93DF93EC01D62EE42E08E010E0FF24F0
:10DE6000F39461E08D2D8F2109F460E0CE010E94D2
:10DE7000F46EFF0C01501109A1F7E11010C0F894E5
:10DE8000E981FA8191818881809589238183E98163
:10DE9000FA81928188818095892382837894DF91A9
:10DEA000CF911F910F91FF90EF90DF900895EF9227
:10DEB000FF920F931F93CF93DF938C017B0140E080
:10DEC00065E50E94236FE70188E0E80EF11C699187
:10DED00040E0C8010E94236FCE15DF05C1F7DF9136
:10DEE000CF911F910F91FF90EF900895FC019081C9
:10DEF0000180F281E02DF8948181292F20958223E1
:10DF0000818378943DE743E050E0315029F1DA0114
:10DF10001197F1F780818923C1F3F89482818223DC
:10DF200082838181892B81837894ABE7B7E0119755
:10DF3000F1F7F894818182238183A3E1B1E0119705
:10DF4000F1F78081982381E009F080E07894E3E69E
:10DF5000F6E03197F1F7089580E008958F929F924F
:10DF6000AF92BF92CF92DF92EF92FF92CF93DF9367
:10DF7000EC018E819F810E94766F40E06CEC8E8177
:10DF80009F810E94236F488164E48E819F810E945B
:10DF9000236F8A81882371F1E981E9508EEEC82EC2
:10DFA00082E0D82EE33038F4F0E0EE0FFF1FED579B
:10DFB000FA4FC080D1808B81882339F1888181110B
:10DFC00024C00E943B6E4B015C010D2C000CEE083E
:10DFD000FF088E819F810E94D06E813059F00E948F
:10DFE0003B6E6C197D098E099F09681579058A05B4
:10DFF0009B0578F3DF91CF91FF90EF90DF90CF906A
:10E00000BF90AF909F908F900895B601DD0C880B64
:10E01000990BDF91CF91FF90EF90DF90CF90BF9061
:10E02000AF909F908F900C94086E6F927F928F921A
:10E030009F92AF92BF92CF92DF92EF92FF920F9397
:10E040001F93CF93DF93EC017B018A018E819F8127
:10E050000E94766F811102C090E037C0B7018E81B7
:10E060009F810E94576F40E06EEB8E819F810E94DE
:10E07000236F7801680189E0C80ED11CAE80BF8093
:10E0800088E0882E912C712C66246394C5010E942F
:10E09000D06E81117628660CE1E08E1A9108B1F7F6
:10E0A000F70171927F01EC15FD0541F78E819F818B
:10E0B0000E94766F813081F668E0C8010E94DE6BB5
:10E0C00091E0F80120852813C7CF892FDF91CF91E8
:10E0D0001F910F91FF90EF90DF90CF90BF90AF9086
:10E0E0009F908F907F906F900895CF93DF9300D093
:10E0F00000D000D0CDB7DEB7AE014F5F5F4F0E94BA
:10E100001570882331F08D818F33A9F020F48F3181
:10E11000A1F080E007C08F3521F08F37D1F78CE078
:10E1200001C08BE029960FB6F894DEBF0FBECDBFBD
:10E13000DF91CF9108958AE0F5CF89E0F3CF0F9377
:10E140001F93CF93DF93CDB7DEB761970FB6F894E7
:10E15000DEBF0FBECDBF8C01462FBE01665F7F4F75
:10E160000E94946E81110FC060E070E08EEF92EC1F
:10E1700061960FB6F894DEBF0FBECDBFDF91CF9191
:10E180001F910F910895AE014F5F5F4FBE01665F13
:10E190007F4FC8010E941570882331F36A8170E0B7
:10E1A000762F6627770F770F770F298148E0249F16
:10E1B00090011124262B372B8A858031D1F4688574
:10E1C00070E08F81AB01481B5109CA019695982FC9
:10E1D0008827979587950E94DBE5CB014097B90189
:10E1E00053E0660F771F5A95E1F760789C01260F80
:10E1F000371F213854EE35070CF4B6CFB901330F71
:10E20000880B990B0E94CBE020E030E040E05CE31B
:10E210000E942AE1ADCFEF92FF920F931F93CF930D
:10E22000DF9300D000D01F921F92CDB7DEB78C01D4
:10E23000DC011696ED91FC911797138615861486CE
:10E240001286118610861782168215821482138216
:10E2500014961C92149715961C92EE24E394BE011A
:10E260006F5F7F4FF801868197810E9441C38823A9
:10E2700009F46FC067E0CE0101960E94DE6B9885BD
:10E280008913EDCFD8018C91811125C016968D91FF
:10E290009C910E94766FBE016F5F7F4FF80186816F
:10E2A00097810E94576F40E064EBD80116968D91DC
:10E2B0009C910E94236FF801868197810E94D06E05
:10E2C000F82ED80116968D919C910E94766FF110D0
:10E2D00002C0F801E082D8011196FC90898180315A
:10E2E000A1F1BE016F5F7F4FC8010E9475708F154D
:10E2F000D0F4F8018181D80111968C93119714966E
:10E300008C9114978F5F14968C938981883231F0A9
:10E31000B0F4803119F0823209F0A1CFF801858183
:10E320008F5F85839CCF8981803111F48CE0E3CFAE
:10E33000BE016F5F7F4FC8010E947570DCCF8B33C9
:10E3400069F3823409F08BCFE9CFFCE0FF1588F246
:10E35000EDCF28960FB6F894DEBF0FBECDBFDF918C
:10E36000CF911F910F91FF90EF9008951F93CF933E
:10E37000DF93EC01162F60E0812F0E94806D612FEA
:10E3800070E0FB01E05EF24EE491E883FB01E652AF
:10E39000F34EE491F0E0EE0FFF1FE054F34E859151
:10E3A00094919A8389831B861D861C861A861986FA
:10E3B00018861F821E821D821C821B82DF91CF91D4
:10E3C0001F9108951F920F920FB60F9211240BB652
:10E3D0000F922F933F934F935F936F937F938F93FE
:10E3E0009F93AF93BF93EF93FF93809120120E946E
:10E3F000226D20912312309124122F5F3F4F3093D2
:10E4000024122093231290912212953618F096E050
:10E4100090931F1290911F12943009F46EC0F8F47B
:10E42000923031F1933009F44CC09091211299232C
:10E4300019F0811171C02F9AFF91EF91BF91AF91A7
:10E440009F918F917F916F915F914F913F912F910C
:10E450000F900BBE0F900FBE0F901F901895953028
:10E4600009F457C0963009F791E09093EF124FC02E
:10E470008111DBCF209123123091241224363105F3
:10E4800028F41092241210922312CFCF1092EF1280
:10E4900010922212E091221291E09E0F909322128C
:10E4A000F0E02091231230912412EE0FFF1FEB5D5C
:10E4B000FD4E31832083109224121092231293E098
:10E4C00019C0813009F0B1CFE091221291E09E0F86
:10E4D00090932212F0E02091231230912412EE0F3B
:10E4E000FF1FEB5DFD4E31832083109224121092AA
:10E4F000231294E090931F1298CF882359F2209111
:10E500002312309124122536310508F48ECF95E080
:10E51000F1CF81118ACFB5CF2F988ECFCF92DF92D6
:10E52000EF92FF92CF93DF93EC01072E000C880B44
:10E53000990B0E94CBE06B017C0120E030E040E4CD
:10E540005FE30E942AE120E030E048E452E40E94C8
:10E5500043E30E94EFE3C617D707D4F020E030E092
:10E5600040EA5FE3C701B6010E942AE120E030E003
:10E5700048E452E40E9443E320E030E040E85FE3F7
:10E580000E9465E20E94EFE321E06C177D070CF426
:10E5900020E0822F90E0DF91CF91FF90EF90DF900D
:10E5A000CF9008950F931F93CF93DF93082F6EE7BB
:10E5B00078E082E891E10E94C4CCC7E0D0E010E0AE
:10E5C000B8010C2E02C0759567950A94E2F7617048
:10E5D000772742E050E082E891E10E9477CC2197D2
:10E5E00078F7DF91CF911F910F9108951092820FCC
:10E5F00081E08093810F10925C0F61E084E10E94C2
:10E600004E6D61E085E10E944E6DE9EBF0E08081A6
:10E610008E7F808380818D7F808388E48093B800A3
:10E6200085E48093BC000895CF93DF9391E09093AD
:10E63000260E8823B9F0C091B800D091BA0080911D
:10E64000BC008A7B8093BC0060E084E10E944E6D38
:10E6500060E085E10E944E6D0E94F672D093BA0090
:10E66000C093B800DF91CF91089585ED8093BC00F1
:10E670008091840F9091850FA091860FB091870FA4
:10E680000796A11DB11D23E0B695A795979587958F
:10E690002A95D1F72091BC0024FD03C01092820F6F
:10E6A00008954091840F5091850F6091860F70916D
:10E6B000870F452B462B472B69F30097A105B10522
:10E6C00041F025E32A95F1F700000197A109B1096E
:10E6D000E1CF8091830F0C9414731F920F920FB6A9
:10E6E0000F9211240BB60F922F933F934F935F938A
:10E6F0006F937F938F939F93AF93BF93EF93FF930A
:10E700008091B900887F803609F44DC008F040C080
:10E71000883209F4A9C028F5803109F49DC0C8F4F5
:10E72000882309F4FBC0883009F496C0FF91EF916B
:10E73000BF91AF919F918F917F916F915F914F9119
:10E740003F912F910F900BBE0F900FBE0F901F9017
:10E750001895883109F488C0803241F78093800F82
:10E7600014C0803409F49DC040F48033B9F3883379
:10E77000E9F68093800F85ECB0C0803509F485C040
:10E78000883509F496C0883489F60E943573CECF57
:10E79000883909F48CC038F5883729F050F4883668
:10E7A00011F0803719F683E08093820F1092690E82
:10E7B00057C0883809F47BC0803919F0803809F0D7
:10E7C000B5CF8091690E803208F071C0E091690E7A
:10E7D00081E08E0F8093690E8091BB00F0E0E75BD3
:10E7E000F14F80833DC0803B39F0E0F4803A09F47A
:10E7F00079C0883A09F09ACF84E08093820F109212
:10E80000480E1092470EE091810EF091820E1995FC
:10E810008091470E81110FC081E08093470E1092C6
:10E82000270E09C0803C09F4A6CF883C09F4A3CF89
:10E83000883B09F07BCFE091480E81E08E0F8093FA
:10E84000480EF0E0E95DF14F80818093BB0090912C
:10E85000480E8091470E29C080915D0F8093BB00C8
:10E8600085EC8093BC0062CF90917F0F80917E0FEA
:10E87000981758F5E0917F0F81E08E0F80937F0FFE
:10E88000F0E0E25AF04F8081E9CFE0917F0F81E024
:10E890008E0F80937F0F8091BB00F0E0E25AF04F23
:10E8A000808390917F0F80917E0F9817C8F285E842
:10E8B000D8CFE0917F0F81E08E0F80937F0F809102
:10E8C000BB00F0E0E25AF04F80838091810F81110C
:10E8D0005CCF81E080935C0F84EA8093BC0010924F
:10E8E000820F24CF85EC8093BC001092820F809120
:10E8F000690E803230F4E091690EF0E0E75BF14F91
:10E9000010826091690E70E0E0917F0EF091800EB0
:10E9100089E49EE019951092690E08CF1092800F3D
:10E9200034CF81E00C94DDAC0F931F93CF938C0117
:10E93000C62FFC0184810E94CDADF8016385C62BF2
:10E940006C2F70E089ED94E10E94EF1389ED94E162
:10E95000CF911F910F910C9491740F931F93CF93AC
:10E960008C01C62F0E9494746C2F6460C8010E94B1
:10E9700094746C2F6B7FC8010E94947483EC90E0B8
:10E980000197F1F7CF911F910F9108950F931F9366
:10E99000CF938C01C62F607F61600E94AD7480E1CF
:10E9A000C89FB00111246160C8010E94AD7481E06C
:10E9B00090E0CF911F910F910895862F642F0E94B0
:10E9C000DAB11092090F8093080F0895CF938EE16A
:10E9D0000E94CDAD62E070E089ED94E10E94EF13FA
:10E9E00061E870E089ED94E10E94EF1389ED94E114
:10E9F0000E94917446E050E06EE170E089ED94E190
:10EA00000E94DD748091080F9091090F891B990B6A
:10EA1000069724F10E94C7B1C82F0E94C7B120E019
:10EA2000822B9C2B9093E50E8093E40E0E94C7B13D
:10EA3000C82F0E94C7B120E0822B9C2B9093E10E3F
:10EA40008093E00E0E94C7B1C82F0E94C7B120E09A
:10EA5000822B9C2B9093E30E8093E20ECF9108952E
:10EA6000EF92FF920F931F93CF93DF93CDB7DEB753
:10EA700068970FB6F894DEBF0FBECDBF8C016EE273
:10EA800077E0CE010D960E940BC96AE379E0CE01D2
:10EA900043960E940BC96EE27AE1C8010E94F9C850
:10EAA000BE016D5E7F4FC8010E9417C865E27AE122
:10EAB000C8010E948FC788E9E82E83E1F82EF7018C
:10EAC000608170E0CE0101960E9419C6BE016F5FA1
:10EAD0007F4FCE0107960E9402C9BE01635F7F4F40
:10EAE000CE0107960E947CC7BC01C8010E9417C8CE
:10EAF000CE0107960E949FC8CE0101960E949FC832
:10EB000068E17AE1C8010E948FC7F7016181062E92
:10EB1000000C770BCE0101960E9419C6BE016F5FF3
:10EB20007F4FCE0107960E9402C9BE01635F7F4FEF
:10EB3000CE0107960E947CC7BC01C8010E9417C87D
:10EB4000CE0107960E949FC8CE0101960E949FC8E1
:10EB50006EE07AE1C8010E948FC7F7016281062E3C
:10EB6000000C770BCE0101960E9419C6BE016F5FA3
:10EB70007F4FCE0107960E9402C9BE01635F7F4F9F
:10EB8000CE0107960E947CC7BC01C8010E9417C82D
:10EB9000CE0107960E949FC8CE0101960E949FC891
:10EBA00066E07AE1C8010E948FC7F7016381748132
:10EBB000CE0101960E9419C6BE016F5F7F4FCE0144
:10EBC00007960E9402C9BE016D5E7F4FCE01079677
:10EBD0000E947CC7BC01C8010E9417C8CE010796DD
:10EBE0000E949FC8CE0101960E949FC86FEE79E1F6
:10EBF000C8010E948FC7F70165817681CE01019619
:10EC00000E9419C6BE016F5F7F4FCE0107960E941A
:10EC100002C9BE01635F7F4FCE0107960E947CC789
:10EC2000BC01C8010E9417C8CE0107960E949FC868
:10EC3000CE0101960E949FC866EE79E1C8010E944C
:10EC40008FC7F7016781062E000C770B6F5F7F4F30
:10EC5000CE0101960E9419C6BE016F5F7F4FCE01A3
:10EC600007960E9402C9BE01635F7F4FCE010796DF
:10EC70000E947CC7BC01C8010E9417C8CE0107963C
:10EC80000E949FC8CE0101960E949FC86BED79E15A
:10EC9000C8010E948FC7F7016085062E000C770B14
:10ECA000CE0101960E9419C6BE016F5F7F4FC80159
:10ECB0000E9417C8CE0101960E949FC8CE014396BC
:10ECC0000E949FC8CE010D960E949FC8C8016896F9
:10ECD0000FB6F894DEBF0FBECDBFDF91CF911F916D
:10ECE0000F91FF90EF9008954F925F926F927F92F5
:10ECF0008F929F92AF92BF92CF92DF92EF92FF924C
:10ED00000F931F93CF93DF93CDB7DEB762970FB604
:10ED1000F894DEBF0FBECDBF8EE492E00E94EBE11F
:10ED200080930A0F8FE492E00E94EBE180930B0F37
:10ED300080910A0F90910B0F1816190664F4109227
:10ED4000EF04019741F410920B0F10920A0F8EE41A
:10ED500092E00E941CB040E052EC61E070E082E87A
:10ED600091E10E9437168091EF04882331F068EE1C
:10ED700073E080E090E00E94086E82E891E10E94DA
:10ED8000B3AA182FD82EF8E9AF2EF3E1BF2EACE2CC
:10ED9000EA2EFF24F394C7010E94EBE1F501819371
:10EDA0005F01FFEFEF1AFF0A46E2E41642E0F406C5
:10EDB00091F78091991318161CF41D3609F011C1B2
:10EDC00061E47CE0CE010D960E940BC9109298136D
:10EDD00088E18093991384E080939A1310929F1393
:10EDE0001092A01362EA7BE0CE010D960E94E2C56C
:10EDF00082EA93E1009739F044E050E0BC01CE0193
:10EE00000D960E949BB081E08093A61383E08093CF
:10EE1000A71382E090E09093A9138093A81385E054
:10EE200090E09093AB138093AA136FE97BE0CE013F
:10EE30000D960E94E2C58CEA93E1009739F044E018
:10EE400050E0BC01CE010D960E949BB082E0809301
:10EE5000B01383E08093B11382E090E09093B313FA
:10EE60008093B21385E090E09093B5138093B41330
:10EE70006CE97BE0CE010D960E94E2C586EB93E142
:10EE8000009739F044E050E0BC01CE010D960E949D
:10EE90009BB083E08093BA138093BB1382E090E031
:10EEA0009093BD138093BC1385E090E09093BF13C3
:10EEB0008093BE136DE379E0CE010D960E94E2C50A
:10EEC00080EC93E1009739F044E050E0BC01CE01C2
:10EED0000D960E949BB085EF8093C41383E08093CE
:10EEE000C51382E090E09093C7138093C61385E02A
:10EEF00090E09093C9138093C8138CE291E00E9434
:10EF0000BEB080917E0E882311F1CE0101960E9441
:10EF10003075BE016F5F7F4F82E891E10E94A8D1FA
:10EF2000CE0101960E949FC86CE87AE182E891E1E7
:10EF30000E94BAD12AE04AE050E060E070E082E846
:10EF400091E10E9404CB82E891E10E9450CB62E5FE
:10EF50007AE1CE0107960E94F9C8BE01695F7F4F32
:10EF600082E891E10E94A8D1F12CE12C80919A13C2
:10EF7000082E000C990BE816F906A4F4B701CE018F
:10EF800001960E94051FBE016F5F7F4F82E891E1ED
:10EF90000E94A8D1CE0101960E949FC88FEFE81A67
:10EFA000F80AE4CFCE0107960E949FC880917E0E9A
:10EFB000882399F06CE67AE182E891E10E94BAD167
:10EFC0002AE04AEF50E060E070E082E891E10E94C0
:10EFD00004CB82E891E10E9450CBCE010D960E94B5
:10EFE0009FC88091A11381118091981380939313EE
:10EFF0000E943B6E60938F137093901380939113D4
:10F000009093921300E0123709F431C7E1EFEE2E2E
:10F01000E2E1FE2E4701B12CA12CC5010E94EBE1DB
:10F02000F40181934F01FFEFAF1ABF0A48E9A4161C
:10F03000B10499F78091F1129091F212A091F3121C
:10F04000B091F41285369105A105B1050CF4D9C132
:10F050008093EB049093EC04A093ED04B093EE0442
:10F060008091F5129091F612A091F712B091F812DA
:10F070008093E7049093E804A093E904B093EA0432
:10F080008091F9129091FA12A091FB12B091FC12AA
:10F090008093E3049093E404A093E504B093E60422
:10F0A0006DE073E1CE0101960E940BC9BE016F5F56
:10F0B0007F4F84E196E10E945AC8CE0101960E94DA
:10F0C0009FC86BE673E1CE0101960E940BC9BE0199
:10F0D0006F5F7F4F8EE096E10E945AC8CE01019685
:10F0E0000E949FC823E030E050E040E064E176E118
:10F0F000CE0107960E941CC923E030E050E040E0BA
:10F100006EE076E1CE0101960E941CC92D813E8100
:10F110008B859C852817390709F589819A816F812C
:10F120007885009759F06115710509F002C1232B0C
:10F1300009F402C1FC01808190E00DC061157105E8
:10F1400009F4FAC0232B09F4F7C0FB01808190E099
:10F1500091958195910901E0892B09F000E0CE019C
:10F1600001960E949FC8CE0107960E949FC8011178
:10F1700006C064E176E18EE096E10E9443C880918A
:10F18000FD129091FE12A091FF12B0910013809396
:10F19000DF049093E004A093E104B093E204809133
:10F1A000011390910213A0910313B0910413809363
:10F1B000DB049093DC04A093DD04B093DE04809123
:10F1C000051390910613A0910713B0910813809333
:10F1D000D7049093D804A093D904B093DA04809113
:10F1E000091390910A13A0910B13B0910C13809303
:10F1F000D3049093D404A093D504B093D604809103
:10F20000691390916A139093F1048093F0048091B4
:10F21000251390912613A0912713B0912813809362
:10F22000F6049093F704A093F804B093F904809146
:10F230003B1390913C13A0913D13B0913E138093EA
:10F24000F2049093F304A093F404B093F504809136
:10F25000151390911613A0911713B0911813809362
:10F26000CF049093D004A093D104B093D2048091A2
:10F27000191390911A13A0911B13B0911C13809332
:10F28000CB049093CC04A093CD04B093CE04A09073
:10F290007713B0907813B5010B2C000C880B990BE9
:10F2A0000E94CBE09B01AC010E94B1E5811104C03A
:10F2B000B0921D0EA0921C0E80908113909082132C
:10F2C000A0908313B0908413A5019401C501B401EB
:10F2D0000E94B1E5811132C08092C7049092C804A7
:10F2E000A092C904B092CA048091851390918613AC
:10F2F0009093C6048093C5042091B3043091B40464
:10F3000090E080E028173907A4F1F70140AD51AD36
:10F3100057FF0AC0FC01EE0FFF1FED54FB4F408169
:10F320005181F70151AF40AF0196F2E0EF0EF11CB1
:10F33000E9CF0E9488E80FCF01E011CF8091C70488
:10F340009091C804A091C904B091CA04809381131C
:10F3500090938213A0938313B093841383E090E07F
:10F36000909386138093851390E080E00E9471B0A3
:10F37000C3CF60911513709116138091171390915C
:10F3800018139B01AC010E94B1E581110FC060917F
:10F39000191370911A1380911B1390911C139B01E8
:10F3A000AC010E94B1E5882309F4BDC40E94A96C98
:10F3B0004FE3A42E43E1B42E54EFE52E5DE0F52E8D
:10F3C0006CE1862E6EE0962EF50141905190619091
:10F3D00071905F01A3019201C301B2010E94B1E5E6
:10F3E000811105C0F7014082518262827382F4E08C
:10F3F000EF0EF11C8E149F0439F781E090E00E941B
:10F40000E4100EE8010F013009F431C51E3609F48D
:10F410002DC58091F1129091F212A091F312B0914A
:10F42000F41285369105A105B1050CF420C5809133
:10F430006713909168138D7F892B41F440E855E262
:10F4400060E070E08BEA9FE00E94371680916713BE
:10F4500090916813019741F440E052EC61E070E054
:10F460008BEA9FE00E94371664E670E080E090E04F
:10F470000E94086E8091671390916813892B09F0A0
:10F48000B7C01E3671F08091F1129091F212A091E6
:10F49000F312B091F41285369105A105B1050CF077
:10F4A000A7C061E47CE0CE0107960E940BC965E429
:10F4B00079E0CE0101960E940BC96EE076E1CE01A3
:10F4C00001960E947CC7BC01CE0107960E9443C8EA
:10F4D000CE0101960E949FC8BE01695F7F4F8BEAF3
:10F4E0009FE00E949AD168EB7BE080E090E00E9470
:10F4F000086EBE01695F7F4FCE0101960E9402C96E
:10F50000CE0101960E94051ECE0101960E949FC861
:10F510006CE271E080E090E00E94086E409112166B
:10F5200050911316425051096EE076E1CE010196DA
:10F530000E943C18BE016F5F7F4FCE0107960E946C
:10F540005AC8CE0101960E949FC8BE01695F7F4FD5
:10F55000CE0101960E9402C9BE01695F7F4FCE01B4
:10F5600001960E947CC7BC01CE0107960E9443C849
:10F57000CE0101960E949FC86DE479E0CE0101960C
:10F580000E940BC9BE01695F7F4FCE0101960E94A8
:10F590007CC7BC01CE0107960E9443C8CE010196EC
:10F5A0000E949FC8BE01695F7F4F8BEA9FE00E9467
:10F5B0009AD168EB7BE080E090E00E94086EBE018B
:10F5C000695F7F4FCE0101960E9402C9CE0101966C
:10F5D0000E94051ECE0101960E949FC86CE271E058
:10F5E00080E090E00E94086ECE0107960E949FC8BE
:10F5F000113659F082E891E10E94B3AAD82E64E650
:10F6000070E080E090E00E94086E0E9405C3F12C3B
:10F61000E12C17E2812F0E94CDAD89ED94E10E948B
:10F620009174811124C510932A164FEFE41AF40A3D
:10F630001F5F103479F7EF2831F46FE679E082E844
:10F6400091E10E946BCB10912A1681E6D8120DC071
:10F6500067E47CE182E891E10E94BAD140E150E0A8
:10F66000612F82E891E10E9454CB809187139091A1
:10F670008813019729F4103319F487E280932A162E
:10F680000E9478C580E40E94D7AD0BEA14E093EBAA
:10F69000E92E94E0F92EF80161918F0186E296E15E
:10F6A0000E94C674E016F106B1F70E943F130E9453
:10F6B000A81069E37CE1CE0101960E94F9C84AE0F6
:10F6C00050E06FEF7FEFCE0101960E94FD19CE0151
:10F6D00001960E949FC80E9405C364E670E080E026
:10F6E00090E00E94086EF1E6DF12D2C481E00E9431
:10F6F000262781E00E94202064E670E080E090E010
:10F700000E94086E6091791370917A1380917B1337
:10F7100090917C136093D70D7093D80D8093D90D81
:10F720009093DA0D00917D1310917E1320917F1339
:10F73000309180130093D30D1093D40D2093D50DE9
:10F740003093D60D9B01AC010E94B1E5882381F076
:10F7500083E393EFACE8B4E48093D70D9093D80D96
:10F76000A093D90DB093DA0D90E080E00E9471B0C3
:10F770006091D30D7091D40D8091D50D9091D60DDF
:10F780009B01AC010E94B1E58823C1F080E090E0CC
:10F79000A8ECB1E48093D30D9093D40DA093D50D34
:10F7A000B093D60D80937D1390937E13A0937F1317
:10F7B000B093801390E080E00E9471B0F89482E0F2
:10F7C0008093B0008093B10094E69093B3001092C0
:10F7D000B20080937000789480931F1210922212CE
:10F7E0008091201260E00E94806D69E27CE1CE0190
:10F7F00001960E94F9C84AE050E06FEF7FEFCE011A
:10F8000001960E94FD19CE0101960E949FC861E4F5
:10F810007CE08EE994E10E94E2C5809167139091AB
:10F820006813892B31F46CEF75E08EE994E10E9446
:10F83000E2C58091671390916813019731F466EFE8
:10F8400075E08EE994E10E94E2C580916713909182
:10F850006813029731F460E076E08EE994E10E944B
:10F86000E2C58091A2149091A314892BC1F06EE09F
:10F8700076E18EE994E10E9417C86EE974E1CE0149
:10F8800001960E9402C94AE050E06FEF7FEFCE017F
:10F8900001960E946313CE0101960E949FC8809139
:10F8A000671390916813019709F05CC0CE01079629
:10F8B0000E94B7498B859C85009709F449C0EF8168
:10F8C000F8852081222309F443C0079708F440C03B
:10F8D00066E17CE18EE994E10E941EC8BE01695F89
:10F8E0007F4F8EE994E10E9417C86EE974E1CE0162
:10F8F00001960E9402C9CE0101960E940B13CE010F
:10F9000001960E949FC86DE07CE1CE0101960E94A5
:10F91000F9C848EC50E06FEF7FEFCE0101960E94EE
:10F920004419CE0101960E949FC8BE01695F7F4FB6
:10F93000CE0101960E9402C948EC50E06FEF7FEFC4
:10F94000CE0101960E946313CE0101960E949FC8CA
:10F9500068EE73E080E090E00E94086ECE010796AA
:10F960000E949FC861EF7BE18EE994E10E941EC86E
:10F970006BE379E0CE0101960E940BC96EE076E15F
:10F98000CE0101960E947CC76EE974E10E947CC79B
:10F99000BC018EE994E10E9443C8CE0101960E9409
:10F9A0009FC86EE974E1CE0101960E9402C9CE01A2
:10F9B00001960E940B13CE0101960E949FC861E43C
:10F9C0007CE08EE994E10E94E2C564E670E080E0AC
:10F9D00090E00E94086E83E090E09093F30D809396
:10F9E000F20D8CE40E9406B16B017C0162E370E0D1
:10F9F00080E090E00E94086EA7019601C701B60161
:10FA00000E94B1E58823B9F086E60E9406B16B0139
:10FA10007C0162E370E080E090E00E94086EA70144
:10FA20009601C701B6010E94B1E5882321F010922A
:10FA3000F30D1092F20D8091F20D9091F30D03975A
:10FA400009F02BC36CED7BE1CE0101960E94F9C851
:10FA5000CE0101960E94051ECE0101960E949FC80C
:10FA600083E08093C2140E9405C380ED0E94A9B276
:10FA7000853509F035C38AEA0E94CCB29093C4144C
:10FA80008093C3148CEA0E94CCB29093C6148093E6
:10FA9000C5148EEA0E94CCB29093C8148093C71408
:10FAA00080EB0E94CCB29093D4148093D31482EB59
:10FAB0000E94CCB29093D6148093D51484EB0E940C
:10FAC000CCB29093D8148093D71486EB0E94CCB21A
:10FAD0009093CA148093C91488EB0E94CCB290937F
:10FAE000CC148093CB148AEB0E94CCB29093CE14AA
:10FAF0008093CD148CEB0E94CCB29093D014809361
:10FB0000CF148EEB0E94CCB29093D2148093D11478
:10FB100063EA7BE18EE994E10E941EC80E9411B362
:10FB20000E94CBE00E94EFE30E94CBE020E030E0B7
:10FB300048EC52E40E9443E3AB01BC0122E0CE0159
:10FB400001960E94A7C8BE016F5F7F4FCE01079646
:10FB50000E9402C966EC79E0CE0107960E9466C752
:10FB6000BC018EE994E10E9417C8CE0107960E945D
:10FB70009FC8CE0101960E949FC86EE974E1CE0134
:10FB800001960E9402C9CE0101960E94051ECE0177
:10FB900001960E949FC86DE87BE18EE994E10E9486
:10FBA0001EC86091EB047091EC048091ED0490917B
:10FBB000EE040E94CBE020E030E048EC52E40E94EA
:10FBC00043E3AB01BC0122E0CE0101960E94A7C82D
:10FBD000BE016F5F7F4FCE0107960E9402C966EC9F
:10FBE00079E0CE0107960E9466C7BC018EE994E1D8
:10FBF0000E9417C8CE0107960E949FC8CE010196A9
:10FC00000E949FC86EE974E1CE0101960E9402C96C
:10FC1000CE0101960E94051ECE0101960E949FC84A
:10FC200064E670E080E090E00E94086E8091F20D42
:10FC30009091F30D892BA1F461E08091A6040E94BC
:10FC4000806D60E08091A4040E94806D6091A004AA
:10FC50007091A1048091A2049091A3040E948B1042
:10FC600060E08091A6040E94806D8091EF0488235B
:10FC700031F068EE73E080E090E00E94086E6FE97A
:10FC80007BE08AEA94E10E94E2C582E090E09093F2
:10FC9000F10D8093F00D8091EF04882309F471C376
:10FCA00063E57BE1CE0101960E94F9C84CE251E088
:10FCB0006FEF7FEFCE0101960E946313CE01019694
:10FCC0000E949FC860919E0470919F048091F004EF
:10FCD0009091F1040E94F61384E1C82ED12CE12CFE
:10FCE000F12C10E000E00F5F1F4FC701B6010E942A
:10FCF000086E60919E0470919F048091F004909131
:10FD0000F1040E94F613033011053CF00A3011058E
:10FD10000CF0F7C1892B09F4F7C144E1C40ED11CE2
:10FD2000E11CF11CE0CFC0901D136C2D0C2C000CBD
:10FD3000770B880B990B0E94CBE09B01AC010E94D2
:10FD4000B1E5811133CBE0901E13F0901F13B70182
:10FD50000F2C000C880B990B0E94CBE09B01AC018F
:10FD60000E94B1E5811122CB00912013602F002E5B
:10FD7000000C770B880B990B0E94CBE09B01AC0128
:10FD80000E94B1E5811112CB809021139090221333
:10FD9000A0902313B0902413A5019401C501B401D0
:10FDA0000E94B1E5811102CB609125137091261359
:10FDB00080912713909128139B01AC010E94B1E51B
:10FDC0008111F4CA60913B1370913C1380913D13F3
:10FDD00090913E139B01AC010E94B1E58111E6CAEE
:10FDE0006091671370916813072E000C880B990BB4
:10FDF0000E94CBE09B01AC010E94B1E58111D6CA03
:10FE00006091691370916A13072E000C880B990B8F
:10FE10000E94CBE09B01AC010E94B1E58111C6CAF2
:10FE20006091771370917813072E000C880B990B53
:10FE30000E94CBE09B01AC010E94B1E58111B6CAE2
:10FE400043E04C150CF4B2CA05300CF0AFCA8BEF8E
:10FE5000E816F1040CF0AACA20E030E0A901C501BF
:10FE6000B4010E94C4E087FDA1CAA2CA0CEF809130
:10FE7000EB049091EC04A091ED04B091EE0480931A
:10FE8000F1129093F212A093F312B093F4128091B6
:10FE9000E7049091E804A091E904B091EA0480930A
:10FEA000F5129093F612A093F712B093F812809186
:10FEB000E3049091E404A091E504B091E6048093FA
:10FEC000F9129093FA12A093FB12B093FC1213371D
:10FED00051F160E084E196E10E94EAC760E08EE0C3
:10FEE00096E10E94EAC740911816509119164115E3
:10FEF000510549F08DE093E1009729F0BC0184E1C0
:10FF000096E10E949BB04091121650911316411534
:10FF1000510549F08BE693E1009729F0BC018EE092
:10FF200096E10E949BB08091DF049091E004A09143
:10FF3000E104B091E2048093FD129093FE12A0932D
:10FF4000FF12B09300138091DB049091DC04A09128
:10FF5000DD04B091DE048093011390930213A0930B
:10FF60000313B09304138091D7049091D804A09107
:10FF7000D904B091DA048093051390930613A093EB
:10FF80000713B09308138091D3049091D404A091E7
:10FF9000D504B091D6048093091390930A13A093CB
:10FFA0000B13B0930C1390E080E00E9471B0E4EF6B
:10FFB000FDE0AFE3B3E141915191619171914D93B6
:10FFC0005D936D937D934EE0EC31F407A1F766E508
:10FFD0007CE1CE0101960E94F9C8CE0101960E94F3
:10FFE000051ECE0101960E949FC823EBA22E24E09D
:10FFF000B22E39E2832E33E1932EF12CE12C809145
:020000021000EC
:10000000B3049091B4048E159F054CF1F5018191D4
:1000100091915F01F401819391934F0180917E0E44
:100020008823C9F06BE379E082E891E10E94C4CCB7
:100030004AE050E0B70182E891E10E9477CC60E4A9
:1000400079E082E891E10E94C4CCF5013297808189
:1000500091810E94B1CCFFEFEF1AFF0AD0CF02309E
:1000600008F0E5C990E080E00E9471B0E0C98430FA
:1000700009F0DECA64E579E082E891E10E94C4CC2F
:1000800040E150E0612F82E891E10E9454CBD0CA58
:1000900080E00E94262780E02DCB86E00E941CC3D2
:1000A000BC0190E080E00E94C9E02AE037ED43EA1D
:1000B0005CE30E942AE123E333E948E853E40E9429
:1000C00064E220E030E048E453E40E94C4E087FFAB
:1000D000C7CC82E090E09093AA048093A904C0CC9E
:1000E00066EB7BE1CE0101960E94F9C8CE01019634
:1000F0000E940B13CE0101960E949FC81092A80483
:100100008FCD892B09F0EBC18091F0049091F1041F
:100110008B30910509F093C180913515909136157A
:10012000A0913715B09138158093EC0D9093ED0D9B
:10013000A093EE0DB093EF0D809131159091321593
:10014000A0913315B09134158093E80D9093E90D8B
:10015000A093EA0DB093EB0D4091EC0D5091ED0D95
:100160006091EE0D7091EF0D21E0CE0101960E949D
:10017000A7C86DEB76E0CE0107960E940BC9BE01C1
:100180006F5F7F4FCE0107960E947CC7BC018EE94E
:1001900094E10E9443C8CE0107960E949FC8CE01F9
:1001A00001960E949FC84091E80D5091E90D609121
:1001B000EA0D7091EB0D21E0CE0101960E94A7C8D7
:1001C00060E878E0CE0107960E940BC9BE016F5F20
:1001D0007F4FCE0107960E947CC7BC018EE994E157
:1001E0000E9417C8CE0107960E949FC8CE010196B3
:1001F0000E949FC868E578E08EE994E10E940DC8EE
:1002000061E47CE0CE0101960E940BC944E150E01C
:1002100070E060E0CE0101960E94FD19CE010196CA
:100220000E949FC8C090EC0DD090ED0DE090EE0DB7
:10023000F090EF0D20E030E0A901C701B6010E9467
:100240004CE420E030E040E05FE387FD18C1C701E7
:10025000B6010E9465E20E94EFE3AB01BC01CE0152
:1002600001960E94ECC5BE016F5F7F4F88E994E163
:100270000E945AC8CE0101960E949FC860E087E0A4
:100280000E94E8AD68E974E186E296E10E949AD1A5
:100290006FED86E296E10E947DCB66E878E086E22B
:1002A00096E10E94C4CC6091E80D7091E90D8091B7
:1002B000EA0D9091EB0D0E94EFE34AE050E086E2F8
:1002C00096E10E9477CC68E578E086E296E10E94AC
:1002D000C4CC64E670E080E090E00E94086EC090BC
:1002E000EC0DD090ED0DE090EE0DF090EF0D20E0D4
:1002F00030E040EF51E4C701B6010E944CE464E4F1
:100300007BE187FF28C020E030E040ED51E4C701E9
:10031000B6010E944CE487FDB7C064E37BE1CE01E7
:1003200001960E94F9C84AE050E06FEF7FEFCE01DE
:1003300001960E946313CE0101960E949FC880918E
:10034000EF04882331F06CED75E080E090E00E94CE
:10035000086E64E27BE1CE0101960E94F9C84AE092
:1003600050E06FEF7FEFCE0101960E946313CE0144
:1003700001960E949FC862E370E080E090E00E94D6
:10038000086E65E77BE18EE994E10E941EC86BE38D
:1003900079E0CE0101960E940BC96EE076E1CE01B4
:1003A00001960E947CC76EE974E10E947CC7BC0183
:1003B0008EE994E10E9443C8CE0101960E949FC835
:1003C0006EE974E1CE0101960E9402C9CE01019648
:1003D0000E940B13CE0101960E949FC861E67BE14B
:1003E0008EE994E10E941EC86EE974E1CE01019687
:1003F0000E9402C9CE0101960E940B13CE01019604
:100400000E949FC861E47CE08EE994E10E94E2C50D
:1004100062960FB6F894DEBF0FBECDBFDF91CF91CD
:100420001F910F91FF90EF90DF90CF90BF90AF9012
:100430009F908F907F906F905F904F90089586313E
:10044000910509F469CE0C9709F086CE8091DF0DF5
:100450009091E00DA091E10DB091E20D8093EC0D33
:100460009093ED0DA093EE0DB093EF0D8091DB0D09
:100470009091DC0DA091DD0DB091DE0D65CEC70130
:10048000B6010E9464E2E7CE20E030E040EB51E4A8
:10049000C701B6010E944CE466E17BE187FF5BCFB8
:1004A00067E07BE1CE0101960E94F9C84AE050E086
:1004B0006FEF7FEFCE0101960E946313CE0101968C
:1004C0000E949FC88091EF04882331F06CED75E0A5
:1004D00080E090E00E94086E69EF7AE13CCF0E94D4
:1004E0003F136EE170E080E090E00E94086E0E9491
:1004F000D8B46B017C0164E670E080E090E00E947B
:10050000086E6DEB76E08EE994E10E94E2C521E091
:10051000B701A601CE0101960E94A7C8BE016F5F78
:100520007F4F8EE994E10E9417C8CE0101960E9488
:100530009FC86EE974E1CE0101960E9402C94AE0AB
:1005400050E070E060E0CE0101960E94FD19CE01FE
:1005500001960E949FC880919D04882379F0809124
:10056000FB04882359F06FED86E296E10E947DCB73
:1005700065E079E086E296E10E94C4CC65EE76E023
:100580008EE994E10E940DC8C092EC0DD092ED0D61
:10059000E092EE0DF092EF0D20E030E040EF51E4FC
:1005A000C701B6010E944CE469EE7AE187FF28C0DA
:1005B00020E030E040ED51E4C701B6010E944CE478
:1005C00087FD3EC069ED7AE1CE0101960E94F9C82F
:1005D0004AE050E06FEF7FEFCE0101960E94631377
:1005E000CE0101960E949FC88091EF04882331F0CC
:1005F0006CED75E080E090E00E94086E69EC7AE1B5
:10060000CE0101960E94F9C84AE050E06FEF7FEFFB
:10061000CE0101960E946313CE0101960E949FC8ED
:100620006CE271E080E090E00E94086E8091EF043F
:10063000882309F4A6CE68EE73E080E090E09FCEB8
:1006400020E030E040EB51E4C701B6010E944CE4E9
:100650006BEB7AE187FFD4CF6CEA7AE1CE010196A9
:100660000E94F9C84AE050E06FEF7FEFCE0101969B
:100670000E946313CE0101960E949FC88091EF04EF
:10068000882331F06CED75E080E090E00E94086E08
:100690006EE97AE1B5CFBF92CF92DF92EF92FF92EF
:1006A0000F931F93CF93DF93CDB7DEB762970FB64B
:1006B000F894DEBF0FBECDBF8C016B0161E47CE01E
:1006C0000E940BC910929C0D61E47CE0CE010D9656
:1006D0000E940BC9FF24F39482E891E10E94D5AAFD
:1006E00020919C0D181619067CF521112DC082E869
:1006F00091E10E94B3AA8A3009F07FC089899A8962
:10070000892B09F482C0F0929C0D65E879E0CE0156
:1007100007960E940BC9BE01635F7F4FCE0107960B
:100720000E947CC7BC01CE0101960E9402C9CE0185
:1007300001960E94051ECE0101960E949FC8CE011F
:1007400007960E949FC861C0F12CE12CBB24B39492
:10075000222309F461C089899A89019709F045C06B
:1007600065E577E0CE0101960E940BC9BE016F5F7F
:100770007F4FCE010D960E944BC7F12C811115C001
:100780006AE079E0CE0107960E940BC9BE01695F5D
:100790007F4FCE010D960E944BC7FF24F394811129
:1007A000F12CCE0107960E949FC8CE0101960E94AF
:1007B0009FC8FF20A1F050E040E0BE01635F7F4F83
:1007C000CE0101960E943C18BE016F5F7F4F8AEAFE
:1007D00094E10E945AC8CE0101960E949FC864E12C
:1007E00070E080E090E00E94086EBE01635F7F4F82
:1007F000CE0101960E94F0C891C08D3009F47ECFE1
:10080000682FCE010D960E94EAC76AE070E080E092
:1008100090E00E94086E60CF8BEA9FE00E94D5AA0C
:100820001816190614F58BEA9FE00E94B3AA8A30C5
:10083000A9F08D3099F090919C0D91110FC0682F07
:10084000CE010D960E94EAC78FEFE81AF80A65E01C
:1008500070E080E090E00E94086EDECF89899A897E
:10086000892BA9F3B0929C0DF2CF64E170E080E097
:1008700090E00E94086EEF28D1F189899A89892B2E
:10088000B1F180917E0E882361F16BE379E0CE01B6
:1008900001960E940BC9BE016F5F7F4FCE010D967E
:1008A0000E944BC7F82ECE0101960E949FC8F110FE
:1008B00018C06EE879E082E891E10E94C4CCBE01E4
:1008C000635F7F4FCE0101960E9402C9BE016F5F38
:1008D0007F4F82E891E10E94A8D1CE0101960E944B
:1008E0009FC864E170E080E090E00E94086E898912
:1008F0009A8920919C0D211130CF009709F02DCFBE
:1009000064E670E080E090E00E94086E0E943B6E1A
:1009100061E47CE0CE0101960E940BC9CE010D96E8
:100920000E949FC8BE016F5F7F4FC8010E9493C89D
:10093000CE0101960E949FC8F80184819581892B80
:1009400079F4B601CE0101960E94736ABE016F5F11
:100950007F4FC8010E9493C8CE0101960E949FC894
:10096000F80184819581892B79F4B601CE01019635
:100970000E940B69BE016F5F7F4FC8010E9493C840
:10098000CE0101960E949FC8C80162960FB6F894E6
:10099000DEBF0FBECDBFDF91CF911F910F91FF90B2
:1009A000EF90DF90CF90BF9008954F925F926F923B
:1009B0007F929F92AF92BF92CF92DF92EF92FF927F
:1009C0000F931F93CF93DF93CDB7DEB7A8970FB6E2
:1009D000F894DEBF0FBECDBFBC0186EB94E10E9450
:1009E00043C80E949EC462EC79E0CE0101960E9449
:1009F0000BC9BE016F5F7F4F86EB94E10E944BC72E
:100A0000182FCE0101960E949FC8112309F4F8C047
:100A10008091C0149091C1144097C0F0F12C8F2D9B
:100A2000A8960FB6F894DEBF0FBECDBFDF91CF9171
:100A30001F910F91FF90EF90DF90CF90BF90AF90FC
:100A40009F907F906F905F904F90089542E050E0AC
:100A50006CEB74E1CE0101960E943C18BE016F5F01
:100A60007F4F88E994E10E945AC8CE0101960E9406
:100A70009FC868E974E1CE0101960E9402C9CE01C7
:100A800001960E94051ECE0101960E949FC888E92A
:100A900094E10E9454C620E030E048EC52E40E9409
:100AA0002AE10E94EFE3AB01BC014093EB045093B9
:100AB000EC046093ED047093EE04CE0101960E9465
:100AC000ECC5CE0101960E94051ECE0101960E9442
:100AD0009FC86091EB047091EC048091ED049091BB
:100AE000EE048B019C0100591F452140310901345E
:100AF0001C4921053105C8F165E979E0CE0101966F
:100B00000E940BC968E974E1CE0101960E947CC77E
:100B100068EA79E00E9466C7BC018EE994E10E9410
:100B200043C8CE0101960E949FC86BE379E0CE01D5
:100B300001960E940BC96EE974E1CE0101960E94F4
:100B40007CC7BC01CE0145960E9402C9CE014596E4
:100B50000E940B13CE0145960E949FC8CE010196BC
:100B60000E949FC81092000548C21A821982FE0195
:100B7000339626E0DF011D922A95E9F70E94CBE02B
:100B800020E030E048EC52E40E9443E38E010F5F26
:100B90001F4F22E047E00E9420DCBC018EE994E177
:100BA0000E9445C668EB79E0CE0145960E940BC9CC
:100BB0006EE974E1CE0145960E947CC765EC79E050
:100BC0000E9466C7BC018EE994E10E9443C8CE0131
:100BD00045960E949FC88091EB049091EC04A091EF
:100BE000ED04B091EE048093F1129093F212A09371
:100BF000F312B093F41290E080E00E9471B095CFB0
:100C00008E010B5E1F4F64E479E1C8010E94F9C8B0
:100C1000B80186EB94E10E944BC7FF24F394811145
:100C200016C06FE379E1CE0101960E94F9C8BE01BA
:100C30006F5F7F4F86EB94E10E944BC7FF24F394D4
:100C4000811101C0F12CCE0101960E949FC8C801FC
:100C50000E949FC8FF2009F471C042E050E06CEB95
:100C600074E1CE0101960E943C18BE016F5F7F4F78
:100C700088E994E10E945AC8CE0101960E949FC85B
:100C80006AE379E1CE0101960E94F9C8BE016F5F67
:100C90007F4F86EB94E10E944BC7E82ECE01019670
:100CA0000E949FC8EE2099F044E050E06CEB74E1A4
:100CB000CE0101960E943C18BE016F5F7F4F88E90C
:100CC00094E10E945AC8CE0101960E949FC888E90B
:100CD00094E10E945FC66730710558F570931D0E50
:100CE00060931C0E80911C0E90911D0E90937813B2
:100CF0008093771390E080E00E9471B06BE379E01D
:100D0000CE0101960E940BC96EE974E1CE010196F5
:100D10000E947CC7BC01C8010E9402C9C8010E9490
:100D20000B13C8010E949FC8CE0101960E949FC864
:100D300076CE10921D0E10921C0ED4CF65E379E191
:100D4000CE0101960E94F9C8BE016F5F7F4F86EB0E
:100D500094E10E944BC7F82ECE0101960E949FC8D5
:100D6000FF20A1F126E030E044E050E06CEB74E1BC
:100D7000CE0101960E941CC9BE016F5F7F4F88E9BA
:100D800094E10E945AC8CE0101960E949FC888E94A
:100D900094E10E945FC670936A1360936913709325
:100DA000F1046093F0046CEB74E1CE0101960E94B3
:100DB00002C9CE0101960E94051ECE0101960E9435
:100DC0009FC890E080E00E9471B0CCCE6EE279E1E5
:100DD000CE0101960E94F9C8BE016F5F7F4F86EB7E
:100DE00094E10E944BC7F82ECE0101960E949FC845
:100DF000FF20A1F146E050E06CEB74E1CE010196DA
:100E00000E943C18BE016F5F7F4F88E994E10E9409
:100E10005AC8CE0101960E949FC880919C1490915F
:100E20009D14892B61F088E994E10E9454C6609377
:100E3000A0047093A1048093A2049093A3046CEB8C
:100E400074E1CE0101960E9402C9CE0101960E9472
:100E5000051ECE0101960E949FC884CE6AEC79E0FF
:100E6000CE0101960E940BC9BE016F5F7F4F86EBDA
:100E700094E10E944BC7F82ECE0101960E949FC8B4
:100E8000FF2009F4BDC06AE279E1CE0101960E941B
:100E9000F9C8BE016F5F7F4F86EB94E10E944BC79C
:100EA000F82ECE0101960E949FC8FF20D1F184E068
:100EB00090E00E942F106093CF047093D004809331
:100EC000D1049093D2046AE179E18EE994E10E9421
:100ED0001EC84091CF045091D0046091D10470910C
:100EE000D20422E0CE0101960E94A7C8BE016F5F26
:100EF0007F4F8EE994E10E9417C8CE0101960E94AF
:100F00009FC88091CF049091D004A091D104B0915A
:100F1000D2048093151390931613A0931713B093D4
:100F200018136DEC79E0CE0101960E940BC9BE0149
:100F30006F5F7F4F86EB94E10E944BC7F82ECE0186
:100F400001960E949FC8FF20F1F18AE090E00E9484
:100F50002F106093CB047093CC048093CD049093B6
:100F6000CE0469E079E18EE994E10E941EC84091C7
:100F7000CB045091CC046091CD047091CE0422E05A
:100F8000CE0101960E94A7C8BE016F5F7F4F8EE918
:100F900094E10E9417C8CE0101960E949FC88091DB
:100FA000CB049091CC04A091CD04B091CE04809359
:100FB000191390931A13A0931B13B0931C1390E072
:100FC00080E00E9471B06BE379E0CE0101960E944F
:100FD0000BC96EE974E1CE0101960E947CC7BC0189
:100FE000C8010E9402C9C8010E940B13C8010E94D7
:100FF0009FC8CE0101960E949FC8FF24F3940FCD95
:1010000064ED78E0CE0101960E940BC9BE016F5FCE
:101010007F4F86EB94E10E944BC7F82ECE010196DC
:101020000E949FC8FF2009F4BDC08091C014909118
:10103000C1140797F8F046E050E06CEB74E1CE0184
:1010400001960E943C18BE016F5F7F4F88E994E1D2
:101050000E945AC8CE0101960E949FC888E994E177
:101060000E9454C66093F6047093F7048093F804CA
:101070009093F90480918D0490918E0499270E9499
:10108000F2112DE038E643E55BE30E942AE16B01B3
:101090007C012091290530912A0540912B05509122
:1010A0002C050E94C4E018160CF460C06091110574
:1010B00070911205809113059091140520E030E0A5
:1010C00048EC52E40E942AE16B017C0120E030E010
:1010D000A9010E94C4E0181634F0C12CD12CF8EA02
:1010E000EF2EF1E4FF2EC092F604D092F704E092C6
:1010F000F804F092F904C0922513D0922613E092DE
:101100002713F092281380917E0E882381F067EFD9
:1011100078E182E891E10E94BAD16091F604709181
:10112000F7048091F8049091F9040E9468CC90E053
:1011300080E00E9471B06DEE78E18EE994E10E944A
:101140001EC84091F6045091F7046091F804709124
:10115000F90422E0CE0101960E94A7C8BE016F5F8C
:101160007F4F8EE994E10E9417C8A6C020913D05EB
:1011700030913E0540913F0550914005C701B601B1
:101180000E944CE487FF05C0C701B6010E943FAF33
:1011900095CF609125057091260580912705909146
:1011A00028058CCF69EE78E1CE0101960E94F9C83E
:1011B000BE016F5F7F4F86EB94E10E944BC7F82E14
:1011C000CE0101960E949FC8FF2009F47DC0709057
:1011D0008B0460E0872D0E94806DE9E1AE2EB12C7A
:1011E000C12CD12C7601872D0E94C06DBC01990FB6
:1011F000880B990B0E94CBE09B01AC01C701B601A3
:101200000E9465E26B017C016AE070E080E090E0A2
:101210000E94086EB1E0AB1AB10829F720E030E077
:1012200040EA50E4C701B6010E942AE120E030EC18
:101230004FE754E40E9443E320E030E048EC51E4FF
:101240000E9443E36093F2047093F3048093F404E8
:101250009093F50460933B1370933C1380933D137C
:1012600090933E1390E080E00E9471B066ED78E1CB
:101270008EE994E10E941EC84091F2045091F3045B
:101280006091F4047091F50422E0CE0101960E9471
:10129000A7C8BE016F5F7F4FC8010E9402C965E207
:1012A00078E0C8010E9466C7BC018EE994E10E9403
:1012B00017C8C8010E949FC8CE0101960E949FC80E
:1012C0006EE974E10C9430936AED78E0CE010196FA
:1012D0000E940BC9BE016F5F7F4F86EB94E10E94B5
:1012E0004BC7F82ECE0101960E949FC8FF2009F43B
:1012F00041C080912013082E000C990B0197039791
:1013000090F589E390E00E94F2112AE137E64CE97A
:1013100050E40E942AE1609321137093221380937A
:1013200023139093241390E080E00E9471B065EB4A
:1013300078E18EE994E10E941EC8409121135091FA
:101340002213609123137091241322E0CE010196A1
:101350000E94A7C8BE016F5F7F4FC8010E9402C9EB
:1013600062ED79E09ECF6FE878E18EE994E10E942A
:101370001EC8A6CF6BE878E1CE0101960E94F9C89D
:10138000BE016F5F7F4F86EB94E10E944BC7F82E42
:10139000CE0101960E949FC8FF2009F439C126E0C2
:1013A00030E044E050E06CEB74E1CE0101960E9425
:1013B0001CC9BE016F5F7F4F88E994E10E945AC843
:1013C000CE0101960E949FC888E994E10E945FC601
:1013D0006B015B016EEE75E0CE0101960E940BC9B8
:1013E000BE016F5F7F4F8CEB94E10E9415C7AC018B
:1013F0004F5F5F4F6CEB74E1C8010E943C18B8016D
:1014000088E994E10E945AC8C8010E949FC8CE0191
:1014100001960E949FC89090890488E994E10E94F7
:1014200054C62B013C0180917E0E8823B9F061EDFA
:1014300074E182E891E10E94BAD14AE050E0B6013D
:1014400082E891E10E9477CC6EE277E082E891E158
:101450000E94C4CCC301B2010E9468CC692DC801AE
:101460000E94B67118870F831D821E82198289E03F
:101470008A8381E08B838C831C8A1B8ACE01019630
:101480000E940B71CE0101960E94AE6FCE010196B3
:101490000E94C1C30E8110E00B30110514F00AE068
:1014A00010E0EBE5CE16D10408F44FC074EFC72E60
:1014B0007DE0D72E5601412C512C3201F12CE12C2C
:1014C0000E151F05B9F06E2DCE0101960E949F707A
:1014D0009B01AC01D5012D933D934D935D935D012F
:1014E000C301B2010E9465E22B013C01BFEFEB1A80
:1014F000FB0AE6CFB7010F2C000C880B990B0E945A
:10150000CBE09B01AC01C301B2010E9443E32B017C
:101510003C0110E000E0E016F106B9F1F60121917E
:101520003191419151916F015F01F4E0AF1AB1081F
:10153000C301B2010E9464E2D5016D937D938D9346
:101540009C9313970F5F1F4FE6CF1A141B040CF0E8
:1015500040C00A151B050CF0860101501109602FCF
:10156000CE0101960E949F709B01AC01000F111FDC
:10157000000F111F0C50124FC301B2010E9464E210
:10158000F8016083718382839383E4EFFDE0AFE32E
:10159000B3E18CE19EE041915191619171914D9344
:1015A0005D936D937D938E179F07A9F790E080E080
:1015B0000E9471B06AE678E18EE994E10E941EC84B
:1015C00044E050E06CEB74E1CE0101960E943C18BF
:1015D000C5CDA114B104C9F634EFE32E3DE0F32EDE
:1015E0000A151B0591F26A2DCE0101960E949F708B
:1015F0009B01AC01C301B2010E9464E2D7016D936B
:101600007D938D939D937D01BFEFAB1ABB0AE8CF0D
:1016100069E377E0CE0101960E940BC9BE016F5FBE
:101620007F4F86EB94E10E944BC7F82ECE010196C6
:101630000E949FC8FF2009F416C127E030E046E071
:1016400050E06CEB74E1CE0101960E941CC9BE0112
:101650006F5F7F4F88E994E10E945AC8CE010196DE
:101660000E949FC888E994E10E945FC67B01609355
:1016700020138CEB94E10E946AC66EE277E0CE0103
:1016800001960E940BC9BE016F5F7F4F8CEB94E106
:101690000E9415C7AC014F5F5F4F6CEB74E1C8014E
:1016A0000E943C18C8010E9454C660932113709395
:1016B00022138093231390932413C8010E949FC880
:1016C000CE0101960E949FC869E578E18EE994E118
:1016D0000E941EC8E4E0EE16F10404F5F2E0EF16F5
:1016E000F1040CF098C0E114F10419F1EA94EF2828
:1016F00009F46AC060912013062E000C770BC80114
:101700000E9419C660EE79E0CE0101960E940BC9D5
:10171000B801CE0101960E947CC749C084E0E8165A
:10172000F10441F768E378E18EE994E10E948FC704
:101730006DC020E030E0A901609121137091221367
:1017400080912313909124130E94C4E0181664F032
:1017500080E090E0A0E8BFE38093211390932213F0
:10176000A0932313B09324132091211330912213BB
:10177000409123135091241360E070E080EA90E4DC
:101780000E9443E3AB01BC0122E0C8010E94A7C84C
:1017900065ED79E0CE0101960E940BC9B801CE013A
:1017A00001960E947CC764EF77E00E9466C7BC0187
:1017B0008EE994E10E9417C8CE0101960E949FC84D
:1017C000C8010E949FC822C06BE478E18EE994E1D1
:1017D0000E948FC720E030E048E453E46091211379
:1017E0007091221380912313909124130E94C4E0DE
:1017F000181664F080E090E4ACE1B5E48093211326
:1018000090932213A0932313B093241390E080E0CD
:101810000E9471B055CD6FE378E18EE994E10E94AA
:101820008FC78AE08E9DB0018F9D700D1124CE016F
:1018300001960E9419C6BE016F5F7F4FC8010E94CA
:1018400002C96DEE77E0C8010E9466C7BC018EE94F
:1018500094E10E9417C8C8010E949FC8CE0101965A
:101860000E949FC8B7CF67EE79E0CE0101960E9433
:101870000BC9BE016F5F7F4F86EB94E10E944BC79F
:10188000F82ECE0101960E949FC8FF2009F4C2C025
:1018900027E030E046E050E06CEB74E1CE010196C9
:1018A0000E941CC9BE016F5F7F4F88E994E10E94CE
:1018B0005AC8CE0101960E949FC888E994E10E940F
:1018C0005FC660931D138CEB94E10E946AC688E9A1
:1018D00094E10E945FC6611571058105910509F0CB
:1018E0006DC085E090E090931F1380931E1390E0ED
:1018F00080E00E9471B067E278E18EE994E10E9495
:101900001EC880911D1383302CF56CE178E18EE9BF
:1019100094E10E948FC760911E1370911F13CE0136
:1019200001960E9419C6BE016F5F7F4FC8010E94D9
:1019300002C968E077E0C8010E9466C7BC018EE971
:1019400094E10E9417C8C8010E949FC8CE01019669
:101950000E949FC880911D1383300CF4B1CC60911C
:101960001E1370911F13CE0183960E9419C66091B9
:101970001D13062E000C770BC8010E9419C660EEDD
:1019800079E0CE0101960E940BC9B801CE01019603
:101990000E947CC7BE016D5D7F4F0E947CC7BC0169
:1019A0008EE994E10E9417C8CE0101960E949FC85B
:1019B000C8010E949FC8CE01839680CC613071051A
:1019C0008105910519F489E190E08DCF6EE277E011
:1019D000CE0101960E940BC9BE016F5F7F4F8CEB59
:1019E00094E10E9415C7AC014F5F5F4F6CEB74E14F
:1019F000C8010E943C18C8010E945FC670931F1363
:101A000060931E13C8010E949FC8CE0101960E94D8
:101A10009FC86DCF6EEE79E0CE0101960E940BC992
:101A2000BE016F5F7F4F86EB94E10E944BC7F82E9B
:101A3000CE0101960E949FC8FF2009F464C08091E6
:101A40008704909188040E94E4126093D3047093F9
:101A5000D4048093D5049093D604609309137093B3
:101A60000A1380930B1390930C1380E090E5A3EC82
:101A7000B7E48093DB049093DC04A093DD04B0937F
:101A8000DE048093011390930213A0930313B09389
:101A9000041380917E0E882381F06EEF77E182E857
:101AA00091E10E94BAD16091D3047091D4048091E5
:101AB000D5049091D6040E9468CC90E080E00E940A
:101AC00071B04091D3045091D4046091D5047091C9
:101AD000D60422E0C8010E94A7C862EF79E0CE01D7
:101AE00001960E940BC9B801CE0101960E947CC7E5
:101AF000BC018EE994E10E9443C8CE0101960E9488
:101B00009FC8C801DBCB6DEF79E0CE0101960E9442
:101B10000BC9BE016F5F7F4F86EB94E10E944BC7FC
:101B2000F82ECE0101960E949FC8FF2009F488C0BC
:101B30008091C0149091C1140497F8F044E050E0F3
:101B40006CEB74E1CE0101960E943C18BE016F5F00
:101B50007F4F88E994E10E945AC8CE0101960E9405
:101B60009FC888E994E10E9454C66093DF04709393
:101B7000E0048093E1049093E2048091DF0490916B
:101B8000E004A091E104B091E2048093FD129093EF
:101B9000FE12A093FF12B093001380917E0E882353
:101BA00091F065EE77E182E891E10E94BAD160910F
:101BB000DF047091E0048091E1049091E20442E03E
:101BC00050E00E9466CC80918704909188040E9426
:101BD000E4126093D7047093D8048093D90490934F
:101BE000DA046093051370930613809307139093A0
:101BF000081380917E0E882381F06BED77E182E8F7
:101C000091E10E94BAD16091D7047091D80480917B
